:020000040800F2
:10000000F0FF0010F99B06086DF20008A9D504085E
:10001000999C0608999C0608999C06080000000017
:1000200000000000000000000000000069F200086D
:1000300065F200080000000061F20008759C0408E9
:10004000999C0608999C0608999C0608999C0608A4
:10005000999C0608999C0608ADE60408D9E70408AF
:100060009DE7040861E7040825E70408C180060845
:10007000B1800608A1800608918006087D800608E8
:100080006980060855800608999C0608999C060810
:10009000999C0608999C0608999C0608E9E60408BC
:1000A00085870408058804087587040829880408DA
:1000B000F9870408E9870408D98704083D8A0608F7
:1000C000458A0608318A0608398A0608999C060876
:1000D000999C060885A00408C99F04080D9F040880
:1000E00071E60408999C06088909010865870408D7
:1000F0009587040855870408B987040841800608D5
:10010000999C06081D460608C9870408999C06089C
:10011000519E0408959D0408150904080109040866
:100120002D8006081980060805800608F17F06085C
:10013000DD7F0608999C0608999C0608999C06088C
:10014000999C0608999C0608999C0608E5EB00080E
:10015000C97F0608B57F0608A17F0608D99C040858
:10016000258A06082D8A0608999C0608999C060887
:10017000999C0608999C0608999C0608999C060873
:08018000999C0608999C0608F1
:08018800A89706000100000029
:100190000E02010002000000045C0020645C0020EC
:1001A00000000000E809000814020100050000003A
:1001B000303E0020685C002000000000EA090008D2
:1001C0001302010004000000BC240020705C002029
:1001D00000000000F00900080D1001007000000090
:1001E000A85A0020745C002000000000EDFB03080A
:1001F0000400080080000000E8590020E45C0020B2
:1002000000000000000000000902010001000000E1
:1002100090590020645D002000000000F4090008EF
:10022000FD0101002400000034590020685D002019
:1002300000000000576B0408FB01010001000000F2
:10024000F05800208C5D0020000000004D8805085B
:10025000FC01010009000000BC570020905D002057
:100260000000000055880508F701010006000000A5
:10027000B05700209C5D002000000000F609000837
:10028000F901010004000000AC570020A45D00202B
:1002900000000000016C0408160215003F00000079
:1002A00050310020A85D002000000000F187050803
:1002B0003400010010000000A0560020E85D00207E
:1002C00000000000D19302081102010008000000A4
:1002D00078560020F85D002000000000FC090008AE
:1002E000121201000400000070560020005E002081
:1002F00000000000040A000818200100320000007D
:100300003C560020045E002000000000E19005083B
:1003100012200100110000005C550020385E002012
:1003200000000000080A0008000201000B000000A5
:10033000985200204C5E002000000000A5880508AF
:10034000FF1101000600000040520020585E00200E
:1003500000000000E1870508081203000F000000FC
:100360004C520020605E002000000000F587050868
:10037000FA01010003000000384C0020705E0020EC
:10038000000000007D8805080A80010028000000A8
:10039000004C0020745E00200000000035150208AB
:1003A000061001001C000000343100209C5E00207B
:1003B00000000000E18805080202010003000000BF
:1003C000A8280020B85E0020000000000000000007
:1003D0000C0201000400000088280020BC5E002000
:1003E00000000000AD880508110001000C000000AD
:1003F00056400020C05E0020000000002DF40308DD
:10040000FE010100140000005C3F0020CC5E0020D3
:100410000000000081870508FD070100760000004C
:1004200080B40020F8B40020000000001579010815
:10043000261001000E00000080B5002070B50020DD
:1004400000000000451C01080B3001001A000000EC
:1004500038AF0020C0B50020000000001C0A0008D2
:100460001F3001002400000074AE0020DCB5002025
:1004700000000000380A0008050201000400000026
:1004800004B1002000B60020000000005C0A000853
:10049000030101000A000000B8AE002004B60020ED
:1004A00000000000DD160108220201001C0100000E
:1004B0005CCD002014D000200000000099900508B9
:1004C0000C200600CC000000D8CB002030D100204A
:1004D0000000000081F20308010201000B0000008F
:1004E0007CCB0020FCD1002000000000958805088E
:1004F0001B0201001000000050CB002008D2002099
:1005000000000000CD8805081B1001000C00000051
:1005100004B8002018D2002000000000897F0108E4
:1005200021020100F000000084B6002024D2002047
:10053000000000005DA1010823120100100000006E
:1005400058C8002014D3002000000000600A0008F2
:10055000371001002E000000C0CA002024D3002064
:1005600000000000700A00081610010006000000DC
:1005700050C8002054D30020000000009E0A00084C
:100580002F10010022000000F0CF00205CD30020DB
:1005900000000000A40A00081E000100090000007D
:1005A00078C7002080D3002000000000C60A0008A1
:1005B0000510010006000000BCC700208CD30020FD
:1005C00000000000D00A0008F5810100680000006A
:1005D00014B6002094D3002000000000D991010837
:1005E0002320010010000000FCC70020FCD30020E5
:1005F0000000000049160208F62101000C0000006E
:1006000040DF002030E1002000000000D80A000890
:100610001C0202001C000000E4DE002080E100203B
:1006200000000000CD9105082820010018000000FE
:1006300000DF00209CE1002000000000352F0208B0
:100640000412010002000000F0E00020B4E10020EC
:1006500000000000E40A00080F0201000100000091
:10066000ECE00020B8E1002000000000E60A0008ED
:100670001400010004000000DCDE0020BCE10020CA
:1006800000000000E80A0008012001000C00000042
:100690001CD70020C0E1002000000000EC0A000888
:1006A0000EF003009E01000004D50020CCE10020E4
:1006B000000000001994020813000100040000006B
:1006C000D4DA00206CE3002000000000F80A0008E3
:1006D000010101000400000050D4002070E300205C
:1006E0000000000000000000000101000400000004
:1006F00048D4002074E3002000000000FC0A000839
:10070000020101000300000044D4002078E300202F
:1007100000000000BDF20308190001000500000000
:10072000A0ED00206CEE002000000000000B00088F
:100730001A0001000E00000028ED002074EE0020D9
:1007400000000000060B0008203201000A00000033
:10075000F4EB002084EE002000000000F593020876
:1007600015001000700000008CE9002090EE0020C1
:1007700000000000000000002A00080060000000E7
:10078000E8ED002000EF002000000000A99302081F
:100790002C0004001000000070EF002060EF00202B
:1007A00000000000819102082B00120024000000CC
:1007B000A4EF002080EF0020000000005591020807
:1007C00029201400780000002CE70020C8EF00204A
:1007D00000000000000000001902010010000000ED
:1007E00060E6002040F00020000000008588050839
:1007F000030001000100000004F4002038F4002090
:100800000000000000000000031201003D00000095
:10081000ACF300203CF4002000000000140B0008A2
:1008200025201E002C01000010F100207CF4002087
:100830000000000000000000101001000200000095
:10084000A4F00020A8F5002000000000520B0008D2
:10085000F821010006000000ECF00020ACF50020BB
:1008600000000000540B0008020001000C00000012
:1008700044FE0020D8FE0020000000000000000020
:10088000290201004000000094F80020E4FE00204E
:10089000000000005A0B00080A02010014000000CA
:1008A00004F8002044FF0020000000004DF203087F
:1008B00028020400040000007C03012058050120E8
:1008C00000000000C9880508270204000400000099
:1008D000780301205C05012000000000BD880508A8
:1008E0001F02080010000000D40001206005012054
:1008F00000000000998705081A0201003C00000072
:1009000098000120700501200000000051910508A9
:10091000381001000100000078FF0020AC05012024
:10092000000000009A0B00082700010004000000EE
:100930006C06012074070120000000009C0B0008D9
:100940000B1201003C0000002C0901208C1A012030
:1009500000000000A00B00080D12010014000000B0
:10096000E0150120C81A012000000000DC0B00087F
:100970000702010002000000741A0120DC1A0120A5
:1009800000000000F00B00081D020200060000003D
:100990003C1A0120E01A01200000000000000000C5
:1009A000060203000C000000481A0120E823012081
:1009B0000000000059920508390001000500000000
:1009C000541A0120F4230120000000006D8805085E
:1009D00010020100010000009C57012098570120DF
:0809E00000000000F20B00080A
:1009E8000000000000FF00000000010000000000FF
:1009F800010000000000000001010101FFFFFFFFEE
:100A080000000001000005533430350000000002EA
:100A180000000000AE014A015E012C0164000200E2
:100A2800000001000A019A01001E0A0000020000ED
:100A380000000000000100000005000001020300A2
:100A4800000000000000000000000000000000009E
:100A58000080070000000000000000000000000007
:100A6800000000000000000020003200C800D0078D
:100A780096001400320028004C044006000550007F
:100A880014000F00080064000100010005000A00BE
:100A98000000F4019600C4090000190000000000DD
:100AA800000000000000000000000000000000003E
:100AB8000000000000000000000000000000000529
:100AC80001000000000000002000030100000000F9
:100AD8000000000001000000020200000000000009
:100AE80003000023E8036400040A000114001E0048
:100AF80000204030900100000000280100007E0521
:100B0800EA05B4053200E803D00700000000000041
:100B180000000000000000000000000000000000CD
:100B280000000000000000000000000000000000BD
:100B380000000000000000000000000000000000AD
:100B48000000000000000000010000050101F401A0
:100B58001400000000000000000000000000000079
:100B6800000000000000000000000000000000007D
:100B7800000000000000000000000000000000006D
:100B8800000000000000000000000000000000005D
:100B9800000000002003000000000000000000002A
:100BA800000000000000000000000000000000003D
:100BB800000000000000000000000000000000002D
:100BC800000000000000000000000000000000001D
:100BD800010000000000000000000000000000000C
:0B0BE8000000000000000000003C00C6
:100BF3000403090412010002EF0201408304563288
:100C0300000201020301000012010002020200407F
:100C1300830440570002010203010800FFFFFFFFA6
:100C2300006002401060024000000000000000006D
:100C3300000B0000000000000000000000000000A6
:100C43000060024028600240010000000000000034
:100C5300060C00000000000000000000000000007F
:100C630000600240406002400200000000000000FB
:100C7300100D000000000000000000000000000054
:100C830000600240586002400300000000000000C2
:100C9300160E00000000000000000000000000002D
:100CA3000060024070600240040000000000000089
:100CB300200F000000000000000000000000000002
:100CC3000060024088600240050000000000000050
:100CD30026100000000000000000000000000000DB
:100CE30000600240A0600240060000000000000017
:100CF30030110000000000000000000000000000B0
:100D030000600240B86002400700000000000000DD
:100D1300362F00000000000000000000000000006B
:100D23000064024010640240000000000000000064
:100D33000038000000000000000000000000000078
:100D4300006402402864024001000000000000002B
:100D53000639000000000000000000000000000051
:100D630000640240406402400200000000000000F2
:100D7300103A000000000000000000000000000026
:100D830000640240586402400300000000000000B9
:100D9300163B0000000000000000000000000000FF
:100DA3000064024070640240040000000000000080
:100DB300203C0000000000000000000000000000D4
:100DC3000064024088640240050000000000000047
:100DD30026440000000000000000000000000000A6
:100DE30000640240A064024006000000000000000E
:100DF300304500000000000000000000000000007B
:100E030000640240B86402400700000000000000D4
:100E13003646000000000000000000000000000053
:100E23007D00000015830008118300080D8300086E
:100E330001830008FD820008098300080583000878
:100E4300000000000D91000885AD0008D190000856
:100E5300C5AE0008E591000885830008718300088A
:100E63005583000831A70008558A0008119400082B
:100E73008594000805950008B5960008690F0108D8
:100E83005D8300084D830008010000000000803FDF
:100E9300493901084D3E0108C5390108051001080B
:100EA300E91101081510010831100108DD0F0108CF
:100EB300CD0F01080000000000000000090220001F
:100EC300010104C0320904000002080650050705A9
:100ED300810240000007050102400000090264008E
:100EE300030100C0320904000001030000000921CE
:100EF300110100012236000705830309000A080BCC
:100F030001020202010009040100010202010005BD
:100F13002400100105240100020424020205240612
:100F23000102070582030800FF09040200020A0008
:100F33000000070501024000000705810240000090
:100F430009024300020100C0320904000001020249
:100F530001000524001001052401000104240202FC
:100F63000524060001070582030800FF09040100A8
:100F7300020A000000070501024000000705810284
:100F830040000000FF00000000FF00000000000020
:100F93000000AA550701000001AA55050100000839
:100FA30000DF0608FF1FFF1F05010905A101A100BE
:100FB3000501093009310932093309350934093684
:100FC30009371581257F75089508810205091901DF
:100FD300290815002501950875018102C0C000008C
:100FE30009022200010100E03209040000010301AB
:100FF30002000921110100012236000705830309BC
:10100300000A0000000000000102030401020304BF
:10101300060708092D202D2D202D2D2D2D202D2DBA
:101023002D2D000000000000000000000000000063
:10103300000000AA550B010000AA5505010000AAF3
:10104300550902000000AA5503009F00010000009B
:10105300C0120000B8B500200000000090B50020C9
:1010630000000000010000009C870708A487070810
:101073000000000045F30308A086010004000000FF
:10108300000000000000000000000000000000005D
:10109300000000000000000000000000000000004D
:1010A30000000000000000009C870708AC870708C9
:1010B300000000007D7D0408E80300000400000038
:1010C300000000000000000000000000000000001D
:1010D300000000000000000000000000000000000D
:1010E3000000000000000000B487070800000000B3
:1010F30000000000855E03087D000000FF00000083
:1011030000000000000000000000000000000000DC
:1011130000000000000000000000000000000000CC
:101123000000000000000000AC0D080800000000F3
:1011330000000000E57103087D000000FF000000CF
:10114300000000000000000000000000000000009C
:10115300000000000000000000000000000000008C
:101163000000000000000000609C07080000000071
:1011730000000000E9B803087D000000FF00000044
:10118300000000000000000000000000000000005C
:10119300000000000000000000000000000000004C
:1011A3000000000000000000BC87070800000000EA
:1011B30000000000E1730408E803000003000000DE
:1011C300000000000000000000000000000000001C
:1011D300000000000000000000000000000000000C
:1011E3000000000000000000C087070800000000A6
:1011F3000000000079270308102700000300000007
:1012030000000000000000000000000000000000DB
:1012130000000000000000000000000000000000CB
:101223000000000000000000C009080800000000E2
:10123300618D02085DD604085F760000050000009A
:10124300000000000000000000000000000000009B
:10125300000000000000000000000000000000008B
:101263000000000000000000500D0808000000000E
:10127300000000007DF404081027000001000000B6
:10128300000000000000000000000000000000005B
:10129300000000000000000000000000000000004B
:1012A3000000000000000000CC87070800000000D9
:1012B3000000000029680408E8030000050000009E
:1012C300000000000000000000000000000000001B
:1012D300000000000000000000000000000000000B
:1012E3000000000000000000D8870708000000008D
:1012F3000000000055FA0308204E00000300000020
:1013030000000000000000000000000000000000DA
:1013130000000000000000000000000000000000CA
:101323000000000000000000E8870708000000003C
:10133300000000003DF80308204E000003000000F9
:10134300000000000000000000000000000000009A
:10135300000000000000000000000000000000008A
:101363000000000000000000F887070800000000EC
:1013730000000000F5790408400D0300030000009D
:10138300000000000000000000000000000000005A
:10139300000000000000000000000000000000004A
:1013A300000000000000000008880708000000009B
:1013B30000000000B1300408102700000100000005
:1013C300000000000000000000000000000000001A
:1013D300000000000000000000000000000000000A
:1013E3000000000000000000108807080000000053
:1013F30000000000F5AD0108102700000300000005
:1014030000000000000000000000000000000000D9
:1014130000000000000000000000000000000000C9
:10142300000000000000000014880708000000000E
:1014330000000000E16A0208A0860100010000002C
:101443000000000000000000000000000000000099
:101453000000000000000000000000000000000089
:1014630000000000000000001C88070800000000C6
:10147300000000006972040850C30000010000006E
:101483000000000000000000000000000000000059
:101493000000000000000000000000000000000049
:1014A300000000000000000024880708000000007E
:1014B3000000000039700408A0860100000000004D
:1014C3000000000000000000000000000000000019
:1014D3000000000000000000000000000000000009
:1014E3000000000000000000308807080000000032
:1014F30000000000216C0408A86100000100000046
:1015030000000000000000000000000000000000D8
:1015130000000000000000000000000000000000C8
:1015230000000000000000003C88070800000000E5
:1015330000000000E1070208A0860100010000008E
:101543000000000000000000000000000000000098
:101553000000000000000000000000000000000088
:101563000000000000000000488807080000000099
:10157300000000002DA50408A00F000001000000DA
:101583000000000000000000000000000000000058
:101593000000000000000000000000000000000048
:1015A300000000000000000054880708000000004D
:1015B30000000000DD020208102700000100000007
:1015C3000000000000000000000000000000000018
:1015D3000000000000000000000000000000000008
:1015E3000000000000000000608807080000000001
:1015F300000000007DF30308A00F000001000000BD
:1016030000000000000000000000000000000000D7
:1016130000000000000000000000000000000000C7
:1016230000000000000000006C88070800000000B4
:10163300000000002DDD01081A4100000100000038
:101643000000000000000000000000000000000097
:101653000000000000000000000000000000000087
:101663000000000000000000708807080000000070
:1016730000000000151701081027000001000000FA
:101683000000000000000000000000000000000057
:101693000000000000000000000000000000000047
:1016A30000000000000000007C8807080000000024
:1016B30000000000E945020850C3000001000000DB
:1016C3000000000000000000000000000000000017
:1016D3000000000000000000000000000000000007
:1016E30000000000000000008088070800000000E0
:1016F300000000005D200108400D03000000000011
:1017030000000000000000000000000000000000D6
:1017130000000000000000000000000000000000C6
:101723000000000000000000888807080000000097
:10173300000000004DF40308400D0300000000000A
:101743000000000000000000000000000000000096
:101753000000000000000000000000000000000086
:10176300000000000000000090880708000000004F
:1017730000000000B5EB010850C3000003000000A7
:101783000000000000000000000000000000000056
:101793000000000000000000000000000000000046
:1017A30000000000000000009C8807080000000003
:1017B30000000000850D040840420F0000000000F7
:1017C3000000000000000000000000000000000016
:1017D3000000000000000000000000000000000006
:1017E3000000000000000000A888070800000000B7
:1017F3000000000011FF030850C3000000000000B8
:1018030000000000000000000000000000000000D5
:1018130000000000000000000000000000000000C5
:1018230000000000000000000100000000000100B3
:10183300E0010000FFFFFFFF01007EFFFFFFFFFF4E
:101843000800000042570200000001064257020050
:101853000000010601FFFF00FFFFFFFF0101010080
:101863004D0B0208000000000000000038E90608E4
:10187300C4D8002018D90020652402088D2202084C
:10188300000000008401070861FA0108000000005D
:1018930000000000E800070805250208000000001A
:1018A30000000000A0000708000000000000000086
:1018B3000000000050FF06080000000000000000C8
:1018C30000000000080007080000000000000000FE
:1018D30000000000B4FF0608000000000000000044
:1018E3006921020899DA0020FF2D202D2D202D2DAE
:1018F3002D2D202D2D2D00000000000000000000E4
:101903000000000000000000FFFFFFFFF5270208B2
:101913000000000000000000E0FE060801000000D7
:10192300FA000000010000000100000001000000B7
:10193300000101010000000016D700200000F4019F
:101943000100000014D700200000F4010100000092
:1019530012D700200000F4010100000010D700207E
:101963000000F401010000000ED700200000F40184
:10197300010000000CD700200000F401010000006A
:101983000AD700200000F4010100000085130208BB
:10199300491302080000000060EB0608FAD6002095
:1019A3000532010008D700206400F40101000000A3
:1019B30006D700206400C40901000000F8D6002007
:1019C300E803D00701000000F6D60020E803D007A3
:1019D30001000000F4D60020E803D0070100000056
:1019E300F2D600201E00B80B0100000000D7002033
:1019F30005000F000100000002D7002003000A00C9
:101A030001000000F0D600201E00F40101000000D8
:101A130004D7002002000000ECEB0608EED60020FD
:101A23001400640001000000FCD600203200E8032B
:101A330001000000ECD600200000C80001000000F7
:101A4300C5D6002000C80100C4D600200050010004
:101A5300C3D60020005A0100C1D6002002000000B6
:101A6300F8EB0608A8930708B09307083E5B00202D
:101A73000100C409000000003C5B00200100C40910
:101A8300000000003A5B00200100C40900000000D0
:101A9300385B00200100C40900000000345B002013
:101AA3000100C40900000000365B00200100C409E6
:101AB30000000000325B00200100C40900000000A8
:101AC300305B00200100C409000000006FD4002037
:101AD30000C801006ED4002000C801006CD40020AF
:101AE3000000FFFF0A0000006AD400200100C800C4
:101AF3000100000068D4002032003075320000007D
:101B030066D400200582050064D4002005002C0162
:101B13000500000062D40020055A05005FD40020B0
:101B230000FF010061D4002002000000FC0F002030
:101B33005DD400200300000020E106085ED40020ED
:101B430000FF010060D4002002000000FC0F002011
:101B53005CD400200300000020E10608D91202082B
:101B6300691202080000000004EC06082CD70020CC
:101B7300EE02CA08010000002AD7002000C80100B5
:101B83006400000029D7002000C8010064000000A1
:101B930028D700200200000010ED060856D40020CC
:101BA3000000803E0500000054D4002080C1803E28
:101BB300050000004ED400200083007D05000000D6
:101BC3004CD4002080C1803E0500000047D4002093
:101BD30000FF010042D400206400F4010100000072
:101BE30040D40020040000001CED06083FD4002070
:101BF3000200000030ED0608F5D400200D000000BF
:101C03003CED0608F2D4002000640100F0D400206B
:101C1300320010270A000000EED400200D0000005F
:101C23003CED0608EDD400200D0000003CED060855
:101C3300ECD400200200000074ED06080000000050
:101C4300000000000000000080ED060832D70020ED
:101C53003E000000B8ED060830D700200100FF7FEA
:101C6300010000002FD7002002000000B4EE060898
:101C7300F7D4002003000000C4EE0608F6D40020C9
:101C830003000000C4EE0608B2D60020000A0100DB
:101C9300B0D600200000E80301000000AED600200B
:101CA3000000E80301000000ACD600200000E803B8
:101CB30001000000AAD600200000E8030100000094
:101CC300A2D600200000E80301000000A8D60020EF
:101CD3000000E80301000000A6D600200000E8038E
:101CE30001000000A4D6002000140100C0D600208B
:101CF30002000000D4EE0608BED600200000F40166
:101D030001000000BCD600200000F4010100000027
:101D1300BAD600200000F40101000000B8D600206C
:101D23000000F40101000000B6D600200000A00F5F
:101D330001000000B4D600200000A00F0100000045
:101D4300D9D6002019640100D8D600200200000073
:101D5300E0EE0608D6D60020E803D0070A0000000C
:101D6300D4D60020006401000A000000C9D6002078
:101D730000640100C8D6002000640100D0D6002012
:101D8300006401000A000000CFD6002000640100B7
:101D93000A000000CED60020006401000A00000003
:101DA300D3D6002000FF01000A000000D2D6002095
:101DB30000FF01000A000000D1D6002000FF01004F
:101DC3000A000000CDD6002001FF01000A00000038
:101DD300CCD6002001FF01000A000000CBD6002072
:101DE30001FF01000A00000000D500200000F401FB
:101DF30001000000FED400200000A00F010000003D
:101E0300FCD400200000A00F01000000FAD4002041
:101E13000000A00F01000000F8D400200000A00F74
:101E230001000000E9DA002000C80100E8DA002020
:101E330000640100E7DA002000640100E6DA002014
:101E430000640100E5DA002000640100E4DA002008
:101E5300FF080100E3DA002001640100D111020848
:101E63009511020800000000ECEE0608ECDA0020F1
:101E730001320100EBDA0020010000005CEF0608EC
:101E8300EADA00200400000064EF0608E2DA00202A
:101E930000640100E0DA00201400E8030100000000
:101EA300DEDA0020E80330750A000000DCDA0020E7
:101EB30000C80100DBDA002000C80100DADA0020E4
:101EC30000C80100D9DA002000320100EEDA002058
:101ED300004B0100EDDA00200400000078EF060853
:101EE300D8DA0020006401000A000000FCDA0020B8
:101EF3000000D00701000000F7DA002000C801004D
:101F0300F6DA002000C80100F5DA002000C801005D
:101F1300FADA00200000D00701000000F4DA002004
:101F230000C80100F3DA002000C80100F2DA002043
:101F330000C80100F8DA00200000D007010000000B
:101F4300F1DA002000C80100F0DA002000C8010027
:101F5300EFDA002000C80100890F0208710F0208A0
:101F6300000000008CEF0608E9D40020005A0100AD
:101F7300E8D4002000C80100E6D40020E803D0071D
:101F8300010000000000000000000000A921020879
:101F930028F0060853544D333246343035000000E0
:101FA3005BD40020000301005AD400200003010089
:101FB300AD0E0208610E0208000000007CF0060866
:101FC300210E0208D90D02080000000018F10608CE
:101FD300F90E0208D92702080000000098F106084C
:101FE30058D40020010301006114020835140208CB
:101FF30000000000F0F40608650D0208210D020838
:102003000000000060F50608990F02082D29020858
:1020130000000000FCF50608F52C02088D140208E8
:1020230000000000A4F60608E90F02080000000003
:102033000000000030F70608C51002086D10020802
:102043000000000094F70608591102081D11020848
:10205300000000003CF80608E18702080D120208A0
:1020630000000000C8F80608EBD6002001060100B6
:1020730031100208FD0F020800000000C4F9060831
:1020830015870208F92902080000000034FA06083F
:1020930029880208C12A02080000000084FB060800
:1020A300EAD6002001030100410F0208110F0208C4
:1020B3000000000058FC06088188020800000000A8
:1020C30000000000BCFC0608A90D0208C127020895
:1020D300000000003CFD06080000000000000000B6
:1020E30000000000C8FD060841120208392B02084F
:1020F3000000000038FE0608000000000000000099
:102103000000000050000708B0B000209CFF2C0125
:1021130000000000F4DB0020E0150C1700000000B5
:1021230084CF002002000000880007083BD4002071
:10213300020000009400070836D4002088136F17AC
:102143000100000038D4002088136F17000000003E
:10215300825B00200000000000000000805B002084
:1021630000000000000000007E5B00200000000073
:10217300000000007C5B0020000000000000000065
:102183007A5B00200000000000000000785B002064
:102193000000000000000000E8050020000000002F
:1021A300000000000CD4002003000000E801070831
:1021B30034D4002088136F1701000000FAB0002008
:1021C30088136F1700000000050C020800000000D0
:1021D30000000000F8010708DDD90020010000001D
:1021E3004C020708FCB00020010000005802070859
:1021F300F2B00020020000006002070800000000A7
:1022030000000000000000006C020708F10B020848
:1022130000000000000000000803070800000000A1
:1022230000000000000000005C030708000000003D
:102233000000000000000000CC0307083AD400208F
:102243000200000004040708F6B00020E0150C1794
:102253000000000001D60101FFFFFFFF0000803FE7
:10226300000000000000000000000000000000006B
:10227300000000000000000000000000000000005B
:10228300000000000000803F00000000000000008C
:10229300000000000000803F00000000000000007C
:1022A300000000000000803F00000000000000006C
:1022B30000000000010000000000FA430000FA43A0
:1022C3000000803FC132040800000000000000004D
:1022D30000000000FFFFFFFFFF0000000000000000
:1022E30034FF0020080000000000000024FF00204D
:1022F30008000000A1380108F91001083938010865
:1023030000000000C90F01082141010889370108B5
:10231300D53301080000000000000000890F010808
:1023230025830008198300085D9000087990000850
:1023330041900008259000080990000859380108C9
:10234300D51001088D37010800000000A10F010816
:10235300D93301085D370108353301080000000057
:1023630000000000950F0108685E0C00FFFFFFFFEF
:1023730002010000A00F0000B80B000002FFFF01E4
:10238300FFFF0000B409080800000802050303006A
:1023930000000000BC09080801000802050403004E
:1023A3000000000070B107080200FE0101100300E5
:1023B3000000000010970708030014020003000048
:1023C30000000000C409080804001F0202000800FE
:1023D30000000000CC09080805001F0202010800E4
:1023E30000000000FFFFFFFF1A03000000000000D1
:1023F30000000000000000000000000000000000DA
:102403000000000004030904120100020000004060
:10241300830420570002010203010B01819905087F
:1024230055990508F998050895890508159905082A
:10243300B998050891890508D41A0020719A0508EE
:10244300919A0508619A0508758905081D9A05087A
:10245300D599050865890508B01A002095920508E5
:102463007D8905087989050871890508DD930508C3
:102473006D89050869890508505A0708BD40010898
:10248300B51001089D3F0108000000000000000096
:102493003537010845360108000000000000000040
:1024A300000000007D0F01081D8A0508118A050838
:1024B300E19A0508FD9A0508C9890508C59A050822
:1024C300A99A0508FFFFFFFF0100000050C30000A9
:1024D300010100001F0000001C0000001F0000009D
:1024E3001E0000001F0000001E0000001F0000006F
:1024F3001F0000001E0000001F0000001E0000005F
:102503001F0000000068214C01250000F056070859
:10251300F0630708F81A0020008002021F00000081
:1025230053544D202020202050726F647574202056
:102533002020202020202020302E30310080020255
:102543001F00000053544D202020202050726F6440
:10255300757420202020202020202020302E303190
:10256300DB160108D7160108CF160108B9140108B4
:10257300C51F0108F11F0108211F0108C516010825
:10258300B5160108A516010895160108B11401082E
:10259300FF010000F4010000FF000000000004013F
:1025A300000000000000000210000000070000000F
:1025B30000000000000000000102030406070809F0
:1025C30001000000601B002000000000000000006C
:1025D30000000000000000000000000000000000F8
:1025E30000000000000000000000000000000000E8
:1025F30000000000000000000000000000000000D8
:1026030000000000000000000000000000000000C7
:1026130000000000000000000000000000000000B7
:082623000000000000000000AF
:0828000000C00F0800001008E1
:10800000F0B401292A4C2B4D23684FF0000694BF91
:1080100000270127EE626662A6626763676B47EA24
:1080200042076763EE63EC6B002A38D144F4957421
:10803000EC631C6824F001041C601C68E407FCD499
:10804000490289085960D8601968EAB921F04001ED
:10805000196019498B421DD018494FF47410C8603B
:10806000196841F01E011960596941F08001596198
:10807000196841F00101196022B90E4AD36A43F030
:108080000803D362F0BC704741F0400119600A490F
:108090008B42E1D14FF0746041F8500CE0E744F0BE
:1080A0001A04EC63EC6A44F00804EC62C1E700BF18
:1080B000C01B0020002C01405864024000640240B4
:1080C0001148002302461178032902F1060216D056
:1080D0000133062BF7D10D4AD36D052B0ED0591C59
:1080E00003EB4303D16500EB4303032040F2EB3184
:1080F00040F2FF32187059809A807047704703EB46
:10810000430300EB4303F0E7F81B0020C01B0020F3
:1081100070B4C3080D4CE25C00F00706B24004EBFB
:10812000D004D2B20020C6F108038B4228BF0B4610
:10813000C3F108052A419840C91A40EA02004FF0ED
:10814000000614F8012FEED170BC7047601C0020AF
:10815000084AD2E9343199420AD0D118013391F852
:10816000D8100170C3F30A03C2F8D0300120704761
:1081700000207047C01B0020064AD2F8D838D2F839
:10818000DC28934294BF4FF400600020013B9B1A0F
:1081900018447047C01B0020012380F851307047FD
:1081A00007B501A8FFF7D4FF0028FAD09DF8040016
:1081B00003B05DF804FB044BD3E93403984288BF55
:1081C00003F50063181A7047C01B00200120704798
:1081D000024BC3F8E028C3F8E4187047C01B002026
:1081E000024BC3F8E828C3F8EC187047C01B002006
:1081F0007047704730B4134DD5E934239A4286BF97
:1082000003F50064A21A9A1A0A44B2F5006F13D853
:10821000A9B101444A1E013810F8014FE918824201
:1082200003F1010381F8D840C3F30A03F4D1C5F880
:10823000D430002030BC7047022030BC7047084664
:10824000F8E700BFC01B0020212838B50C4605D038
:1082500022282ED0202813D0002038BD0029FBD0A2
:10826000072AF9D11A4BD3F8F00893F8F41893F8C9
:10827000F52893F8F638206021716271A371EBE75D
:108280000029E9D0072AE7D1114DD5F8E4381BB110
:108290000968D5F8E0089847206821796279A379C0
:1082A000C5F8F00885F8F41885F8F52885F8F6384B
:1082B000D2E70029D0D0022ACED1054AD2F8EC3834
:1082C000002BC9D00988D2F8E8089847C4E700BF56
:1082D000C01B0020024B0020C3F8F808704700BF05
:1082E000C01B0020044B00200522C3F8F828C3F867
:1082F000EC08C3F8E4087047C01B0020704700BFBB
:10830000704700BF704700BF704700BF704700BF95
:10831000704700BF704700BF042301480B807047BF
:108320008801002010B4074A074B92F8FC08122479
:1083300003F114020C8001280CBF184610465DF8AA
:10834000044B7047C01B00208C0100200048704780
:10835000481C002000487047481C0020034B93F83D
:108360008400032894BF002001207047C01B002018
:10837000034B93F88400032894BF0020012070472A
:10838000C01B0020034B93F88400003818BF012065
:10839000704700BFC01B0020A0B182680D4B12B116
:1083A00007229A7070471978DA6003294FF00400A9
:1083B0000CBF80214FF48071C3E901111A611A7555
:1083C00098707047034B41F2E47101225A545A707D
:1083D000704700BFE08E00200378022B10D00069A8
:1083E00008B9012070470C4B1B78032B0EBF0B4BB9
:1083F00080B24FF6F773984294BF00200120704777
:108400000549436841F650028A58B3EB422F2CBF0E
:1084100001200020704700BFE08E0020F7FFFF0F13
:108420000378022B14D030B4104A4368006941F637
:10843000480402F5C2511559096841F63C042B4025
:1084400012595B0A023801FB0030104430BC7047FF
:10845000064B426841F6340141F63000595818582D
:1084600000EB410000EB5220704700BFE08E00207F
:1084700008B5124BD3F8BC00828940F2E933028977
:10848000013B12F0020F9BB212D0FF23838140F216
:10849000E9330289013B12F0010F9BB202D08089BF
:1084A000C0B208BD002BF4D146F0C6FBC0B208BD77
:1084B000002BE4D146F0C0FBC0B2F8E7C01B00209F
:1084C00070B505460E460924FFF7D2FFFF2803D1F9
:1084D000013CF9D1012070BDFE2801D0022070BD01
:1084E000064933462A46D1F8BC0000215FF022FE3F
:1084F000FFF7BEFFFFF7BCFF002070BDC01B0020D0
:1085000010B51D4C0023C4F88030FFF7B1FFD4F83C
:10851000BC00828940F2E9330289013B12F0020F6C
:108520009BB217D0FD23838140F2E9330289013BDE
:1085300012F0010F9BB212D08389FFF799FFFF2839
:1085400012D1FFF795FFFF280ED10423022084F8F3
:10855000843010BD002BDFD146F06EFBEDE7002B21
:10856000E4D146F069FBE8E7D4F8003963670923F2
:10857000002084F8843010BDC01B002070B582B08C
:1085800040F040060C0E05460A0A080C95238DF8AB
:1085900001408DF804108DF800608DF802008DF810
:1085A00003208DF805300824FFF762FFFF2802D072
:1085B000013CF9D125BB1A4BD3F8BC0006258389B1
:1085C0006E464FF47A734FF6FF713EB316F8012BE7
:1085D0000489013BA4079BB215D593B283814FF464
:1085E0007A730489E40703F1FF3211D5013D8289D2
:1085F000EBD10924FFF73CFFFF2802D1013CF9D160
:10860000FF2002B070BD8B42E2D146F015FBF0E7CF
:1086100093B28B42E5D146F00FFBEAE7FF22D7E7A2
:10862000C01B00202DE9F041684C00234FF4F0728C
:108630002021064604F6081084F8043964F05BFE35
:1086400004F6E8204FF4F072202164F054FE94F810
:10865000C90C10B194F8CA2C1AB900252846BDE8F7
:10866000F08144F083FC0746C4F8D40C44F052FF78
:1086700005460028F1D00FB12323FB80092138469D
:1086800040F006FDD4F8D40C514F44F065FF94F847
:10869000CA0C013840B246F039FC0223102184F89C
:1086A000CC3CC4F8D00C5FF013FD798D494846F0FE
:1086B00079FAD4F8D40C44F049FFFF218C205AF009
:1086C00017FF8046D4F8D40C44F046FFD4F8D00C01
:1086D00004215FF0FDFCB8F11B0F05D0D4F8D40CD9
:1086E000202140F0D5FCB8E7D4F8D43C012284F82E
:1086F00004290BB12322DA80798D364846F052FAEC
:10870000D4F8D40C44F022FF40210A205AF0F0FEA5
:10871000FF218A205AF0ECFEC0F38013D4F8D40C69
:1087200084F8D83C44F018FFD4F8D00C04215FF052
:10873000CFFC94F8C83C012B3FD0022B37D0CBB3F1
:1087400094F8D93C182B08D194F8D82C7B8DA4F838
:10875000DC6CA4F8DE2CA4F8E03C798D1D4846F0D2
:1087600021FA798D1B4846F01DFAD4F8D40C44F058
:10877000EDFE022100205AF0BBFED4F8D40C44F0E8
:10878000EBFE0421D4F8D00C5FF0A2FC94F8E92CA5
:1087900094F8EA3C94F8E81C84F8E41CC2F1200246
:1087A000C3F1100384F8EB2C84F8EC3C56E7082363
:1087B0007B85C5E710237B85C2E7002EF7D094F8B0
:1087C000D83C002B14BF08231023F1E7C01B002066
:1087D000880100208C2800202DE9F84F564B984244
:1087E00010D003F568530833984267D0534B0020EC
:1087F000A3F8480DA3F8540DC3F84C0DC3F8500D61
:10880000BDE8F88F4D4C4E4E02224FF0000BC4F8DD
:10881000F02C04F6F445D9464FF4007A4FF48078F2
:10882000F26A01275A455946BB4403D0D4F8640D77
:1088300054F0E2F994F8682D85F82420D4F8640DFA
:10884000A5F804A04FF000724FF48031A960EA60EF
:10885000A5F8108085F81290A5F806802F7628627A
:10886000B72154F0BFFBD4F8F02C364B6F7693450C
:1088700045F8283BD4DB84F8569DD4F8F01CB4F8B6
:10888000F82CD4F8003DD4F8FC0CB4F8045DC4F81E
:108890006C3D12FB01F203FB01F3A4F8482DB4F880
:1088A000FA1C294AC4F84C0DC4F8503DA4F8545D94
:1088B000A4F84A1DC4F8442D0120A1E71F4C204E06
:1088C0000223C4F8F03C04F6F4454FF0000B4FF4DB
:1088D000806A4FF040094FF40068F26A01275A4558
:1088E0005946BB4403D0D4F8640D54F085F9D4F84C
:1088F000641D94F8682D296285F824204FF4003116
:108900004FF00062C5E90212A5F804A0A5F8109086
:10891000A5F80680AF74FFF7D3FB28466F7654F0B6
:10892000B3FAD4F8F02C094B45F8283B9345D4DB37
:1089300084F8567DA1E700BF1971EF00C01B00202D
:108940008801002098D30608F0D30608C4D306088F
:10895000F8B51A4C94F8703D002BFBD159B3014483
:108960004E1E451ED4F8DC28D4F8D81815F8017F1F
:10897000531CC3F30A038B422CBF4FF4006000204A
:10898000C91A22440144012982F8747DC4F8DC38F4
:108990000FD1012041F0CAF8D4F8D838D4F8DC1847
:1089A0008B4294BF4FF4006200225B1A1344012BE8
:1089B000EFD0B542D6D10020F8BD00BFC01B0020CB
:1089C00010B5094CD4F8F838084611465BB1D4F814
:1089D000F838052B07D1002AD4F8003903DDFFF75A
:1089E000B7FFD4F8003910BDC01B002010B590F8B7
:1089F0005010002380F8503081B10B4CD4F8F82887
:108A000072B1D4F8F828052A0CD13C30D4F80039DA
:108A1000FFF79EFFD4F80039012010BD0120FCE7CC
:108A20001046FAE71846F8E7C01B0020002280F83D
:108A30005120DBE790F85020531C0244DBB280F851
:108A4000503082F83C1090F851200AB1132B00D915
:108A5000CCE770472DE9F04143794F4C002B14BF10
:108A60000122002284F8B02003D184F88430BDE8CC
:108A7000F08190F8018008F1FF3676B20546304665
:108A80000F4646F043FA0223C4F8BC0084F8B8301D
:108A90002B78002B5BD1ED78002D4CD14FF48071F9
:108AA000D4F8BC00C4F8C0505FF012FB4FF47A70E9
:108AB00041F03CF8D4F8C00044F04EFDD4F8BC00BE
:108AC0000A2683894FF6FF714FF47A73FF270289D4
:108AD000950719D587814FF47A730289D20703F17C
:108AE000FF3524D5013E8289F1D12C4B02899207B2
:108AF00013D5028912F080020FD1D4F8001984F83E
:108B0000782001236167B0E7013B9BB28B42DED145
:108B100046F092F8D4F8BC00E7E7013BE6D194F8C0
:108B2000782084F88430531C84F878309FE7ABB207
:108B30008B42D2D1ECE7284644F018FA054608B13A
:108B40001E23C3800921284640F0A2FAA6E706EBBF
:108B500086063E44414696F90320002041F078FC09
:108B6000064630B140685DF0A9FFB36884F8CE30A6
:108B700018B9002384F8C4308DE7094A431E02EB7C
:108B8000431317210022C4F8C8305DF0A9FF012368
:108B900084F8C4307FE700BFC01B0020A18601001D
:108BA000B80100202DE9F04FCF4DDFF87083DFF8DA
:108BB000789384460F4616460FCD44462DED068B1E
:108BC0000FC40FCD0FC495E807008BB099F87E3421
:108BD000029684E80700CDE906C7042B00F25C8109
:108BE000DFE813F0BD015A0155010500CD019FEDED
:108BF000BF8ADFEDBF8ABF49C8F81C10BE49BF4B12
:108C0000BF4AC8F818100299002918BF134638EE59
:108C1000887AF5EE006A86EE87AAC8F82430B94F44
:108C2000B94B03930026DFEDB97A9FEDB99A28EE90
:108C3000278AF0EE679A079BB34200F02281039BDC
:108C400013F8014B039306F1010B5FFA8BF2002C32
:108C500000F09881DFF8D4C2002303E00133152B24
:108C600000F0908103EB43015D001CF80100A0427D
:108C7000F4D14944049291F89914002900F08A81B2
:108C800020463FF0DBFF03680593824618463FF01D
:108C9000C1FF9AF805103FF0F1FF90F800C0BCF159
:108CA000000F40F06F8109EB05002509013D049A92
:108CB00080F8D9240321052D80F8D814059B04F0F1
:108CC0000F0000F23781934C04EB450CBCF8B0C0A8
:108CD0004CFA00FE1EF0010E00F03E81012303FA63
:108CE00000F0013800EA0C002544049260F00CFE0C
:108CF00095F8BC50DFF838C2049A28440CEBC00544
:108D00000321A971EA715CF830007D6100F13F41F7
:108D100001F57E0104EB9124012394F8C4109AF824
:108D2000082001F01F044909032903FA04F300F0A5
:108D30000E81042900F00681022900F0FE80AB8834
:108D40000893B3FA83F3C3F11F03C3F3CC0100EB21
:108D5000810103F007030C6A9B000F259D4024EA64
:108D600005040C620C6A02FA03F323430B6202232C
:108D700008A909930BF01CFDDAF80030029A002ACA
:108D800000F0A280B9F87C2400EE102AB8EEC00AE8
:108D9000FCEEC07A17EE901A5F4A934200F0818091
:108DA000A2F5806293427CD002F58042934278D053
:108DB00002F58062934274D002F58062934270D0D3
:108DC000D9F8042850084FF6FF73B0FBF1F21A44AB
:108DD000120CB0FBF2F20298002865D0B2FBF1F160
:108DE00099F87E0404288BB263D007EE902AF8EE3F
:108DF000676A66EE887A29EE677A99F87F040699A1
:108E00000091A6EEA87A019051463846C7ED027A45
:108E100087ED037A37F066FA002E60DD7B68D8F8BC
:108E2000382093425DD0012E59D0D8F8502093427B
:108E300057D0022E53D0D8F86820934251D0032E39
:108E40004DD0D8F8802093424BD0042E47D0D8F88C
:108E50009820934245D0052E41D0D8F8B0209342B7
:108E60003FD0062E3BD0D8F8C820D31A18BF012314
:108E70005E460122082E3B747A7407F118077FF4CE
:108E8000DAAE26480BB0BDEC068BBDE8F08F9FED47
:108E9000248AF0EE488AAEE69FED228AF0EE488AF8
:108EA000A9E6D9F804088EE799F87E040428194643
:108EB0009BD107EE901A07EE102AF8EE677AF8EECB
:108EC000476A67EEA97A96E7B0EE4A0A049361F022
:108ED00067FEFCEEC07A049B17EE901A5CE7012354
:108EE000C6E70023C4E700BF1CD40608ACC5A737FB
:108EF000ACC5A73611F80308ED6B040829EE03088A
:108F0000E16B0408480000103B3100206F12833AE7
:108F100000007A4498D306080004014014000010B1
:108F2000282930386F120339B82C00205031002026
:108F3000BC310020C7F814C020E717494C6C23430C
:108F40004B64FCE614490C6B23430B63F7E61249B0
:108F50000C6C23430B64F2E6C7F814E00EE79FEDB8
:108F60000F8A0F4BC8F8183000230E4A06930123CE
:108F70000293C8F81C200C4BF0EE488A47E69FEDA0
:108F80000B8AEEE70A4A084BC8F81C20C8F82430C0
:108F9000002077E70B68FFDE003802406F12833A4B
:108FA000ED6B040811F80308E16B040800000000F1
:108FB00021F10308F8B5114ED6F8044805460068BB
:108FC0000F4664080BF0F8FAB4FBF7F1B1F5803FF7
:108FD00003D3012CFAD96408F6E72246284689B261
:108FE0003FF0AAFC41F26C03054AF25028460549BD
:108FF000BDE8F84000223FF01FBC00BFB82C0020A5
:1090000005FE0108243D002010B5044C04480A4622
:1090100021460AF013F9204610BD00BF2C3D002068
:10902000B486070810B5044C04480A4621460AF0E5
:1090300005F9204610BD00BF2C3D0020C48607085E
:1090400010B5044C04480A4621460AF0F7F82046B9
:1090500010BD00BF2C3D0020D086070810B5044C81
:1090600004480A4621460AF0E9F8204610BD00BF30
:109070002C3D0020DC86070810B5044C04480A4645
:1090800021460AF0DBF8204610BD00BF2C3D002031
:10909000E886070810B50C4C94F8CD200023C4F8DE
:1090A00080300AB1094AD3675BF018FB20B1042372
:1090B000022084F8843010BDD4F800396367092396
:1090C00084F8843010BD00BFC01B0020B03D0020DC
:1090D00070B50D4D95F88430042B04460E460AD029
:1090E000082B06D1EB6F83420CD0FFF7D3FF022889
:1090F00001D0012070BD0823C5E91F4685F88430E2
:10910000022070BD022070BDC01B002070B54379E5
:10911000234C002B14BF0123002384F8B03003D16B
:10912000002384F8843070BD1E4D002195F9832002
:10913000032041F08DF90028F2D0466830465DF0FA
:10914000BDFC84F8CC000028EAD095F88130003BC3
:1091500018BF0123304684F8CD305AF08BFE0AF058
:109160001DF838B994F8783084F88400013384F815
:10917000783070BD5BF098FB40B194F878300022F5
:10918000013384F8783084F8842070BDD4F8002945
:1091900084F878000123626784F8843070BD00BFD2
:1091A000C01B0020B03D002010B55BF07DFB58B126
:1091B0000B4C94F878300133DBB2072B84F878300D
:1091C00003D9002384F8843010BD09F0E7FF00289C
:1091D000F7D0D4F800396367012384F8843010BDD8
:1091E000C01B00202DE9F041874C94F8B050002DB1
:1091F00000F0F78094F88420844F0226531E082B39
:1092000040D8DFE803F036389D3F674F153F050033
:109210005BF064FA002840F0EB80636FD4F800291B
:10922000FA3393422BD2FFF7BFFF94F88420E5E78F
:109230005BF054FA0028F0D0D4F880300022012BE3
:1092400084F8782040F2D880E16F94F8CD00013B9B
:109250000131C4E91F1308B16C4BDA67082284F8A6
:109260008420A2F10805B5FA85F56D092846BDE808
:10927000F08184F884605BF031FA002841D194F8E1
:109280008420531EDBB2022B09D8D4F80039616F59
:109290005B1AC82BE5D9FFF787FF94F88420042ACE
:1092A000DFD1E3E7236B002BDBD1E66ED4F8003986
:1092B0006367072284F88420002ED2D0D4E91821D5
:1092C000236F0120B047DAE7636FD4F800196433E5
:1092D0008B42C6D2D4F82C80B8F1000FF4D15BF0E9
:1092E000FDF90028A1D0E66E84F87880042384F884
:1092F0008430002E7AD0D4E91821236F4046B0473D
:10930000BDE75AF089FE0028B9D197F88530002BC7
:10931000A3F10203B3FA83F314BF022201225B0913
:1093200084F8792084F87A305AF076FE00287FF4A9
:109330007AAFD7F8D030C4F88830032384F884306B
:109340005AF06AFE00289AD1304BC4F8800093F896
:10935000B460B3F8B600D3F8B8E0D3F8B8C0D3F827
:10936000B870D3F8B82084F88E6093F8BC10A4F8D5
:109370008C0093F8BD6084F8922093F8BD00D3F878
:10938000C020C4F89420B3F8C680B3F8C62084F88F
:109390009310B3F8C610C2F30B1343EA182303F07B
:1093A0000F0301F00F024FEA1E6E4FEA1C4C3F0AFA
:1093B000360900F00F0003F5FA63042184F89900E0
:1093C00084F88FE084F890C084F8917084F89860F5
:1093D000A4F89A3084F89C2084F884102846BDE8CC
:1093E000F08184F884502846BDE8F08105463DE7C9
:1093F000042384F8843039E7FAD1FFF74BFE94F860
:109400008420531E3EE700BFC01B0020B03D00205B
:109410002DE9F8431A4C94F88460042E05468946D9
:1094200090461F4608D0082E02D00020BDE8F883E1
:10943000FFF766F80228F8D1D4F8C00044F086F8A7
:1094400094F87A3093B969021120FFF797F898B928
:10945000D4F80039C4F860900522C4E91B8765661A
:1094600084F8842063670120BDE8F8832946112031
:10947000FFF784F80028EBD009F066FED5E700BFBF
:10948000C01B002070B51E4C94F88430042B064697
:109490000D4608D0082B22D1E36F83422DD0FFF771
:1094A0002FF802281BD1D4F8C00044F04FF8002157
:1094B0003720FFF763F829461720FFF75FF8B0B9A8
:1094C00094F87A306BB971021920FFF757F870B928
:1094D0000823C4E91F6584F88430022070BD012090
:1094E00070BD31461920FFF749F80028F0D009F087
:1094F0002BFE09F065FE032070BD022070BD00BF89
:10950000C01B00202DE9F043694D91B006460F467F
:109510009046994695F88430042B0DD0082B07D13E
:10952000EB6FB34200F0C080FEF7EAFF0228F1D0F3
:10953000012011B0BDE8F083D5F8C00044F006F872
:1095400095F87A30002B40F09E8071021820FFF7CA
:1095500015F8002840F0A28095F88440FEF788FFB7
:10956000082C0CBFFC22FE22D5F8BC00818940F2F9
:10957000E9330189013B11F0020F9BB24FD093B246
:10958000838140F2E9340389013C13F0010FA4B256
:1095900076D0838995F8C430002B48D001A80AF012
:1095A00033FED5F8BC30D5F8C82095F8CE105068F9
:1095B00003970C334022029300234906CDE9083378
:1095C00004920B934FF4806206930A934FF4007356
:1095D0000792019105930AF055FED5F8C83001A90C
:1095E00058680AF023FED5F8C830D5F8BC20596871
:1095F0000B6843F001030B6093889BB243F00203B6
:109600009380012206230020C5E91B892F666E6620
:1096100085F8682085F8843011B0BDE8F083002B10
:10962000A7D145F009FB95F8C430002BB6D1D5F889
:10963000BC00BE4683894FF480724FF47A744FF6B3
:10964000FF71BEF1000F19D01EF8013BB0F808C041
:10965000013C1CF0020FA4B217D09BB283814FF4DF
:109660007A74B0F808C01CF0010F04F1FF3311D078
:10967000013A8389C5D0BEF1000FE5D1FF23E5E7AC
:10968000002C80D1CDE7314660E78C42DED145F039
:10969000D3FAB6E79CB28C42E3D1F8E709F054FD67
:1096A00009F08EFD032044E7FEF7E2FEFC225BE7B3
:1096B000C01B00202DE9F04FA44C94F8B06087B097
:1096C000002E00F0D68194F88420DFF88892DFF82D
:1096D00088829F4F4FF6FF75531E082B00F295802E
:1096E000DFE813F0A700D1006B01930082000900AE
:1096F00014019300FF0094F8C430002B40F03E8228
:10970000D4F8BC00236E94F868E0828903EB0E2C39
:109710004FF480714FF47A73BCF1000F00F0B78101
:109720001CF801AB0289013B92079BB240F1EE812C
:109730001FFA8AF383814FF47A730289D20703F107
:10974000FF3A40F1EB8101398289E5D10EF1010E3A
:109750005FFA8EFEBEF1020F84F868E052D1D4F8B1
:10976000BC00838940F2E9330289013B12F0020F09
:109770009BB200F0C7810023838140F2E933028964
:10978000013B12F0010F9BB200F0B4818389838901
:1097900040F2E9330289013B12F0020F9BB200F064
:1097A000A5810023838140F2E9330289013B12F055
:1097B000010F9BB200F094818389FEF759FE00F0FF
:1097C0001F00052800F0A18209F0FAFCD4F86CA073
:1097D000BAF1000F00F0CC810022236F616E0120EE
:1097E000D04794F8842077E7206E4FF40071FEF79D
:1097F00067FE012800F0A481022800F0A88100285B
:1098000000F0EF8194F88420531EDBB2022B00F2AB
:109810003A81D4F80039616F5B1AC82B00F22F81AE
:10982000A2F10806B6FA86F67609304607B0BDE81A
:10983000F08FD4F8C00043F089FE00210846FEF7FF
:109840009DFE824609F080FCBAF1010FDAD10023B7
:10985000D4F8C00084F8793043F078FE40F2AB11C0
:109860000820FEF78BFE052800F08581012800F016
:10987000118109F069FC94F87920002A00F04282F5
:10988000022384F88430D4F8C00043F05FFE94F8DB
:109890007930022B0CBF4FF0804A4FF0000A0021B4
:1098A0003720FEF76BFE51462920FEF767FE824601
:1098B00009F04AFCBAF1000FA4D194F87930022BD8
:1098C00000F0A48184F87AA0D4F8C00043F03EFEF2
:1098D00000210920FEF752FE00283FD009F034FC99
:1098E00090E74FF0080AFEF7C3FDFF2800F0208242
:1098F000BAF1010AF7D1636FD4F80029FA33934221
:1099000080D209F05DFC94F88420E5E6FEF7B0FD16
:10991000FF284FF0080A06D0BAF1010AEBD0FEF793
:10992000A7FDFF28F8D1D4F880300022012B84F85D
:10993000782040F20382E26F08210132013BC4E942
:109940001F2384F884100A466AE700BFC01B00206A
:10995000006402400F64024000600240C5481021CC
:10996000FEF7AEFD83460028B8D101217F20FEF727
:10997000CFFB01288246B1D158460221FEF7C8FB31
:10998000002800F0A0810128A8D116213A20FEF776
:10999000BFFB01308002C4F8880009F0D5FBD4F881
:1099A000C00043F0D3FD00210A20FEF7E7FD0028A8
:1099B00040F06481032384F88430102102A8FEF76C
:1099C0007FFD00287FF41EAF9DF815309DF816101E
:1099D0009DF810209DF809009DF80AC01B01DBB21C
:1099E00043EA111303F5FA63A4F89A30DDF8113055
:1099F00001F00F0184F89C101BBA110902F00F024C
:109A00004CEA002084F8981084F899209DF80810FA
:109A10009DF80B20C4F89430039BC4F89030A4F850
:109A20008C0084F88E1084F88F2009F08DFB94F858
:109A30007A307BB9D4F8C00043F088FD4FF4007150
:109A40001020FEF79BFD824609F07EFBBAF1000F65
:109A50007FF457AFD4F8BC0004215EF039FB00223C
:109A600004233046C4F8802084F8843007B0BDE871
:109A7000F08F304684F8846007B0BDE8F08F09F0BD
:109A80009FFB94F88420042A7FF4CAAECDE64FF001
:109A9000FF0A47E6D4F8BC004FF0040E838902A900
:109AA0004FF47A734FF0FF0C028992073CD5A0F86F
:109AB0000CC04FF47A730289D20703F1FF3A3AD50A
:109AC000828992B209B101F8012BBEF1010EEBD1EE
:109AD0009DF80B30AB2B04BF022384F87930C8E625
:109AE000002B7FF462AE45F0A7F866E6002B7FF40A
:109AF00051AEF8E7002B7FF442AE45F09DF8D4F864
:109B0000BC0044E6002B7FF42FAEF6E7AB427FF4B7
:109B100009AE45F091F894F868E017E61FFA8AF369
:109B2000AB427FF40AAEF4E7013B9BB2AB42BBD140
:109B300045F082F8CCE71FFA8AF3AB42BBD1F7E7D6
:109B4000636FD4F8002964339342BFF45BAE09F02D
:109B5000FBFA09F035FBD4F86CA0BAF1000F07D07E
:109B600000221046236F616ED04794F88420B3E53D
:109B700094F88420B0E584F879A07AE6D4F8C83067
:109B80005968DB69494594BF4046384613F0005F89
:109B900000F08B80D0F804C0DFF8DCE003EA0C0CA6
:109BA0001CEA0E0F3FF43CAE03EA0E03C3600B68E1
:109BB000D4F8BC0023F001030B600389D90703D557
:109BC00083890389DA07FBD403899B07FCD50389C2
:109BD0001906F9D4838823F002031B041B0C83802D
:109BE000BFE5019009F0B0FAE56E019884F87800BD
:109BF000042384F88430002D3FF417AED4E91821F3
:109C0000236FA84794F88420531EFEE5D4F8C000C3
:109C100043F09CFC51463A20FEF7B0FCD4F8BC104F
:109C200082468B894FF0040E4FF47A7302A84FF0EE
:109C3000FF0C0A89920728D5A1F80CC04FF47A735B
:109C40000A89D20703F1FF3B2AD58A8992B208B16B
:109C500000F8012BBEF1010EEBD1BAF1000F0DD1CE
:109C600009F072FA029B1BBAC3F3807384F87A304E
:109C70002AE600BF601C00207D0F7D0F09F064FA0A
:109C800009F09EFA94F8842026E5013B9BB2AB4292
:109C9000CFD1084644F0D0FFBAF1000FEED1DFE794
:109CA0001FFA8BF3AB42CBD1F3E7D0F800C0DFF85B
:109CB000ACE003EA0C0C1CEA0E0F3FF4B1AD03EA72
:109CC0000E03836073E704212C20FEF721FA0321A1
:109CD00083464E20FEF71CFA0C21034636200193E2
:109CE000FEF716FA019B421C02339A400AFA0BFA5D
:109CF000A2FB0A01420A42EAC152C4F8882009F0D4
:109D000023FA4CE684F884208AE5E56ED4F800391D
:109D10006367072284F88420002D3FF481ADD4E9E5
:109D20001821236F0120A84794F88420531E6CE566
:109D300009F00AFA042384F8843076E508D0042375
:109D400084F8843009F000FA94F88420531E5CE50E
:109D5000FEF7D6FB02287FF455ADBFE57D0F7D0FE2
:109D60002DE9F04FC14C94F8E01083B00546C1F3E3
:109D70004001D4F8E80043F0F5FB94F8E010D4F883
:109D8000E400C94301F001016F1E43F0EBFBFBB29D
:109D90000193002D00F0D080B54EDFF8DC82B54D88
:109DA0004FF01009D4F8E80043F0C0FBD4F8E40009
:109DB00043F0BCFBB4F8F030002B40F04E8194F837
:109DC000F210D4F8F40043F0CDFB4FF0FA0A4FF450
:109DD0007A710120D8F80430C3F30803002B40F057
:109DE0000F81EFF31183002B40F00A81D6F8002990
:109DF000D5F808C0D6F800399A42F7D1D4F818310E
:109E00009C45F3D8D4F8147101FB07F3A3EB0C03C2
:109E1000B3FBF7F301FB0232D8F80430C3F30803B5
:109E2000002B40F0AB80EFF31183002B40F0A680B5
:109E3000D6F80039D5F808B0D6F80079BB42F7D18A
:109E4000D4F81871BB45F3D8D4F8147101FB07FCA2
:109E5000ACEB0B0CBCFBF7FC01FB03C39B1AB3F58B
:109E60007A7FD9D3BAF1010AB4D1D4F8E80043F02B
:109E70005DFBD4F8E40043F059FBB4F8F030002B5C
:109E800040F0DF8094F8F210D4F8F40081F0010182
:109E900043F068FBFA204FF47A714FF0010CD8F8C8
:109EA0000430C3F30803002B40F08980EFF31183E3
:109EB000002B40F08480D6F80029D5F808E0D6F8C9
:109EC00000399A42F7D1D4F818319E45F3D8D4F826
:109ED00014A101FB0AF3A3EB0E03B3FBFAF301FB9E
:109EE0000232D8F80430C3F3080343BBEFF3118305
:109EF0002BBBD6F80039D5F808B0D6F80079BB42AC
:109F0000F7D1D4F81871BB45F3D8D4F814A101FBEC
:109F10000AFEAEEB0B0EBEFBFAFE01FB03E39B1A3F
:109F2000B3F57A7FDDD30138B9D1019B5F1EFBB257
:109F3000FF2B01937FF436AF03B0BDE8F08FEFF352
:109F4000118A89F31288AF682B68DB0344BFC4F819
:109F500010C1AF68D6F80039D4F810E15FFA8AFA78
:109F60008AF31188D4F814A1734401FB0AFEAEEB06
:109F7000070EBEFBFAFE01FB03E3D0E7EFF3118E01
:109F800089F31288D5F808B02B68DF0344BFC4F802
:109F90001001D5F808B0D6F80039D4F810C15FFA2E
:109FA0008EFE8EF31188D4F81471634401FB07FC14
:109FB000ACEB0B0CBCFBF7FC01FB03C34EE7EFF370
:109FC000118E89F31288D5F808A02B68DA0344BFF4
:109FD000C4F810C1D5F808A0D6F80039D4F810217B
:109FE0005FFA8EFE8EF31188D4F814E11A4401FB57
:109FF0000EF3A3EB0A03B3FBFEF301FB023270E79F
:10A00000EFF3118C89F31288D5F808E02B68DB0395
:10A0100044BFC4F81001D5F808E0D6F80039D4F8E8
:10A0200010215FFA8CFC8CF31188D4F814711A4457
:10A0300001FB07F3A3EB0E03B3FBF7F301FB0232C3
:10A04000EAE6D4F80C31002B3FF424AFD4F8F83012
:10A05000C3F800A084F809A11CE7D4F80C31002B48
:10A060003FF4B3AE3FF026FEAFE600BFB03D0020A8
:10A07000C01B002010E000E000ED00E02DE9F04FF3
:10A08000BD4CBE4E94F8E010D4F8E800DFF8F4823E
:10A09000BB4D83B0C1F3400143F064FA94F8E01083
:10A0A000D4F8E400C94301F0010143F05BFA052351
:10A0B00001934FF01009D4F8E80043F037FAD4F8D0
:10A0C000E40043F033FAB4F8F030002B40F04C8158
:10A0D00094F8F210D4F8F40043F044FA32274FF425
:10A0E0007A710120D8F80430C3F30803002B40F044
:10A0F0000F81EFF31183002B40F00A81D6F800297D
:10A10000D5F808C0D6F800399A42F7D1D4F81831FA
:10A110009C45F3D8D4F814E101FB0EF3A3EB0C0338
:10A12000B3FBFEF301FB0232D8F80430C3F308039B
:10A13000002B40F0AB80EFF31183002B40F0A680A2
:10A14000D6F80039D5F808B0D6F800C96345F7D17C
:10A15000D4F818C1E345F3D8D4F814E101FB0EFCA0
:10A16000ACEB0B0CBCFBFEFC01FB03C39B1AB3F571
:10A170007A7FD9D3013FB5D1D4F8E80043F0D6F9BE
:10A18000D4F8E40043F0D2F9B4F8F030002B40F0FA
:10A19000E08094F8F210D4F8F40081F0010143F06B
:10A1A000E1F932204FF47A710127D8F80430C3F373
:10A1B0000803002B40F08B80EFF31183002B40F05D
:10A1C0008680D6F80029D5F808E0D6F800399A42FA
:10A1D000F7D1D4F818319E45F3D8D4F814A101FB77
:10A1E0000AF3A3EB0E03B3FBFAF301FB0232D8F838
:10A1F0000430C3F3080343BBEFF311832BBBD6F842
:10A200000039D5F808B0D6F800E97345F7D1D4F88D
:10A2100018E1F345F3D8D4F814A101FB0AFEAEEB24
:10A220000B0EBEFBFAFE01FB03E39B1AB3F57A7F2C
:10A23000DDD30138B9D1019B5F1E17F0FF030193F5
:10A240007FF439AF03B0BDE8F08FEFF3118A89F3E3
:10A250001288D5F808B02B68DB0344BFC4F810712E
:10A26000D5F808B0D6F80039D4F810E15FFA8AFAC8
:10A270008AF31188D4F814A1734401FB0AFEAEEBF3
:10A280000B0EBEFBFAFE01FB03E3CEE7EFF3118EEC
:10A2900089F31288D5F808B02B68DB0344BFC4F8F3
:10A2A0001001D5F808B0D6F80039D4F810C15FFA1B
:10A2B0008EFE8EF31188D4F814E1634401FB0EFC8A
:10A2C000ACEB0B0CBCFBFEFC01FB03C34EE7EFF356
:10A2D000118E89F31288D5F808A02B68DA0344BFE1
:10A2E000C4F81071D5F808A0D6F80039D4F81021B8
:10A2F0005FFA8EFE8EF31188D4F814E11A4401FB44
:10A300000EF3A3EB0A03B3FBFEF301FB02326EE78D
:10A31000EFF3118C89F31288D5F808E02B68DA0383
:10A3200044BFC4F81001D5F808E0D6F80039D4F8D5
:10A3300010215FFA8CFC8CF31188D4F814C11A44F4
:10A3400001FB0CF3A3EB0E03B3FBFCF301FB0232A6
:10A35000EAE6D4F80C31002B3FF423AFD4F8F83000
:10A360001F6084F809711CE7D4F80C31002B3FF40E
:10A37000B5AE3FF09FFCB1E6B03D0020C01B002011
:10A3800010E000E000ED00E000F01F0240090123B2
:10A39000032803FA02F304D004280CD0022805D0C5
:10A3A0007047074A116C0B4313647047044A516CA1
:10A3B0000B4353647047024A116B0B43136370479E
:10A3C0000038024000285FD00368374A2DE9F04189
:10A3D00003F13F4404F57E0402EB9422012492F839
:10A3E000C42002F01F055209032A04FA05F456D0CE
:10A3F000042A4FD0022A48D08588B5FA85F0C0F1EA
:10A400001F00C0F3CC0603EB860600F007008200B5
:10A410000F24306A944020EA04003062306A01FA66
:10A4200002F20243002132624FF0010E0A464FF061
:10A43000030C02270EFA02F838EA050002F10102C5
:10A440001CD118680CFA01F420EA0400186018689E
:10A4500007FA01F606431E609E6826EA04069E601F
:10A4600098689860586820EA0800586058685860F2
:10A47000D86820EA0400D860D868D860102A01F1B2
:10A480000201D7D1BDE8F0817047084A556C2C43D2
:10A490005464B1E7054A156B2C431463ACE7034AD7
:10A4A000156C2C431464A7E798D3060800380240C3
:10A4B000002861D00368384A03F13F4101F57E016D
:10A4C00002EB91222DE9F04192F8C42002F01F0422
:10A4D00052090121032A01FA04F158D0042A51D06B
:10A4E000022A4AD08588B5FA85F2C2F11F02C2F36A
:10A4F000CC0403EB840402F00702216A92000F20CF
:10A50000904021EA00012162206A0C2101FA02F246
:10A5100002430021226208464FF0010E4FF0030C67
:10A5200002270EFA00F838EA050200F101001DD1F9
:10A530001C680CFA01F224EA02041C601E6807FA87
:10A5400001F434431C609E6826EA02069E609E6801
:10A5500016439E605C6824EA08045C605C685C608A
:10A56000DC6824EA0202DA60DA68DA60102801F1B5
:10A570000201D6D1BDE8F0817047084A546C2143EE
:10A580005164AFE7054A146B21431163AAE7034AFC
:10A59000146C21431164A5E798D3060800380240E3
:10A5A00058B183884FF00042B3FA83F332FA03F3D1
:10A5B00003D002490A6813430B607047003C014016
:10A5C000134B0268196821EA02011960596821EAEF
:10A5D0000201596019680A431A609968026821EA01
:10A5E00002019960D96821EA0201D96041791029F4
:10A5F00007D001F1804303F59E3319680A431A60BE
:10A600007047996811439960D9680A43DA607047C6
:10A61000003C0140002864D0F0B58388B3FA83F38E
:10A62000202B0A4685B00446C3F11F0143D02D4DAF
:10A630002D4E05EB81037718C3F81C21002197F8F4
:10A64000CC703EF025FDB4F804C02268274CBCFA5B
:10A650008CFCCCF11F0303F0FC0101F1804101F5FA
:10A660009C3103F0030398004FF00F0E02F13F43BB
:10A670008A680EFA00FE22EA0E0203F57E038A6063
:10A68000C3F38723834088684FF0004222FA0CF21C
:10A6900003433D448B6002A8626101234FF40061D3
:10A6A0008DF80E300292ADF80C10FFF789FF95F887
:10A6B0005C31F02B01D805B0F0BD3E44F02196F896
:10A6C000DC308DF8043003224FF4807301A885F844
:10A6D0005C118DF80520ADF8063009F02BFD05B0B2
:10A6E000F0BD7047B03D002098D30608003C014003
:10A6F00010B4B8B10D4CD4F86431102B05D15DF80D
:10A70000044B052100203EF0ABBF03EB4302224483
:10A7100082F8691101210B4482F8680182F86A11FC
:10A72000C4F864315DF8044B704700BFB03D0020B1
:10A73000C0782021DCE700BF2DE9F04FDFF87CA3D3
:10A740002DED028B9AF8AC110022CAE96722CAE902
:10A75000692297B0CAF8982119B19AF8AD218AF800
:10A7600098219AF8AE211AB19AF8AF218AF8A72158
:10A770009AF8B2211AB19AF8B3218AF8A2219AF86C
:10A78000B0211AB19AF8B1218AF89D219AF8B43112
:10A7900005935A1ED3B257B204937B1C00F0AA80D3
:10A7A000BC4ABD4E52F83780029602EBC702002326
:10A7B0001279019308EE102A1D46344699462678F0
:10A7C0003946304645F0F6FE83463046BBF1000F71
:10A7D0001ED042F0CBFBEA1D1321D2B220B14FF0C4
:10A7E000000E827180F807E03EF052FC207845F0C0
:10A7F00013FF4FF0070309F1010223714FF001032A
:10A8000084F802906070CDF804B05FFA82F9E370CA
:10A810000135042D04F10504D1D118EE100A029E71
:10A82000CDF80C90FFF7B0FD9C499D4A4868024066
:10A8300042F440324A600FB9019B5BB9994C482001
:10A84000FFF7A2FD204602215EF00EF9A26842F059
:10A850000102A2609148934A4168BAF8B64141F4B6
:10A8600000014160516821F480515160916B21F4E5
:10A87000401141F480119163D16841F46001D160CD
:10A88000956B85F44011C1F3015101EB81011F204B
:10A8900000FA01FC25EA0C0C112505FA01F141EA48
:10A8A0000C019163D16841F4E011D160956BC5F35F
:10A8B0000151C1F10401C9B201EB810188404FF09F
:10A8C000100C25EA00000CFA01F108439063E4B192
:10A8D000BAF8B811CAF8C041A1B1BAF8BA21CAF899
:10A8E000C41162B1019B7048521A90FBF2F2CAF88F
:10A8F000C8216BB917B0BDEC028BBDE8F08F6B4A75
:10A900001288EFE76A4A1188E7E76A4A1488DFE7A6
:10A91000404603995EF0A8F85F4B012003F114094B
:10A920000723F278441CE4B252B375783279A5F16A
:10A930000A0101EB410105EB450C092D03FA01FE6B
:10A9400003FA0CFB02FA01F140F28E80D8F80C20D9
:10A9500022EA0E0E41EA0E01C8F80C10421E02EB6C
:10A9600082021F21062801FA02FC05FA02F261D8D0
:10A97000D8F8341021EA0C010A432046C8F83420E4
:10A980000536B145CDD1D8F80820049942F40072BB
:10A99000C8F80820D8F8082042F48072C8F80820C7
:10A9A000D8F80820574442F00102C8F8082097F967
:10A9B000BC2102203FF04CFD044600289AD040689C
:10A9C0005CF07CF8059A06215CF08AF8606809F072
:10A9D00059FC07A809F018FC039EA368364A0793A0
:10A9E000012E8CBF4FF48060002000230D9008F1F1
:10A9F0004C054FF40060089509920A934FF4807259
:10AA00000C930E904FF4003360680B9607A94FF437
:10AA10000055CDE90F52119309F008FC62681368E4
:10AA200043F001031360D8F8083043F08043C8F8BE
:10AA300008305FE7C11FA0F10D0201EB81014FF06B
:10AA40001F0E02EB82020C280EFA01FC0EFA02F035
:10AA500005FA01F113D8D8F8302022EA0C0211438C
:10AA60002046C8F830108BE7D8F8101002FA0CF224
:10AA700021EA0B0B42EA0B02C8F810206EE7D8F867
:10AA80002C1005FA02F221EA00010A432046C8F818
:10AA90002C2075E77CD40608483F002000230140A5
:10AAA000E030FCFF00200140803801002E7AFF1FBB
:10AAB0002C7AFF1F2A7AFF1F7C3F0020B03D002028
:10AAC000F8B5264E00EBC00406EB8404D4F8D85148
:10AAD000002D36D094F8E9C10CF0FF07BCF1000F4F
:10AAE0002FD149004FF0010CC9B284F8EA1184F863
:10AAF000EB2184F8EDC184F8EE7184F8ECC184F8A0
:10AB0000E9C184F8E871AA88C4E97C33940502D5C8
:10AB100001273846F8BD2B88D9050CD44FF4805353
:10AB200001E0013B10D02A889205FAD42B889BB211
:10AB300043F480732B80AB889BB243F44073AB80AB
:10AB4000E6E700273846F8BDB6F8403201339BB23D
:10AB5000A6F840325DF034FCDBE700BFB03D0020DA
:10AB600070B5464E96F8424204EB440306EBC3032D
:10AB7000650093F84432032B6ED8DFE803F05929BF
:10AB80001E02254406EBC505D5F84802002870D101
:10AB900096F8A4329C425FD0013404F00302934241
:10ABA00086F8422258D002EB420406EBC40402238A
:10ABB000C4F8480284F8443270BD2B1906EBC30375
:10ABC000D3F8482272B1013AC3F84822002070BD80
:10ABD0002B1906EBC303D3F84822002AF3D1022233
:10ABE00083F84422254406EBC50595F85032013B15
:10ABF000DBB285F850328BBB214B96F8A462D3F8B8
:10AC00003012D5F84C02621C02F003024B1E0324E2
:10AC1000B242034485F84442B3FBF1F0C5F8480260
:10AC20001AD0994218D80138C5F84802012070BDE1
:10AC300044F02EFB80B1124B2C44D3F8302206EBAB
:10AC4000C404012102F51C5384F844120F33B3FBF2
:10AC5000F2F3C4F8483270BD012070BD084BD3F840
:10AC60003022012002F2E733B3FBF2F3C5F8483299
:10AC700070BD0138C5F84802002070BDB03D00200D
:10AC800088010020054B93F8A522002AFBD1D3F8B8
:10AC9000083E03491B6801F10C001847B03D002035
:10ACA000584000202DE9F84F3249DFF8D4B091F830
:10ACB000851001240229074619461046CBF82C407E
:10ACC0004FF000022C4C1D4618BF7F02FDF798F98B
:10ACD0002A4B63626B02A362E36A40F2FF5943F0BE
:10ACE00093034FF400704FF48A62E3620121C4F8C9
:10ACF0003890A0601020E26059F0DAFA012D40F29D
:10AD000051434E46C4F83890CA4640F252488EBF6E
:10AD10004FF0120998464FF011090A25C4F838A0DF
:10AD20000121A7604846C4F80C8059F0C1FA0346D7
:10AD30004FF0000C40F2774201213720A6632BB977
:10AD400000231846CBF82830BDE8F88FA663C4F876
:10AD500008C0E26059F0ACFA013DA6630028EFD0CC
:10AD600015F0FF05DAD10346CBF82C50CBF828308C
:10AD7000BDE8F88FB03D0020002C014000E1F50552
:10AD8000C01B00202DE9F843184C94F88460042E71
:10AD90000546894690461F4608D0082E02D000205E
:10ADA000BDE8F883FEF776F90228F8D101234A4678
:10ADB00028460021FFF776FF50B1FEF7F5F9E56E62
:10ADC000002DECD00022236F616E1046A847E6E705
:10ADD000D4F80039C4F860900522C4E91B87656681
:10ADE00084F8842063670120BDE8F883C01B00203D
:10ADF0002DE9F84F2F49DFF8C49091F885101E46D1
:10AE000002292D4B07464FF0010418BF4702012EBF
:10AE100040F259481C6398BF4FF48B683B469346F9
:10AE2000474640F2FF55B0468CBF4FF0190A4FF02D
:10AE3000180A0A241E4640F2FF53C9F8383001218F
:10AE4000C9F808605046C9F80C7059F031FA034649
:10AE50004FF0000C40F2774201213720C9F83850FA
:10AE6000A3B9584641460122FDF7CAF84646134A9F
:10AE7000134B536276029662D36A43F09103D36216
:10AE80000D4B002108469962BDE8F88FC9F838508B
:10AE9000C9F808C0C9F80C2059F00AFA013CC9F8F1
:10AEA00038500028DDD014F0FF04C4D1024B1C63DD
:10AEB000BDE8F88FB03D0020C01B0020002C0140F1
:10AEC00000E1F5052DE9F047374C82B005460E4606
:10AED0001746984694F8840004280CD0082806D118
:10AEE000E36FAB4207D0FEF7D5F80228F2D001207D
:10AEF00002B0BDE8F087DFF8B8A02666DAF87C90EB
:10AF00006566C9F34F210F294FEA592223D8D4F897
:10AF100080300193FBB194F8CD00E0B1B9F5005F4A
:10AF200013D0224831464FF40072484462F082F94F
:10AF300009F50072C2F34F211029CAF87C204FEAAC
:10AF4000522202D0019B012B21D192B2013A174E1D
:10AF5000AD1A0B4600E0012332462846062601259D
:10AF60000021E766C4F8708084F8685084F8846033
:10AF7000FFF73EFF0028BBD0FEF716F9E66E86B15C
:10AF80002846236F616E0022B0470320B0E7E26FCE
:10AF9000013B01320421C4E91F2384F884100220FC
:10AFA000A6E70320A4E700BFC01B0020E05E00204E
:10AFB000B03D002070B52E4D95F80C4E022C84B09B
:10AFC0001AD0012C02D0002004B070BD95F9104EAB
:10AFD000631CF8D0032CF6DC0091134695F8111E83
:10AFE000024620465DF07EFB0028ECD0204604B0EF
:10AFF000BDE870405DF012BCD5F8143E13B11C687A
:10B000009B886383D5F8106EB38940F2E9343389A5
:10B01000013C13F0020FA4B219D084B2B48140F203
:10B02000E9343389013C13F0010FA4B21BD0B3897A
:10B03000134630460A4600215DF07CF8D5F8143EF0
:10B04000A3B11A689B881383012004B070BD002C43
:10B05000DDD13046CDE9021243F0EEFDDDE902120A
:10B06000D5F8106EE4E7002CDBD1F2E70120ABE766
:10B07000B03D002010B50278022A044613D0012A00
:10B0800001D0002010BD2D4B90F9040083F84C2E08
:10B09000421CF6D00328F4DC0A4603F64C636179BF
:10B0A000BDE810400CE5836813B11A689B88538390
:10B0B0006368988940F2E9321889013A10F0020F6A
:10B0C00092B225D089B2998140F2E9321989013AC8
:10B0D00011F0010F92B22BD09A899A8940F2E9328D
:10B0E0001989013A11F0020F92B21ED001229A8101
:10B0F00040F2E9321989013A11F0010F92B20ED0F3
:10B100009B89A368BBB11A689B881383012010BD7B
:10B11000002AD1D1184643F08FFD6368DDE7002A8D
:10B12000E8D1184643F088FDEBE7002AD8D1F8E7CC
:10B13000002ACBD1EEE7012010BD00BFB03D0020BA
:10B1400010B50C4C94F80C3E022B11D1D4F8140E0F
:10B1500042F002FAD4F8140E08B12123C380012171
:10B160003DF096FFBDE810400348082143F01ABDAA
:10B1700010BD00BFB03D0020BC4B002073B50D4E8C
:10B1800005460C46FF230A46014630468DF8073037
:10B1900043F03AFE01230DF1070245F080013046ED
:10B1A00043F0F6FD9DF80700031B5842584102B0DA
:10B1B00070BD00BFBC4B0020094B93F87E34042BBC
:10B1C00008D9053B032B08D801231A4600B10370A8
:10B1D0001046704700230122F8E700231A46F5E7DE
:10B1E000B82C0020F0B40D6800240CE0BCF1050F71
:10B1F00018D8A0F137030A2B14D104EB840415F8F6
:10B20000010B03EB4404A0F13003DEB2092EA0F1E0
:10B210006107A0F1410CF0D9052FE7D8A0F1570341
:10B220000A2BEAD00D601460F0BC70479FED737A72
:10B2300007EE901A20EE070AF8EE677A27EE800AEA
:10B24000FDEEC07A17EE903A2033402B00F2C78013
:10B25000DFED6B7AB4EEE70AF1EE10FAF0EE407A29
:10B260000CDD9FED686ADFED686AB0EE677AB4EED8
:10B27000E67AF1EE10FA77EEC67AF6DC9FED637AA5
:10B28000F4EEC77AF1EE10FA0CD59FED5E6ADFEDB1
:10B29000606AB0EE677AB4EEE67AF1EE10FA77EE15
:10B2A000867AF6D49FED5B7AF4EEC77AF1EE10FA67
:10B2B00000F38D809FED587AF4EEC77AF1EE10FA24
:10B2C00044BF9FED527A77EE677A27EEA76ADFEDEB
:10B2D000535A9FED537ADFED536AA6EE257A67EE57
:10B2E000865AE6EE076AB6EE007AE5EEA67A27EE13
:10B2F000877ADFED486A70EE267ABDEEE76A16EED1
:10B30000103A2033402B67D8B4EEE60AF1EE10FA7B
:10B310000CDDDFED3C5A9FED3C6AF0EE676AF4EE1F
:10B32000C66AF1EE10FA77EEE57AF6DCDFED376A01
:10B33000F4EEE67AF1EE10FA0CD5DFED325A9FED1D
:10B34000346AF0EE676AF4EEC66AF1EE10FA77EE50
:10B35000A57AF6D4DFED2F6AF4EEE67AF1EE10FA74
:10B3600040DDDFED276A76EEE77A67EEA75A9FEDBC
:10B370002B5A9FED2B6ADFED2B6AA5EE856A27EE2F
:10B38000A55AE5EE866AB8EE006AE5EE267A67EE23
:10B39000867AC7EE206A0023836143610362C3613A
:10B3A000B7EE006A76EE865A76EE666A86EE257A03
:10B3B00067EE277A66EE876AC0ED017AC0ED037A00
:10B3C00080ED007A80ED027AC0ED046A70479FED4F
:10B3D0000C7A77EE677A78E7DFED137AD9E79FED9D
:10B3E000127A86E7DFED0C6AF4EEE67AF1EE10FAF7
:10B3F00044BFDFED066A76EEE77AB6E727D4D236A9
:10B40000DB0F4940DB0FC940E4CB1641DB0F49C0DD
:10B41000E4CB16C1DB0FC93FDB0FC9BF92E741B9CF
:10B420009730083C15A82ABE000000002DE9F04125
:10B430008C4B82B093F84D2E0190002A40F00C8185
:10B4400093F8702EB3F8721EDFED876AB3F8748E2E
:10B45000864D07EE102A07EE901AB8EEC76AB7EECF
:10B46000007AB3F86E1EA5F80081F0EE475A4FEA55
:10B470004804E6EE665A8C42B8BF0C46A6EE267A21
:10B48000A6B20121F8EEE77AA5F8046167EEA67A84
:10B49000C5ED3D5A85ED3E7AC5ED3F7A83F84D1EE8
:10B4A000002A00F0D680DDED017A9FED710AF8EEFA
:10B4B000677AA4B280EE270A5FF0B8FB6400B0FBA5
:10B4C000F4F4012CB8BF0124E4B2B0FBF4F39BB256
:10B4D000074685F8084100EE103ABBEEED0A85ED0F
:10B4E000430A5FF0A3FB634BDFED636AB8FBF0F048
:10B4F000A3FB0737FF0807EE907AF8EEE77A0228F9
:10B5000086EEA77AB8BF02205C4985F810010023B7
:10B510009FED5B1A9FED5B6ADFED5B1ADFED5B5A17
:10B520009FED5B2ADFED5B2A9FED5B3ADFED5B3A37
:10B530009FED5B4A85ED457A07EE903AB8EEE77AE3
:10B54000F0EE467AE7EE017AFDEEE76A16EE902A13
:10B550002032402A7AD8B4EEE17AF1EE10FA0CDD0E
:10B56000DFED506A9FED507AB0EE675AB4EEC75ADD
:10B57000F1EE10FA77EEE67AF6DCF4EEE57AF1EE2B
:10B5800010FA0CD5DFED476A9FED487AB0EE675AA6
:10B59000B4EEC75AF1EE10FA77EEA67AF6D4F4EECE
:10B5A000C67AF1EE10FA49DD74EE677A67EEA76AA3
:10B5B000F0EE624AE6EE824AF0EE430AE6EEA40AB4
:10B5C000B7EE007A27EEE65A77EE677AB6EE007AA3
:10B5D000E5EE207A67EE877A0133202BE1EC017AE1
:10B5E000AAD107EE904AF8EEE77AF7EE006A86EE07
:10B5F000A77A2F4B2F4AC5F8B43703F12801A83397
:10B60000C5F8B0171020C5F8C0372021142385F8DD
:10B610001146A5F8AC07A5F8BC1707EE906AF8EE3E
:10B62000677AA5F8B83782ED007AC2EDAC7AC2ED40
:10B63000AD7AC2EDAE7A02B0BDE8F081F4EEE37A05
:10B64000F1EE10FA48BF75EEE77AAFE7F6EE007A52
:10B65000C2E7194B1A7026E7044D95F80841B5F872
:10B660000461BEE7B03D00200AD7233C140000105F
:10B6700000247449ABAAAAAADB0FC9412C0100100F
:10B680003C8C4F3EDB0FC93F0100F840DB0F49C047
:10B6900092E741B99730083C15A82ABEDB0FC9BF15
:10B6A000DB0F4940DB0FC940E4CB1641E4CB16C1A8
:10B6B00094D4060828060010000000100848002353
:10B6C00002461178022902F1060204D00133062B4A
:10B6D000F7D10020704703EB430300EB43007047B2
:10B6E000F81B002010B50021094C82B00846C4F8B0
:10B6F000781E34F0D9FD074B0193042304F67C60D7
:10B700000DEB0302062143F009FB02B010BD00BFA0
:10B71000B03D00205475C52A70B5461E00F13105B4
:10B72000344614F8011F601E801BFF29C0B201D0EF
:10B7300034F0BAFDAC42F4D1A02052F04BF8012114
:10B74000022034F0B1FD0E4D40F2E93401E0013C3D
:10B7500005D04221284643F093FA0028F7D1622110
:10B76000074843F08DFA1321242034F09DFD252055
:10B77000092134F099FDBDE87040A02052F02AB8AC
:10B780002C4C00202DE9F04F2DED108B034697B087
:10B7900004331593DFEDCACA149002238A4613922C
:10B7A0008B461293149C4FEADB0604EB461202EB25
:10B7B00006103101A6EB86034FEAC60806EB4605E4
:10B7C000CDE9000100EBC303043108F10400119638
:10B7D000204421442C01C6EBC60C0394EC00119DBF
:10B7E00004944FEACC0405946C0106EB860E029497
:10B7F000159D009C03EB46174FEACE0E02EBC606E2
:10B800004FEACB094FF0000C51ED01AAD3ED001A1D
:10B8100092ED007A94ED005A96ED004AD7ED007A49
:10B8200015ED012A50ED016A32EE07BA76EE840A70
:10B830007AEE855A31EEA70A3BEE256A70EE804A11
:10B8400076EEC46A36EE244A36EE646A05ED014AA5
:10B8500082ED006AD0ED00BAD6ED012AD3ED019A4F
:10B8600095ED00AA92ED016A97ED013A91ED00CABB
:10B87000D4ED014A7BEEE23A36EEE19A32EE472A07
:10B8800073EEE98A3AEE464A39EE279A78EE838AD1
:10B89000B0EE428AA9EE6C8ADC44E24573EEC33A0C
:10B8A000B0EE441AA8EEEC1A76EEE77A33EEA97AF7
:10B8B0007CEE643A77EEA17A3AEE066A7AEEC51A21
:10B8C0003CEE24AA74EECC4A39EE833A35EE6A5A3D
:10B8D000F0EE639AF0EE48AAE7EE2C9AA8EEAC4A96
:10B8E000E7EE2C4AE7EE6CAAF0EE418AB0EE427A1F
:10B8F000B0EE612A7BEE656A7BEEA22A76EE4A5AAA
:10B90000A9EE2C7AA7EEAC2AA7EEAC5AE7EEEC8AA9
:10B9100032EE83BA76EEC3BA35EEE09A75EEC07AAF
:10B9200036EE0A6A76EEE26A36EE0BAA76EE836AA5
:10B9300077EEA07A34EE423A77EE290A36EE4B6A79
:10B940007BEEA22A39EE000A73EEAA3A78EE244A78
:10B9500037EE697A31EE055A71EEA85A32EE044A92
:10B9600085ED00AA82ED016A4D4441ED012A4A4469
:10B97000C4ED006A81ED000AC4ED017A494440ED4E
:10B98000010A4C4487ED007AC6ED003AC3ED004A47
:10B9900080ED003A87ED014A484486ED015A4F4454
:10B9A000C3ED015A4E444B443FF62EAF119B072B7B
:10B9B00040F2C781029D149E019B03980499059A49
:10B9C000083575190C330E95354608F108080EF147
:10B9D0000804EB1808300831083246442C1928189E
:10B9E0006918AA18079305F10C030D960C940B9097
:10B9F0000A91099208934FF001084FF0000E129B34
:10BA00009E44139B03EBCE0303EBCE02109302EB99
:10BA1000CE0303EBCE01029101EBCE0101EBCE058B
:10BA200005EBCE06D6ED007A0F93AEEB8E030191B7
:10BA300006EB031303EBCE07D3ED01AACDED067A97
:10BA4000019BD5ED007A97ED01BACDED057AD3EDE6
:10BA5000007A029BCDED047AD3ED007A0F9BCDEDF9
:10BA6000037A07EBCE0CD3ED007ADCED01BACDED15
:10BA7000027A0CEBCE01D2ED007A109A009101EB24
:10BA8000CE00014691ED01DACDED017A0099D2EDBB
:10BA9000007A91ED01CA00EBCE0000EBCE0494EDEC
:10BAA00001EAD0ED01DACDED007ADDE90776DDE9D6
:10BAB0000954DDE90B01DDE90D23C44602E000BFB6
:10BAC000F304353F94ED009A90ED00FA91ED006A91
:10BAD000D5ED007AD3ED006A57ED014A92ED005A98
:10BAE00056ED013A96ED00AA35EE060A73EEA65A17
:10BAF00039EE278A34EE8F7A70EE082A75EE87EADF
:10BB000035EE465A3EEEA26A73EEE63A06ED016A5B
:10BB1000D1ED019AD2ED01FAD4ED016AD3ED011A0B
:10BB200095ED013AD0ED018A97ED004A3FEEE96AC2
:10BB300035EE491A76EE660A31EE271A3AEE612A98
:10BB400075EE677A70EE830A3FEEA95A74EECF9ACB
:10BB500077EE897A7AEE211AB0EE42AA74EE68FA8C
:10BB6000A0EEECAADC44E24535EEC77AB0EE639A6B
:10BB700074EE285A38EEC44AF0EE698AA1EE6C9A47
:10BB8000E7EEAC8A36EE436A7FEE644A36EE266A0A
:10BB9000A0EEAC2AF0EE4A0AE7EEEC0AE7EEAC4A79
:10BBA000F0EE687AF0EE498A36EE833AE6EE6C8A79
:10BBB000E1EE2C3AB0EE6F1AA6EE2C1A71EEE56AA1
:10BBC000A6EE2C4A71EEA55A75EE031A7EEEE22A15
:10BBD00037EE43FA75EEE1EAB0EE686A76EEC08AB7
:10BBE00039EE044A7FEE86FA76EEC86A33EE816A51
:10BBF00038EE888A73EEC13A37EE457A2CEE2E1A6B
:10BC00003FEE055A22EECC9A9DED03FA70EE266ABD
:10BC100033EE077AAFEE221AAFEE2E9A7AEE244A6E
:10BC20009DED01FA79EEA09A25EE4BAA72EE670A15
:10BC300037EE822A6BEE087AAFEE08AAEFEE057AAD
:10BC40002DEEA63A9DED05FA67EE6D8AAFEE073A46
:10BC5000EFEE268A66EE6A2A9DED00FA2AEEA00A29
:10BC6000EFEE202A6EEE02EADDED060A23EECE5A52
:10BC7000E0EEA3EA2BEEA98ADDED023AAFEE060A6A
:10BC8000A3EE848A24EE6B7A6DEE246A9DED044A5D
:10BC90002FEECD6AA0EE825AA3EEA97AE4EE2F6AC7
:10BCA000A4EE246A75EEA15AC6ED005A83ED001A7F
:10BCB00083ED019A4E4447ED017A87ED00AA4B448B
:10BCC00080ED003AC0ED018A4F4482ED000A4844FD
:10BCD000C2ED012AC5ED00EA85ED015A4A44C1EDE5
:10BCE000006A81ED016A4D4484ED008A84ED017A99
:10BCF00049444C443FF6E6AE0E9B08330E930D9B31
:10BD000008330D930C9B08330C930B9B08330B9358
:10BD10000A9B08330A93099B08330993089B08334D
:10BD20000893079B08330793119B08F101084345CB
:10BD30007FF465AE129BDDF844B0DB009BB212933A
:10BD400030E517B0BDEC108BBDE8F08F30B5044680
:10BD500083B000BF806841F0F9FB4CF2050301AAF3
:10BD60006946ADF800306068032300258DF8025065
:10BD70005CF0E0F9A06841F0EFFB00BF9DF8060021
:10BD800003B030BDF0B5BE4FBE4885B024220021BF
:10BD900061F0B1FA97F8896E002E3AD1BA4C354667
:10BDA000D4F8443D5BB39B6A4BB3B848984783686B
:10BDB0002BB30388DFF8CCC2013B9BB260466646DA
:10BDC00000213778032F06F106061BD00131062922
:10BDD000F7D100220178022900F1060000F0A580C9
:10BDE0000132062AF6D1E16D052908D0481C02FB74
:10BDF00001C2E06502200021938010705180284626
:10BE000005B0F0BD062303FB01414B8F013B9BB204
:10BE1000DFE797F8880E07F56963C7F88C3E10B91D
:10BE2000994C0025BCE741F0A1F80446C7F8980EEC
:10BE300041F070FB05460028F2D0013E022370B2AB
:10BE400087F8903E43F062F80028E9D0C7F8940ED6
:10BE50000CB12023E380204609213DF019F9D7F8E1
:10BE60008C3E894C986841F077FBD7F88C3E1021C6
:10BE700058685CF02DF9864BD7F88C2EC4F8642DE9
:10BE800093E803000123009032208DF8041084F819
:10BE9000683D00263DF04AFE052302AA6946D7F810
:10BEA0008C0E8DF80A608DF8096042F0B3FE9DF8A3
:10BEB0000A009DF809109DF80B20764B000240EA1D
:10BEC00001401043984200F0AE8032DCA3F5F1133C
:10BED00098425ED042DD704B984252D00233984275
:10BEE00062D14FF400724FF48073A4F8482DA4F887
:10BEF000543DB4F8542DB4F8483D120202FB03F34C
:10BF000000204FF48071B3F1807FC4F84C2DC4F849
:10BF1000503D84F8560DA4F84A1D7BD85F4BC4F8F9
:10BF2000443D012284F85D2D3AE7062101FB02C25F
:10BF300060E75B4B984234DC053B984234DD594B5B
:10BF40000344032B77D801A252F823F093BF0008D3
:10BF500083BF000875BF0008E3BE0008A3F52203F5
:10BF6000013B984267D051DD4F4B984209D00133D5
:10BF7000984219D14FF48073A4F8483DA4F8543D79
:10BF8000B7E780224FF48073A4F8482DA4F8543DFD
:10BF9000AFE740224FF48073A4F8482DA4F8543D35
:10BFA000A7E7424B9842E5D00023A4F8483DA4F807
:10BFB000543DC4F84C3DC4F8503DFCF70DFC03461D
:10BFC00000287FF4EDAE9DF80B009DF80A209DF847
:10BFD0000C10000240EA0240354A0843904232D039
:10BFE000A4F8483DA4F8543DC4F84C3DC4F8503D75
:10BFF000FCF7F2FB064600287FF4D2AE97F8880ED5
:10C0000040F0B4FF42F0AEFD3546C9E6294B9842F8
:10C01000B0D0C9E70123D4F8640D84F85C3DB721A2
:10C0200050F0E0FF7AE74FF480621023A4F8482D27
:10C03000A4F8543D5DE720224FF48073A4F8482D06
:10C04000A4F8543D55E71C4BC4F8483D4FF400316B
:10C0500040234FF000620126A4F8543DC4F84C1D63
:10C06000C4F8502D84F8566DFCF72AF8074884F878
:10C070005D6D50F009FF114BC4F8443D90E600BFE0
:10C08000B03D0020F81B0020C01B00200429002028
:10C09000BCD506081640E0001720C20098D3060859
:10C0A0001940EF00EABF10FF17BA20001870EF0028
:10C0B00021AAEF001860010000040008C4D306089C
:10C0C0002DE9F041C94BCA4ECA4DCB4C0822C3F8EA
:10C0D0008820336B82B043F00103336307464FF48B
:10C0E000C052284640F2023388466946CDE9002313
:10C0F00008F05EFB6B6AC14ADFF848C323F4704363
:10C100006B626B6A43F420436B626B6A23F47023A7
:10C110006B626B6A43F420236B62736CB84D43F41B
:10C12000804304F5A4517364736BC1F8008041F23D
:10C13000884143F08003675041F2844EB1497363F4
:10C140000227C4F8A01EB04EB04BB14944F80E50BF
:10C1500084F8A47E4FF0A045AE4FC4F8A85EC4F8A2
:10C16000AC6EC4F8B43EC4F8F01E05F5326506F5B1
:10C17000A07603F51073A1F5D071C4F8B87EC4F8A9
:10C18000F45EC4F8BC6EC4F8F83EC4F8C01E0123C7
:10C1900007F51077A5F5E465A6F5A066A1F58C6115
:10C1A000C4F89CCEC4F8FC7EC4F8B05EC4F8686FD6
:10C1B00084F8A73E05F5A075536106F5B076C4F87E
:10C1C0002C1F84F8AE3F1946934B944AC4F8345F51
:10C1D000A7F5BC67A035C4F8406F914EC4F83C7F0A
:10C1E000C4F8443F07F5D45703F56953C4F8485FD2
:10C1F0004FF050250020DFF850E2DFF850C2C4F8BD
:10C200006C2FC4F8707F02F5A04207F5A047C4F870
:10C21000746FC4F8783F06F5A046A3F54853C4F8F8
:10C220007C5F04F69C65C4F8802FC4F8886FC4F85E
:10C23000A83FC4F830EFC4F838CF0246C4F8847F72
:10C240002B4684F8B00F402683F81C21A3F8222146
:10C250000132042AC3E9496083F81D1183F81F01E4
:10C26000C3F8300103F12803EED1002211462B461A
:10C27000402083F87423A3F87A230132042AC3E907
:10C28000DF0183F8751383F87713C3F8881303F17C
:10C290002803EED14FF0A04362489A6822F00102D1
:10C2A0009A60DA6842F04002DA6007F007FB94F81F
:10C2B000A53E0022212161F317420BB142F4801206
:10C2C00094F89F1ED4F8A83E01299A6300F0E380F9
:10C2D000DA68D4F8A86FD4F8AC0EC2F3076121F085
:10C2E000600141F0400161F31F620021DA603160BA
:10C2F000026861F3CC22026094F8A72E012A00F0B4
:10C30000B7801021484807F02BFE474807F00EFE83
:10C31000D4F8AC0E94F89D3E00224FF0FF3102613C
:10C3200042618161C26153B305F114073F4E11466A
:10C3300007EB83074FEA830C4FF0FF0E56F8042FEC
:10C340001368002BACBF00234FF09043B74213603B
:10C350001161C2F808E0F1D105F15003344963449A
:10C360000027FF2651F8042F1568002DACBF0025CB
:10C370004FF090459942156017619660F2D10369BC
:10C3800094F89F1E43F480730129036160D0D4F8B0
:10C39000A82E28480023936100294FF0FF336FF047
:10C3A000804151615360516114BF0023102390619B
:10C3B00043F47013916943F4605343F008030B4353
:10C3C000936141F284419368615843F001039360A3
:10C3D0000B689847184B194ADA606846184B009367
:10C3E00007F0A8FE02B0BDE8F08100BF00E100E068
:10C3F0000038024000000240B03D0020003C0140F7
:10C40000BC0300204000400100080050000900501B
:10C41000000B005020090050C005005000100050D3
:10C4200000300050584C00204C4C0020604C002044
:10C430009C4C00200008008000ED00E00005FA059B
:10C44000430200010804010020050050600500506F
:10C45000D4F8A82E144B03636FF08041134D0023D2
:10C460004FF0FF30936151615060516195619FE7DA
:10C4700001680F4A0F4E41F00301016080215962AB
:10C480009E62C3F80421E022C3F80821C0F24002F2
:10C49000C3F80C2135E79A6822F03E0141F02A01E9
:10C4A00061F307029A6013E703018100000800802E
:10C4B000A00040008000200010B51A4C94F89A03A8
:10C4C000C0B9194B83F8B100C3F8B40094F89D3398
:10C4D000012B05D0022B21D0D4F8A0331BB910BDFD
:10C4E000124BC4F8A03312495B68BDE81040A1F1BB
:10C4F0000C00184740F03AFD94F89C230A49003A92
:10C5000018BF012281F8B120C1F8B4000028DDD0A5
:10C510001F22C28020213CF0BBFDD7E7054BC4F8A9
:10C52000A033E0E7A84E0020C01B0020FC03002041
:10C530004C520020D803002099B10A6B824216D9D0
:10C54000154BD3F8E423914221D34C3991421ED3A9
:10C550000B6B9842F9D38B6B9842F6D80B46184672
:10C5600070470D4BD3F8E4130A6B904212D30B685B
:10C570000BB9F4E70A6B90420B4602D38A6B9042E8
:10C58000EDD951F84C3F002BF4D1184670470023E9
:10C59000184670470A46D8E7A84E00202DE9F04714
:10C5A000CC0143D10346224A43F8082B4FF0FF3217
:10C5B0004260022418467E26DFF87880D8F8E89397
:10C5C0002644013E051D49466FF070474FF0010AB1
:10C5D00008E0A3421CD0631C45F8043C321B1C46F7
:10C5E0000435CAB10B6BA34202D88B6BA34204D2B1
:10C5F0002046FFF7A1FF014690B10A794B6B002A54
:10C60000E7D1A34204D0E6D245F8042C631CE5E749
:10C6100045F8047C631CE1E7C8F8E813BDE8F0873F
:10C6200045F804AC321B631C4946D8E78026C3E7B3
:10C63000F8FFFF0FA84E0020036870B55E6A26B1B0
:10C6400033460522BDE87040184704460D464E1D8E
:10C6500000E023689B68204698470028F9D02368AB
:10C6600015F8011B1B6820469847B542F1D170BDF3
:10C67000036870B55E6A26B133460822BDE8704093
:10C68000184704460D4601F1080600E023689B6840
:10C69000204698470028F9D0236815F8011B1B682D
:10C6A00020469847B542F1D170BD00BF2DE9F04753
:10C6B000164D0746002095F9F59305F57F7684B071
:10C6C00007EB010805F29C6504464FF0B60A336893
:10C6D000ABB193F83830142B11D019F1020F01D0FF
:10C6E0004B450CD1002269463046CDE90244CDE9E4
:10C6F0000078ADF808A08DF80E4034F093FCE036D9
:10C70000B542E4D104B0BDE8F08700BFA84E0020D8
:10C710002DE9F743124E0124A02318255FFA84F86F
:10C72000FF2B14DCD6F89C06E9B2C1F11C02827220
:10C730005F1C026880F80B80DBB20093C1F11B0123
:10C74000D2F8189000234246C9B2C8473B46013D83
:10C75000E6D10134052CE0D103B0BDE8F08300BF81
:10C76000A84E002010B50A4C94F8B906003818BF3E
:10C770000120FBF757FF50B1064904F5D46042F0A1
:10C7800081F904F5D46010F0BFFA04F5D46010BD4F
:10C79000A84E0020C4D5060870B4447941BB036894
:10C7A0004FF400524FF40076202502213CBB1A8C36
:10C7B00022F001021204120C1A841A8B188C22F037
:10C7C000F30280B2120420F00A00120C014342F07E
:10C7D000010241F001011A8319841A8B22F00C0224
:10C7E0001204120C1A831A8B92B270BC1A8370470F
:10C7F00000220368164615461146002CD7D0042C9B
:10C8000021D0082C38D0198C21F480510904090C4E
:10C8100019849C8B1D8C45F6FF7040F6FF41284023
:10C820002140024342F4805241F4807199831A847A
:10C830009A8B22F440621204120C9A839A8B92B261
:10C8400070BC9A8370471A8C22F010021204120CEA
:10C850001A84188B198C89B240F6FF4221F0A0018E
:10C8600002400D4342F4807245F010051A831D8486
:10C870001A8B22F44062B3E71A8C22F480721204FD
:10C88000120C1A84998B1A8C21F0F30192B20904CC
:10C8900022F42062090C324342F4807241F001011B
:10C8A00099831A849A8B22F00C02C4E738B50F4D95
:10C8B0000446006807F080FED5F804282046520898
:10C8C0004FF6FF713CF038F820460021FFF764FF77
:10C8D00041F27003064AEA5005F5835120460022D2
:10C8E000BDE8384010313BF0A7BF00BFB82C002096
:10C8F000A1CE01082DE9F0479AB0DDE9226ADDF802
:10C90000909004460D461746984602E020683DF098
:10C91000FDFD20683DF002FE0028F7D101466422AB
:10C9200001A860F0E8FC264B8DF80450CDF85CA01F
:10C930000293002D40D0AB1E012B3FD9042D14BF14
:10C94000002203221F4B0396D3F800398DF80520EF
:10C950001E440123CDE9059404968DF85B3037B170
:10C960004246394607A860F065FC8DF85A80164E9D
:10C9700096F80A9700231893B9F1000F19D196F889
:10C980000907642202FB006001A900F20C7060F04C
:10C9900051FC012386F8099786F80A37236843B1CA
:10C9A00043463A46294620461AB0BDE8F04712F001
:10C9B000DFB81AB0BDE8F0870522C3E70222C1E75D
:10C9C00070550020C01B0020A84E00200C480D4BC5
:10C9D000D0F88C1710B40C4CC0F87C378A1E22316A
:10C9E000B0F8A6371B01A4FB03C3DB08A3F5B063B3
:10C9F00022F8023F9142F3D15DF8044B704700BF2B
:10CA0000A84E0020258A0208CDCCCCCC70B5084CAD
:10CA1000251D2E4614F8010B34F0D4FC28B1037800
:10CA200005F8013BB442F5D170BDFF23F8E700BF24
:10CA3000705600202DE9F0471D4F012607F108052B
:10CA4000B2464FF03C094FF0000817F8010B40F0D8
:10CA50008DFA044690B180F80690C671FB7803F019
:10CA60007F02012A18D013F0800F20460DD185F8DF
:10CA7000048040F06BFD85F805802C600136052EA2
:10CA800005F10805E1D1BDE8F08785F804A040F084
:10CA900063FD85F805A0F0E71B0605D401212046BB
:10CAA0003CF0F6FAFB78DEE740F056FDF6E700BF13
:10CAB000785600202DE9F04FDFF8E491DFF8E4A18B
:10CAC00083B009F10C05012419F8018BB8F1000FAE
:10CAD00000F0C0804FEA1817013F052F08F00F0241
:10CAE00000F2BB800AEB4703B3F8B00040FA02F64D
:10CAF00016F0010600F0C38001239340013B18406B
:10CB000057445CF001FF97F8BC305F4E184406EBC9
:10CB1000C00604236E61F471B371002303E0013396
:10CB2000152B00F09780594903EB43025F00895CA5
:10CB30004145F4D1564B1A4492F89914002900F05B
:10CB4000A08040463CF07AF8804600683CF062F8ED
:10CB500098F805103CF092F80378002B7AD14C4BF2
:10CB60003B44042283F8D94483F8D824002E58D0BB
:10CB7000336898F8080003F13F4202F57E020AEBA1
:10CB80009222012792F8C42002F01F015209032AC1
:10CB900007FA01F169D0042A62D0022A6AD0B6F8F5
:10CBA00004C0BCFA8CF2C2F11F02C2F3CC0103EB49
:10CBB000810102F007020E6A92000F27974026EAD1
:10CBC00007060E620E6A90403043002208624FF062
:10CBD000010B11460BFA01FE3EEA0C001CD118684D
:10CBE0000326964020EA060018601F680220904045
:10CBF000384318609F6827EA06079F609868986026
:10CC0000586820EA0E00586058685860D86820EAD2
:10CC10000600D860D868D8600131102902F10202FC
:10CC2000D8D11C4B1C4AB3F8F817B3F8FA37009167
:10CC3000002001340190B2FBF3F328469BB2414639
:10CC4000E4B233F04FFB0123092C6B7405F1180596
:10CC50007FF43AAF03B0BDE8F08F00266E615CE769
:10CC60000E4F3A6B0A433A6399E70C4A176C394303
:10CC7000116494E7094A576C394351648FE76E6138
:10CC80004BE70B68FFDE00BFBC31002050310020B5
:10CC9000B82C0020A84E002040420F00003802406F
:10CCA000A456002098D3060870B5044684B04FF40B
:10CCB000004036F031F880B300234FF4E131032512
:10CCC00090F904000293CDE900151A464FF4004193
:10CCD00036F083F8124BC3F8C808F0B1012C40F6C7
:10CCE000980208BF4FF496620E480F4DA3F8D4285F
:10CCF0004FF461710D4AC3F8E0080A2683F8CC4866
:10CD0000C3F8D068A3F8D618A3F8D818C3F8DC582D
:10CD1000C3F8E428012004B070BD0020FBE700BF89
:10CD2000A84E00203DCF01087D83010871830108D2
:10CD30002DE9F041214E224F96F8073987F8E0306F
:10CD400006F6041607F1E40500244FF0050816F86E
:10CD5000010B20BB28600134032C05F10405F6D13A
:10CD600097F8E010D7F8E400C94301F0010140F062
:10CD7000F9FB97F8E010D7F8E80081F00201C1F361
:10CD8000400140F0EFFB97F8E010D7F8EC0081F09D
:10CD90000401BDE8F041C1F3800140F0E3BB40F085
:10CDA000E5F8013401212860E3B210B180F8068073
:10CDB000C37128683CF06CF9CEE700BFA84E002094
:10CDC000B03D00202DE9F0412A4C2B4DB4F80C6900
:10CDD000A5F8F06082B0EEB994F8080940F0C6F802
:10CDE00094F80929C5F8F400003A18BF012285F823
:10CDF000F22048B194F80A192B22002914BF1121FE
:10CE00000121C2803CF044F9002002B0BDE8F041AD
:10CE100041F0E6BB94F80889002240462B213BF004
:10CE20007DFF0746404640F0A1F8F8B1F7B12B224C
:10CE3000C5F80C01C280397AFDF7C4FA4FF000083A
:10CE40000E4AB2FBF6F3C3F34F0000909BB2394693
:10CE5000CDF8048005F1F800A4F80E6933F042FA29
:10CE6000D5F8F830C3F8008085F8098102B0BDE834
:10CE7000F08100BFA84E0020B03D002040420F00CE
:10CE80002DE9F84F254C94F81C3984F8103904F634
:10CE90001317002604F513645FFA86FB0BF10108F3
:10CEA0005FFA88F8012117F8010F42460E448A46BE
:10CEB0003BF034FF4FF00009054640B3387804F8E2
:10CEC0000E9C04F80D9C04F80FBC04F810AC44F858
:10CED000045C40F04BF818B180F806A080F8078099
:10CEE000297AFDF76FFA0E4A002128463BF024FD0F
:10CEF0000C4B23600C4B221D21462846C4E9013906
:10CF00003BF09AFC697928684A4633F07FF9082E8D
:10CF100004F11C04C0D1BDE8F88F00BFA84E00206A
:10CF200040420F0045020408F5EB030870B52C4C95
:10CF30002C4B94F8480AC4F8403A00220221C4F865
:10CF4000002AC4F8042AC4F8082AC4F83C2AA4F821
:10CF5000442A3BF0E3FE002841D0234B06680546F7
:10CF600003F1C0015A7C12B15A6896422BD0183393
:10CF70008B42F7D1002394F8480AC4F82C5984F85E
:10CF800020393FF0F3FF08B10223C380297AFDF76F
:10CF900019FA2846154A00213BF0CEFC144A1549DF
:10CFA000C4F830190026111F2846134BC4F8343931
:10CFB000C4F838693BF040FC697928683246BDE81E
:10CFC000704033F023B9304657F036FE328D0B49AE
:10CFD00092B2531CB0FBF3F081F89802CAE770BD1F
:10CFE000A84E002000FFFF004800001040420F0044
:10CFF000DC5700201DEC0308BDED0308880100206C
:10D000002DE9F04FB64DDFF814A385B00B4604466A
:10D01000C02205F134000021019360F06CF99AF808
:10D02000493A002B71D09AF84A3A002B00F08C80D4
:10D03000DFF8CCB29BF88C34012B00F0AE80022BD1
:10D0400000F08F80A74BA84E02931C460FCE0FC452
:10D050000FCE0FC49BF882749BF87E3496E80700CD
:10D06000A24EC5F82C693E1E18BF0126072B84E886
:10D07000070085F84C6900F20981042B00F2138146
:10D08000DFF89C82DFF880A20026019B5FFA86F918
:10D0900009F10107FFB2B3423A464FF0030129DD1F
:10D0A0001AF8014B20463BF039FE034620461C4649
:10D0B00013B33FF05BFFC8F8140018B14FF003033F
:10D0C0008371C7719BF87F349BF87E24002B00F09E
:10D0D000E880E37983F0010349462046013659F0A0
:10D0E000DFFD48B14FF00103082E88F8113008F138
:10D0F0001808CAD1029B06E07D4B7E4AC5F8383934
:10D10000C5F830290023C5F84839D5F8483963B146
:10D110000022019883F82C00012183F82D101A6356
:10D1200083F82E2005B0BDE8F08F734E734C0FCE00
:10D130000FC40FCE0FC496E80700A4F1200384E8C3
:10D140000700C5F84839EDE76D4B019993F8802445
:10D15000003A204618BF0122FBF724FDC5F8480914
:10D16000D3E79BF88234002B3FF46CAF9BF87E34FE
:10D17000082B12D15C4E5D4F0FCE05F614140294AD
:10D180000FC40FCE0FC496E80700012384E8070000
:10D1900085F84C39C5F82C797BE05A4C019BC5F8D1
:10D1A00050390FCCDFF86881A8E80F000FCCA8E851
:10D1B0000F0094E807009BF882349BF87E448AF8BD
:10D1C000844A003B18BF012388E807000026A8F620
:10D1D000CC0285F84C394C4B039208F15C078AF875
:10D1E0004C6A02930BE040F0B1F9039AFB6853617B
:10D1F000082E02F1180307F1200703934DD0D5F84C
:10D200005039B34249DD029B13F8018B029340462B
:10D210003BF0B8FD044640463FF0A8FE9BF87F2453
:10D2200094F8078081460AB188F0010808F00104EB
:10D2300095F84C2901348AF84B4A0AB188F0010864
:10D24000484640F067F900283DD0484641F006FACC
:10D250006101013641F0090179617860C7F80C90ED
:10D2600087F81080F2B2B9F1000F05D04FF0030338
:10D2700089F8063089F8072048463BF009FF18F086
:10D28000010F4846AFD140F067F9AEE7082B7FF4B5
:10D29000F7AE1E4BC5F85439F2E61D48C5F84809EB
:10D2A00033E7E37918E79BF881341A4AC5F8542923
:10D2B000012B05D0022B06BFB7FA87F35B090023C9
:10D2C00085F85839DCE60B4A134BC5F8FC28C5F83D
:10D2D000F838074AC5F8042901238AF84C3ADDE7F3
:10D2E000140000102809001040D60608CD58060882
:10D2F000E16B0408E96B040814D60608F85800200E
:10D30000B82C00206CD606083B310020CDF604086E
:10D31000F4080010FDF60408ED6B0408A84E002088
:10D3200048000010F8B56E4F97F8A00797F8A1577E
:10D330003FF01CFE60B12D23C380202104463BF04A
:10D34000A7FE0A203CF0D4FA204641F07DF918B936
:10D35000D7F8883ADA0000D5F8BD013D092DFBD891
:10D3600097F89F47D4B9402035F0D6FC0028F3D079
:10D3700090F9043097F87517092BC8BF143B3B444C
:10D380000A2993F88C4A00F09D8093F8983A97F810
:10D390009E27002A08BF1C46002CDDD020463FF007
:10D3A000E5FD0546002800F085802D23C38001217E
:10D3B0003BF06EFE0121084640F0DCF82B68AA889D
:10D3C0001A833C203CF0B2FB0021012040F0D2F84F
:10D3D00097F8A137002B4CD0424C00261FE02B6859
:10D3E000AA885A833CF084FA94F8E010D4F8E40058
:10D3F00001F0010140F0B6F894F8E010D4F8EC0028
:10D40000C1F3800140F0AEF82B68AA881A83782017
:10D410003CF06EFA97F8A13701369E4229DA94F86B
:10D42000E010D4F8E400C94301F0010140F09AF89B
:10D4300094F8E010D4F8EC0081F00401C1F380010D
:10D4400040F090F87820002DC9D178203CF050FAB7
:10D4500094F8E010D4F8E40001F0010140F082F803
:10D4600094F8E010D4F8EC00C1F3800140F07AF8B1
:10D47000CDE797F89F37ABB997F8A037002B7FF42B
:10D480006BAF97F8A237012B7FF466AFD7F8883AD5
:10D4900013F080537FF460AF87F8A137BDE8F84000
:10D4A0004AF0A4BF32203CF041FB284600213BF06B
:10D4B000EFFDE1E701213BF0EBFD0121084640F0E3
:10D4C00059F87EE7D7F8B03A5B057FF545AF09F02C
:10D4D000DDFD00287FF440AF002C7FF45FAF3BE719
:10D4E000A84E0020B03D0020094BD3F8B40AD3F871
:10D4F000B82AD3F8BC3A904202DC114602460846EC
:10D50000984204DD9A42B8BF1A46104670477047E9
:10D51000A84E0020124A02F52C6030B419C8984277
:10D52000D2F8CC1AD2F8D02A02DC1D46034628468F
:10D53000914202DC15460A4629468842A8BF0846A1
:10D540009342B8BF1346844202DB2246044610468B
:10D55000984203DD9C422046B8BF184630BC704755
:10D56000A84E00200B6810B414681B1B036054689D
:10D570004B681B1B43608B6892685DF8044B9B1AD9
:10D58000836070472DE9F047041E0D4612DB092C1D
:10D5900026DC824A0B468248A0FB0410C00800EB40
:10D5A0008000A4EB40000021125C1A7059702846DC
:10D5B000BDE8F08764422D23092C01F8013B24D8F3
:10D5C000764A774BA3FB0403DB0803EB8303A4EB4E
:10D5D00043030020D35C48700B702846BDE8F087F9
:10D5E0006F4B632CA3FB04264FEAD60621DC6B4A63
:10D5F0000B466B49A1FB0601C90801EB8101A6EBB3
:10D600004101515C03F8011BC5E7654A632CA2FB8D
:10D6100004364FEAD60637D8604A614BA3FB0603AF
:10D62000DB0803EB8303A6EB4303D35C01F8013B68
:10D63000C7E7A3FB0627B4F57A7F4FEAD7070DD2D9
:10D64000564A0B465649A1FB0701C90801EB810167
:10D65000A7EB4101515C03F8011BCAE7A3FB0728B4
:10D6600042F20F7294424FEAD80836D84B4A0B4622
:10D670004B49A1FB0801C90801EB8101A8EB41015D
:10D68000515C03F8011BDDE7A2FB0637B4F57A7F96
:10D690004FEAD7070CD2414A414BA3FB0703DB08F3
:10D6A00003EB8303A7EB4303D35C01F8013BB4E72F
:10D6B000A2FB073842F20F739C424FEAD80821D8E8
:10D6C000364A374BA3FB0803DB0803EB8303A8EBC5
:10D6D0004303D35C01F8013BDEE7324AA3FB0809B0
:10D6E00094424FEAD90921D82C4A0B462C49A1FB78
:10D6F0000901C90801EB8101A9EB4101515C03F863
:10D70000011BB5E7274BA2FB08099C424FEAD90948
:10D7100021D8224A224BA3FB0903DB0803EB830336
:10D72000A9EB4303D35C01F8013BCAE71E4AA3FB04
:10D73000090394424FEAD30A21D80B461849174AE5
:10D74000A1FB0A01C90801EB8101AAEB4101515C6F
:10D7500003F8011BCAE7144BA2FB09029C424FEAE3
:10D76000D20A13D80E4B0D4AA3FB0A03DB0803EBC6
:10D770008303AAEB4303D35C01F8013BCAE70A2207
:10D78000BAFBF2F04AF024F90346D7E70A22BAFBC3
:10D79000F2F04AF01DF90146E4E700BF00870708F0
:10D7A000CDCCCCCC9F8601003F420F0070B43448F2
:10D7B00090F8D43AA3F13001092957D800F6D424BF
:10D7C000224600F6E32012F8015FA5F13001092995
:10D7D00004D88242F7D1002070BC7047141B022C81
:10D7E0004ADD2848002101E010F8013B01EB8101EE
:10D7F00003EB4103161A303B022E044603F0FF01EF
:10D80000F2DC214B03FB01F1A2424FF000030DD9E2
:10D8100003EB830314F8016B5B00303B3344A242FB
:10D8200003F0FF03F4D1194800FB03F32E2D06D0BB
:10D830001748A0FB032301EB930070BC7047013233
:10D8400004200024157804EB8404303D6400092D85
:10D8500000F1FF30A4B202D82C44A4B2013210F07F
:10D86000FF00EFD1642202FB0433E1E700211D46F3
:10D8700000F6D4220B46D9E7064C0021C4E700BFCE
:10D88000A84E00207D5900208096980040420F004D
:10D89000ABAAAAAA7C59002038B504460D460A4610
:10D8A0000068FF215FF027FD21682944216038BD11
:10D8B00083B50C461646054633F0F2FD204633F09C
:10D8C000EFFD0021204B0846002E08BF1E463FF00A
:10D8D00051FE002101203FF04DFE28463CF01EFE87
:10D8E000B0B1012100203FF045FE28463CF00EFE7D
:10D8F000074620463CF00EFE0028FAD03946204666
:10D900003CF010FE3846B047002108463FF032FE9A
:10D9100020463CF003FE0028DFD0012100203FF02C
:10D9200029FE20463CF0F2FD0146284601913CF0DC
:10D93000F1FD01990028F8D028463CF0F3FD0021C4
:10D9400008463FF017FEC8E749F40308F0B5002386
:10D950000B604B608B60CB600B610268DFF88CC0A2
:10D9600089B004ADC2F385572E4647FA03F0C007CD
:10D97000344604D513F80C0004F8010B2646013395
:10D98000062BF2D11748C2F303240444002394F871
:10D99000084333708DF8184000F5447CC2F3053716
:10D9A0000DF1190647FA03F0C007344604D513F801
:10D9B0000C0004F8010B26460133062BF2D100239C
:10D9C0003370C2F3834406ABCDE90134084602F05C
:10D9D0000F0305490095C2F303124EF0F9FC09B09C
:10D9E000F0BD00BF98D306082887070898D6060818
:10D9F00070B5094CD4F8E42A054662B10026D4F883
:10DA0000E40A2D21013641F011FCAE42F7DBBDE8FE
:10DA1000704042F0D1BE70BDA84E00202DE9F04FFD
:10DA20005FFA81F8002185B00746084616463FF0A8
:10DA3000A1FD002101203FF09DFD3FF075FA022E6F
:10DA40000AD0042E44F6C01918BF4FF49649B8F115
:10DA5000070F07D900200CE0B8F1FF0F4FF416496B
:10DA6000F5D10326CE4D95F8E83A2BB90020C5F83C
:10DA7000EC0A05B0BDE8F08F032ECA4C0DD0A044CF
:10DA8000002298F8830403213BF048F90028EDD0E8
:10DA9000C4F84C08C3799A07E8D441F2670395F8B3
:10DAA000E80AE654002203213BF038F9C4F8500C90
:10DAB0000028DBD04FF48061BB4BC4F80838C4F8B1
:10DAC00014180323C4F8181841F25801A4F80C38AC
:10DAD0000023635441F254014FF0010AB34A24F881
:10DAE00001A041F2640102F14800635241F2660173
:10DAF000C4F81C08032E02F24C406354C4F810987A
:10DB0000C4F83438C4F82838C4F82438C4F82008D5
:10DB1000C4F83038C4F82C38C2F8583890460ED0C3
:10DB2000D4F84CB89BF804003FF020FAC4F8480839
:10DB3000584612F079F85146404612F089F83220E2
:10DB40003BF0F4FF002E63D1D4F8509CD9F80000CC
:10DB500006F032FD4846964A22213AF0EDFE41F2A7
:10DB60006C03944AE25008F66401324648463AF0A3
:10DB700063FED4F84C98D9F8000006F01DFD8C4ADD
:10DB80004FF6FF7148463AF0D7FE31464846FEF759
:10DB900003FE41F27003884AE25008F668013246FB
:10DBA00048463AF049FEC5F8EC8A4FF0060A022EC4
:10DBB00012D0D5F8EC0A3CF0B1FC68B1012100208C
:10DBC0003FF0D8FCD5F8EC0A3CF0A8FC0146002850
:10DBD00040F09E803FF0CEFC38463CF09FFC88B180
:10DBE000012108463FF0C6FC4FF0050B4FF000083E
:10DBF00038463CF093FC0146002840F0928001201A
:10DC00003FF0B8FC042ED4D005203BF08FFFCEE7C8
:10DC1000012E09D1D4F8500C4946FBF7CBF9D4F8C2
:10DC20004C08FEF743FEBEE7022E09D1D4F84C089B
:10DC300011F0E9FFD4F8500C4946FBF7BBF9B2E705
:10DC4000032E5DD14FF0000A41F2680351465B4854
:10DC500004F803A040225FF04EFBDFF864B18DF8BA
:10DC60000FA0DFF860A19DF80F30072B09D94F48AE
:10DC7000012111F0EDFFD4F8500C4946FBF79AF959
:10DC800091E79DF80F3003EB43030BEBC30393F8CD
:10DC9000453073B39DF80F3003EB43030BEBC30325
:10DCA0009B6C33B39DF80F30234493F8830400B387
:10DCB000002203213BF032F80190D0B111F0A3FF14
:10DCC0009DF80F309AF80010019A03EB43030BEB19
:10DCD000C30305EBC1009B6CC0F8F03AD379DB07B6
:10DCE00048BF012301F1010148BF80F8F43A8AF8E6
:10DCF00000109DF80F300133DBB28DF80F30B2E722
:10DD0000042E7FF450AFD4F84C0811F07CFF81E76B
:10DD1000D5F8EC0A3CF0FAFB014638463CF002FC30
:10DD200050E738463CF0F2FB95F83E3B01468BB994
:10DD3000242803D14FF0010385F83E3B012E04D186
:10DD4000384601913CF0EEFB0199D5F8EC0A3CF025
:10DD5000E9FB4DE7012B06D14D280CBF0223002320
:10DD600085F83E3BEAE7022B06D13C280CBF032393
:10DD7000002385F83E3BE1E7032B25D10A2802D991
:10DD800085F83E8BDAE7042385F8310B85F8308B74
:10DD900085F8338B85F8320B85F83E3BCEE700BF24
:10DDA000A84E0020B82C0020B0D60608C0340020B1
:10DDB00040420F00DDFC0108BDCD0108985900204C
:10DDC00014000010203D0020042B09D195F8323BAF
:10DDD00085F83F0B434085F8323B85F83EBBADE705
:10DDE000052BABD195F8303B95F8319B95F8320B6C
:10DDF0004B4509D25A1C2B44484085F8320B85F814
:10DE0000302B83F8341B99E78842B9D195F83F3B12
:10DE100085F83EABF42B91D1B9F1000F8ED12421BE
:10DE2000384685F83E9B3CF07DFB4D2138463CF062
:10DE300079FB3E2138463CF075FB494638463CF0BC
:10DE400071FBF42138463CF06DFBF42138463CF080
:10DE500069FB032E1BD0D4F84C08437901689D0858
:10DE60000223AB40DB439BB20B828D892B408B811D
:10DE70000079202111F0B6FED4F84C084A464946F4
:10DE80003AF0DAFCD4F84C38186806F095FB00221A
:10DE9000D4F8500C11463AF0CFFCD4F8503C186836
:10DEA00006F08AFB0120E4E5114A013002EBC000D4
:10DEB000F0B4D0F84CC30F4E0023336033613362AB
:10DEC00033633364336533663367BCF1000F0DD0C1
:10DED00090F8487357B13F0100240CEB04030FCBBB
:10DEE00035191034A74285E80F00F6D1F0BC704711
:10DEF00098D30608E859002038B50F4C94F8C71B92
:10DF000001F03F018B1C024601F10A0584F8C53B74
:10DF100084F8C25B04F53C6084F8C32B08311DF023
:10DF200087FB254485F8BE0B94F8C23B1C44000ACD
:10DF300084F8BF0B38BD00BFA84E002070B51D4C43
:10DF40000968D4F8EC5B1C4ED4F8E84BD6EDA77A00
:10DF5000DFED1A6A491B00EE901A0168F8EEE00A3C
:10DF6000091B60EEA70A00EE101A20EEA07AB8EEA8
:10DF7000C00A1C46A0EE007AB1EE400AF1EEC77A64
:10DF800067EEA67AFCEEE77AC2ED007A4EF012FB5D
:10DF90009FED0B7ADFED0B7AE0EE077AFDEEE77A84
:10DFA00017EE902A002ABCBF02F50C42A032226074
:10DFB00070BD00BFA84E0020880100202C7D8E3F40
:10DFC000A00CB34500A00C4638B50B4C002501222F
:10DFD0008021204634F08CFE30B194F9040034F0F6
:10DFE000BBFE08B1006838BD0135092D04F10C04F1
:10DFF000EDD10020F7E700BFA85A002038B5041F74
:10E0000000F1080554F8043FD81780EA430017F0E0
:10E010009DF9A542F6D138BD2DE9F041D24CDFED96
:10E02000D37AD4F85C3A94F8F50A07EE103A2DED5D
:10E03000028BB8EE478A28EE278A002840F0CA8073
:10E04000D4F8002B94F8F41A94F8113B002A19DD47
:10E0500007EE902ADFEDC66AF8EEE77AC3F16403B3
:10E0600086EEA77A00EE103AB8EEC00A20EE070A54
:10E0700029B920EE000ADFEDBF7A20EE270A5CF016
:10E08000D5FD80B2B4F8F63AA4F8F60A834200F05F
:10E09000A18094F8607AB84EDFEDB88A4FF000089E
:10E0A000002594F8143B2B41DB0714D594F8F43A7F
:10E0B000002B7FD1B4F8F63A07EE103A002F00F0AB
:10E0C000FB80B8EE477AC8EE877A77EE887A88EEDA
:10E0D000277A86ED027A0135042D06F12406E0D177
:10E0E00094F8F95AB4F8FC6A002D40F0E880002F4B
:10E0F0005CD194F8103B84F81C5B84F8183B002E2C
:10E1000054D0002D52D007EE906A0123B8EE678AF2
:10E11000DFED9A7A84F8203B9D42C7EE888A28D0AA
:10E12000022D43D1D4F85C1A9548B0EE480A45F068
:10E1300027FB94F81C3B012B00F01181022B35D1F9
:10E14000D4F85C1A8F48B0EE480A45F019FB94F8F1
:10E150001C3B012B00F0FE80022B27D1B0EE480AB9
:10E16000BDEC028BD4F85C1A8748BDE8F04145F05D
:10E1700007BB864AD2ED007A78EEA76A134687EE8F
:10E18000A67A002143F8041F83ED017A78EEA76A8E
:10E19000002187EEA67A996083ED037A77EEA88A4C
:10E1A000002287EEA87A1A6183ED057ABDEC028B16
:10E1B000BDE8F081B4F8F63AD4F85C1A00EE103AF3
:10E1C000301DB8EE400A002F70D145F0D9FA94F80E
:10E1D000607A80E794F8607A002F3FF45CAF94F89F
:10E1E000F95AB4F8FC6A002DE0D0694A94F8FA3A7A
:10E1F000D2F8702C92F883201343D7D1D4F8002B97
:10E2000094F8113B002A65DD07EE902ADFED586A8D
:10E21000F8EEE77AC3F1640386EEA77A012D00EEEB
:10E22000103AB8EEC00A27EE000A60D05CF0FEFC9F
:10E2300080B2A4F8FC0A002F79D08642B6D000281C
:10E24000B4D094F81C3B002BB0D007EE900AB8EE87
:10E25000678ADFED4A7A012BC7EE888A4ED0022BFF
:10E26000A4D1D4F85C1A4648B0EE480A45F072F9D9
:10E2700094F81C3B012B6AD0022B97D1D4F85C1A7E
:10E280004048B0EE480A45F065F994F81C3B012B74
:10E2900058D0022B8AD1B0EE480ABDEC028BD4F8DC
:10E2A0005C1A3948BDE8F04145F054B9301D45F0DD
:10E2B00051F994F8607A0EE7C6F8048001E7344A11
:10E2C00094F8FA3AD2F8702C92F8832013437FF432
:10E2D0000EAF93E70023A4F8FC3A002F7FF466AF5B
:10E2E00094F8103B84F81C5B84F8183B5EE720EE42
:10E2F000000ADFED207A20EE270A97E7234A13462B
:10E30000F3EC017A78EEA76A87EEA67A83ED017ABC
:10E31000D2ED007A78EEA76A87EEA67A83ED037ACB
:10E3200077EEA88A87EEA87A83ED057A3EE794F81F
:10E33000103B84F81C5B84F8183B00283FF436AF90
:10E340000646E0E6114AD2ED007A131DE8E70F4ACF
:10E35000131DDDE70D4AD2ED007A131D1EE70B4AAF
:10E36000D2ED007A131D11E714000010BD37863579
:10E3700000409C45CDCC4C3C740A001083F9223EF1
:10E38000380B00105C0B0010800B0010A40B001069
:10E39000A84E0020F8B5214C1D270E46054684F8EE
:10E3A000747C1DF06BFA00201DF00AFA08201DF0A5
:10E3B00007FA0E201DF004FA38461DF001FA042079
:10E3C0001DF0FEF904201DF0FBF900201DF0F8F906
:10E3D00030201DF0F5F900201DF0F2F930461DF057
:10E3E000EFF900201DF0ECF91DF034FA04F6754049
:10E3F0001DF03AF9234670B194F8752C62B994F87F
:10E40000762C302A00D03AB993F8772C22B993F8B9
:10E41000783C2B700120F8BD0120FCE7A84E0020BD
:10E42000104B034410B5044693F8200410F022FF6B
:10E430000D4800EB44040A23B4F9881CB1F5FA6FC7
:10E44000A8BF4FF4FA61B1F57A7FB8BF4FF47A7183
:10E45000A1F57A71BDE81040B1FBF3F10920C9B212
:10E4600010F036BF98D30608A84E00201D4991F839
:10E47000D42AA2B3F0B400260546334630463746C8
:10E480001BB991F8D44A2D2C23D02E2A19D0CA18A2
:10E4900000EB800092F8D44AA4F13002092A4FEA36
:10E4A00040009CBFA0F13002A0180E2B14D80133FD
:10E4B000CA1892F8D42A002AE2D106B14042F0BC30
:10E4C00070470133002DF8D0CA182A4482F8D47A54
:10E4D000DDE701231E46EBE70020F0BC704700207B
:10E4E000704700BFA84E00201FB503AC8DF80C305C
:10E4F000009400238DF80D300FF0F4F904B010BD36
:10E50000F8B50546262026F011F8134C0146F8B957
:10E51000D4F8AC0C90F838301E3B012B01D93CF0FC
:10E5200001F80E4F0026AE420ADBB4F8D03C0133AE
:10E53000A4F8D03C0A4BD3F80039C4F8E03CF8BD4D
:10E5400017F8011BD4F8AC0C3BF0ECFF0136EAE7FE
:10E55000002384F8DE3CEDE7A84E0020585B002045
:10E56000C01B002010B58021044604F08DFE20461B
:10E57000002104F089FE2046BDE8104005F0C4B932
:10E580002DE9F041B14C94F8F73CC4F8E40C82B0AA
:10E5900088465A2B00F2B980DFE813F0CC00B700B0
:10E5A000B700DC00B700B700B700B700B700B7008E
:10E5B000B700B700B700B700B700B700B700B700A3
:10E5C0000F01B700B700B700B700B700B700B7003A
:10E5D00033017400B700B7007400B700B700B7008C
:10E5E000B700B801B7006201B700B7007C00B70000
:10E5F0000902B700B700B700B7005B00B700B7006B
:10E60000B700B700B700B700B700B700B700B70052
:10E61000B700B700B700B700B700B700B700B70042
:10E62000B700B700B700B700B700B700B700B70032
:10E63000B700B700B700B700B700B700B700B70022
:10E64000B700B700B700B700B700B700B700B70012
:10E65000E40194F8F83C9B0700F16982B4F8FE3CB1
:10E66000D4F8F92CD4F8381D5BBA9BB212BAD01882
:10E670008842C4F8443DC4F8402D03D904F0C4FDD9
:10E68000002854DB0020A4F8300D0546284602B0CF
:10E69000BDE8F08194F83C3D002B40F0FF8094F9F8
:10E6A000F43C002B31DAD4F82C3D08469B6898479F
:10E6B000002840F01E82B4F8FE0CD4F8F92CD4F8EF
:10E6C000383D40BA80B212BA15189D42C4F8440DC4
:10E6D000C4F8402D07D904F097FD002827DBD4F8B3
:10E6E000402DD4F8440DD4F8343DD4F8F06C03FB3D
:10E6F00000F003FB02F20225B042C4F8402DC4F83A
:10E70000440D84F83C5D00F0CF8094F8083D5A1C1D
:10E71000D2B204EBC30305204FF40051042A84F85D
:10E72000082D83F80C0DC3F8101D00F0A0814FF0E8
:10E73000FF35ABE7D4F8F03C002BE6D1D4F82C3D04
:10E7400008469B6898470546002840F0D281A4F807
:10E75000300D9BE73E4B002203F1120103F8012F1D
:10E760008B42FBD13B4994F8323D94F8080D70255B
:10E770000D7098424FF00C05CD7110D004EBC30022
:10E78000013390F80C5D8D70B0F8100DDBB2042BE6
:10E7900040BA888114BF84F8323D84F8322D94F851
:10E7A000FB3C12229342A4F8302D98BFA4F8303DD0
:10E7B0000025284602B0BDE8F08194F8F83CDA075D
:10E7C00000F13E81D4F82C3D94F8FB0CDA6901EBA2
:10E7D000C10102EB81010A79531D834228BF034620
:10E7E000A4F8303D002BE3D0013B1A489BB2013323
:10E7F0001944034411F8012D03F8012D8342F9D186
:10E80000D6E7154E154F35460823073EC5F10700DC
:10E81000A4F8303D002202E092F840241D462B4629
:10E82000B54203F8012900EB030217FA82F2F3D193
:10E83000D4F82C3D4046DB6898470028B8D0AB7828
:10E8400063F07F03AB70002520E700BFA84E0020D7
:10E85000DF7E0020E07E0020E77E002098D30608BF
:10E86000D4F82C3DC74A5B680846111D98470546F9
:10E87000002840F03E81D4F8383DC34AD4F8341D16
:10E88000013B180E1070180C09BAD37050701B0A97
:10E89000082093705160A4F8300DF7E6D4F8446D69
:10E8A000D4F8402DD4F8343DD4F82C5DB2FBF3F20B
:10E8B0004FF48057BE4228BF3E462D69B249A4F8A6
:10E8C000307D4046B6FBF3F39BB2A8470028C0F268
:10E8D000BC803346AC4AD4F8E40C812104F008FD36
:10E8E000D4F8402DD4F8440DD4F8503D3244851B63
:10E8F0009E1BC4F8402DC4F8445DC4F8506D002D33
:10E900007FF456AF032384F83C3DBFE69E4E0027BC
:10E91000334606F10C0203F8017B9A42FBD1D4F88E
:10E920002C3D40465B686A4601A998470546002889
:10E9300040F0E980019BBDF80020013B190E52BA5E
:10E94000F3713171190C1B0A71710820B371022126
:10E9500072810C23BDF80220F07031727272A4F83B
:10E96000303D93E6894E8A4F30460823073EC0F17A
:10E970000705A4F8303D002202E092F8482418462A
:10E980000346864203F8012905EB030217FA82F2D7
:10E99000F3D1D4F82C3D4046DB68984700283FF47B
:10E9A00007AFF37863F07F03F37000256EE694F809
:10E9B0003C3D002B61D194F9F43C002BFFF6A5AE51
:10E9C000D4F82C3D08469B689847002840F0918079
:10E9D000D4F82C3D4046DB6898470546002840F0B7
:10E9E000BA80B4F8FE3CD4F8F92CD4F8381D5BBAE0
:10E9F0009BB212BAD0188842C4F8443DC4F8402DE6
:10EA000000F29F80D4F8341DD4F8F00C03FB01F31E
:10EA100002FB01F28342C4F8402DC4F8443D7FF468
:10EA200074AEB3F5805F28BF4FF480530121D4F852
:10EA3000E40C554A84F83C1D9BB204F083FD25E6A6
:10EA400007235449A4F8303DCEE694F8083D5A1CFB
:10EA5000D2B204EBC30304204FF48851824284F8FD
:10EA6000082D83F80C0DC3F8101D7FF460AE002351
:10EA700084F8083D4FF0FF3508E6D4F8446DD4F82B
:10EA80002C0DD4F8343DD4F8402D4569B2FBF3F297
:10EA9000B6F5805F28BF4FF480560846B6FBF3F307
:10EAA00039499BB2A847002862DBD4F8402DD4F83E
:10EAB000445DD4F8503D3244AD1B9B1BC4F8402D3F
:10EAC000C4F8445DC4F8503D2DB9D4F8E40C29468F
:10EAD00004F08CFDDAE5B5F5805F28BF4FF4805572
:10EAE000ABB2D4F8E40C284A012104F02BFD002538
:10EAF000CCE594F8083D5A1CD2B204EBC3030220C3
:10EB00004FF468510AE694F8083D04EBC302013360
:10EB1000DBB202204FF46851042B82F80C0DC2F8CE
:10EB2000101D22D084F8083D4FF0FF35AEE594F873
:10EB3000083D5A1CD2B204EBC30305204FF4105118
:10EB4000ECE504F061FB0028FFF6F1ADD4F8402DB0
:10EB5000D4F8443D56E794F8083D5A1CD2B204EB71
:10EB6000C30302204FF41C51D8E584F8087DDEE58C
:10EB700094F8083D5A1CD2B204EBC30304204FF4AE
:10EB800040716BE7DC5B0020E07E0020E77E002028
:10EB900098D30608D0D7060810B51C203EF0E6F939
:10EBA000112104463AF074FA20463EF0CFFCC8200A
:10EBB0003AF0BCFF2046BDE810403EF0CDBC00BF9F
:10EBC00008B500203EF0D2F9054BC3F8580D08B146
:10EBD0002A23C380BDE8084040213AF059BA00BF5B
:10EBE000A84E00202DE9F04FB34CD4F8A83E5A6946
:10EBF000D2078BB002D50BB0BDE8F08F5A699B6984
:10EC000012EA030AF7D0CAF307431AF4002F00935D
:10EC100040F00281009B5D0743D41AF0020F5FFAB7
:10EC20008AF503D0D4F8A83E02225A61BAF1000F47
:10EC3000C0F211821AF4006FCAF3072740F08481F2
:10EC40002E0708D59D4B9E48D3F8AC329847D4F890
:10EC5000A83E08225A61ED0600F1E981F80600F1AC
:10EC6000A981B90600F12E81009BDA0609D5934BE4
:10EC70009348D3F8BC329847D4F8A83E4FF480129A
:10EC80005A61009B9B06B6D58C4B8D48D3F8C03299
:10EC90009847D4F8A83E4FF400125A610BB0BDE873
:10ECA000F08FD4F8AC2E9369D26913401FFA83FB1E
:10ECB000BBF1000FB1D0DFF80882CDF80CA04546BB
:10ECC0004FF0000909E05FEA5B0B09F1010908F167
:10ECD000040805F1280500F0DA811BF0010FF2D0DD
:10ECE000D4F8AC1E5FFA89F708694A6B04EB870316
:10ECF000FA40D3F8B43ED2019B68D2B202431A4024
:10ED0000D007D3B216D54B6BD8F81820012000FAE3
:10ED100009F023EA00034B63684B6948D3F8A43237
:10ED2000012191603946984794F89F6E012E00F0BA
:10ED3000038201231A0703D5D8F81820082393600B
:10ED4000DE0603D5D8F8182010239360580603D5A3
:10ED5000D8F8182040239360990703D5D8F81820D5
:10ED6000022393601A06AED5D5E94C60D5F824315C
:10ED7000D8F818C0311A8B42DCF8182028BF0B468F
:10ED8000033392B2B2EB930F9DD9D4F8AC2E323745
:10ED900004EB8703CDE9019890469946B04238D2FA
:10EDA000BEB3D5F8241194F89F3ED5F82821371A20
:10EDB000B94228BF394601F1030E4FEA9E0E83B9CE
:10EDC0008FB20337BF10D9F8A4AE0AD0013352F87E
:10EDD000040BCAF800009F42F8D1D5E94C60D5F881
:10EDE0002821DCF8183008440A44B042C5F828212C
:10EDF000C5F834010AD195F81C11D8F83420012740
:10EE000007FA01F122EA0102C8F834209BB29E45BC
:10EE1000C4D3DDE9019856E7D4F8AC3E9D69DB69BF
:10EE20001D402D0C3FF4F6AE04F69C66DFF88CB066
:10EE3000B046B146002708E06D0807F1010706F16A
:10EE4000040608F128083FF4E5AEEB07F4D5F9B263
:10EE500004EB8102D4F8AC3ED2F8F02E92685B69E4
:10EE60001A40D007D3B218D594F89F0E726D0123C3
:10EE70009842936007D11269D8F87C33C2F312022A
:10EE80009B1AC8F88C33DBF8A0324846984794F8B0
:10EE90009F3E012B00F05E8101239A0702D5726D1F
:10EEA000022393601B07C7D5DBF8A8324846984772
:10EEB000736D08229A60BFE7B03D002088010020F2
:10EEC0004C4C0020D4F8AC3ED4F8B41E9A680868C4
:10EED000C2F34102022A08BF03224FF0000514BF0B
:10EEE00065F30A0062F30A0008605A6842F480720F
:10EEF0005A6006A805F00EFCD4F8A82ED4F8AC0E83
:10EF0000D368BE49079D6FF38D23D3608068C0F33B
:10EF10004100014491F85014032900F0D380B8490E
:10EF2000B8480126294484F89E6E81424FF040067D
:10EF3000A4F8A06E00F21C810E2161F38D234FF422
:10EF40000051D36051618FE6AF4B94F8AE2FD3F8E8
:10EF5000B432AE4800218DF817108DF8172098476D
:10EF6000D4F8AC1ED4F8A82E94F8A63E88684FF4C6
:10EF700000615161002B3FF463AEC3077FF560AEC3
:10EF800094F8B13F012B7FF45BAE9DF81730032B53
:10EF90007FF456AED4F8A83F9D491A6842F00102AA
:10EFA0001A601A6842F003021A600B6943F0060304
:10EFB0000B6145E6D4F8AC2E944853684FF0000836
:10EFC00023F001034146536004F0CAFF94F89D6E9C
:10EFD000414656B18F4BFF2203EB860653F8045F80
:10EFE000D86BAA609E428260F8D1D4F8AC3E8748C4
:10EFF0004FF0FF329A614FF00112DA610B2262F397
:10F00000070162F30708C3F8148019611A686FF3E7
:10F010000A121A6004F078FCD4F8A82E7A4B7B48C8
:10F02000D3F8B0324FF480515161984719E6D4F8C3
:10F03000A83E9A6922F010029A611A6AC2F343400C
:10F04000022802F00F0148D0062823D09A6942F026
:10F0500010029A6102E694F8A63E3BB1D4F8A82FBC
:10F06000136823F0030161F307031360D4F8AC2E97
:10F0700065495368D1F8B812644823F0010353601E
:10F080008847D4F8A83E4FF000425A61D2E5DDF837
:10F090000CA0C2E5D4F86C6F01EB810104EBC10157
:10F0A00041F2282541F2684C306844F80C00485978
:10F0B000C2F30A1241F26C4C0244306844F80C006E
:10F0C0004A51C3E700214FF4007084F89E1E0921C5
:10F0D000A4F8A00E61F38D2331E747F6F0701042DB
:10F0E000B4D001EB8100C2F30A1204EBC00041F27C
:10F0F0001C2502F1030C5FEAAC0C4559D4F86CEF07
:10F100004FEA810818BF002006D00130DEF8006009
:10F1100045F8046B8445F8D1414404EBC10141F248
:10F120001C2C41F2282651F80C50885915440244F1
:10F1300041F80C508A5189E7B9F1000F7FF4F9AD1D
:10F1400094F8AD3F042B7FF4F4AD304804F0DCFBC1
:10F150003346EFE5002F7FF49FAE94F8AD2F052ADC
:10F160007FF49AAE4846019304F0CEFB019B94E6EF
:10F170002948A5F57401A1F51051814203D80D214C
:10F1800061F38D23DBE6254925482944814203D2DA
:10F190000C2161F38D23D2E62248A5F18C71A1F5F3
:10F1A0004341814203D80B2161F38D23C7E61E49F9
:10F1B0001E482944814203D20A2161F38D23BEE611
:10F1C0001B491C482944814203D2092161F38D2344
:10F1D000B5E61948A5F1B771A1F55851814203D29E
:10F1E000082161F38D23AAE6144915482944814278
:10F1F00028D2072161F38D23A1E600BF98D306082A
:10F20000401E1BFF3F420F00880100204C4C002095
:10F2100000ED00E0604C0020DFC810002013FBFE72
:10F2200020D61300FF69180000D3CEFE40771B00E4
:10F23000C05BB3FEC091210040AC2700C01D6AFE38
:10F2400040E13300044905482944814234BF062186
:10F25000052161F38D2372E6803C36FEE09C41007F
:10F26000704700BF704700BF704700BF704700BFC6
:10F270002DE9F0414FF0FF35324A33482C46002348
:10F2800004E001330B2B02F1100215D0917A04290E
:10F29000F7D103F5B17100EB0111C979CF07F0D4B3
:10F2A000661C116801D0A942EBD21C4601330B2B1E
:10F2B0000D4602F11002E9D1631C02D10120BDE824
:10F2C000F081214D04F5B17705EB07139988F1B969
:10F2D000DFF880802601AB19D8F8A0231B491669F6
:10F2E0001B4A41F2186001EB442118580023B04733
:10F2F000D0B1022808D141F2CC6205EB0717AB5818
:10F30000013B0121AB50B9710020BDE8F081DFF86D
:10F31000448005EB0413D8F8A02341F21860D268AA
:10F32000185826019047D6E741F2CC6205EB071743
:10F33000AB580321B97141F2D061013B0124AB50BC
:10F340006C54BCE7FCA40020E08E0020F88E002066
:10F3500071F30008A84E0020044B41F2E472995C5E
:10F3600009B90121995401225A707047E08E00209A
:10F3700038B5174D174B41F2D0640020285504E0F2
:10F3800001300B2803F1100314D053F80E4C8C42BB
:10F39000F6D11C78032CF3D16AB10F4B03EB402359
:10F3A0009A4201D0FFF7D8FF00F5B17005EB0010CD
:10F3B0000123837138BD41F2CC6100F5B1736A5805
:10F3C00005EB03130420013298716A5038BD00BF69
:10F3D000E08E002006A50020F88E002038B5134BE3
:10F3E00000209C7B14B11D688D4205D001300B2894
:10F3F00003F11003F5D138BD72B10D4B03EB40237F
:10F400009A4210D0FFF7A8FF0A4B00F5B17003EB4A
:10F4100000100123837138BD064B00F5B17003EB7A
:10F420000010827138BD022CECD1EDE7F8A4002069
:10F43000F88E0020E08E00202DE9F84F12F0020E29
:10F440009B4606D028B9FFF787FF02252846BDE86E
:10F45000F88F804C41F638056559002D5BD14FF08F
:10F46000FF367D4FB146B046B24600253B68984214
:10F4700000F0B68097F80EC0BCF1000F5BD0BCF175
:10F48000010F15D105F5B17C04EB0C1C9CF807C0ED
:10F490001CF0010F0CD11CF07E0F09D15FEADC13C8
:10F4A00040F0A880D7F808C0D44501D2E246A9466A
:10F4B00001350B2D07F11007D8D1751C04D1B8F117
:10F4C000FF3F00F09F80464641F2C86806F5B177DD
:10F4D00054F80850013544F8085004EB061C41F27A
:10F4E0001C694FEA07184CF8095044F8085041F2DB
:10F4F000186904EB07154FF000084CF80900C5F82F
:10F50000048004EB0715AD79042D9CD8DFE805F0E5
:10F510001A330F334D0004F5C25741F63C063F68DD
:10F52000A65907FB0565A84299D3FFF715FF0025EB
:10F530002846BDE8F88F2E4601350B2D07F1100740
:10F5400094D1BAE712F0010C70D104EB0710D5107A
:10F5500090F80780BBF1030F65F3C71880F80780A8
:10F5600062D94FF6FF7083455B4628BF03469BB2C6
:10F5700004EB07108380BEF1000F16D004EB0613D6
:10F5800003F5B0531833987B04280ED041F2C865B8
:10F590004FF0040C60590130605141F2CC65586065
:10F5A00083F80EC0635901336351500705D504EB4E
:10F5B0000710C37943F00103C371D30608D504EBE8
:10F5C0000714E379C3F34502013262F34603E371A2
:10F5D000224B012503EB46260E602846BDE8F88F36
:10F5E00005F5B17704EB07164FEA071CB67986B923
:10F5F0002E4669E7A84601350B2D07F110077FF469
:10F6000035AF5AE7B9F1FF3F18BF4E467FF45CAF04
:10F610008DE741F2C8682E4654F80850013544F889
:10F62000085044F80C506CE76346A1E70C4B0B49BB
:10F63000D3F8A0330B4AD3F8088001EB462100230E
:10F64000C04700283FF473AF04EB07140223A371F3
:10F65000FCE600BFE08E0020F8A40020F88E002019
:10F66000A84E0020DDF30008F0B5124D2B7841F6CE
:10F670003002022B0BBF070AC0F3D417C4B200F04C
:10F680007F04A85883B00E4600230122384401A904
:10F69000FFF7D2FE01280AD12B78022B019B16BF5F
:10F6A00053F8243033F8143023F07043336003B040
:10F6B000F0BD00BFE08E002010B5144602070B46D7
:10F6C00010D50B4941F2C472581C8B58834204D3A5
:10F6D00005D100232360012010BDFFF73DFE20600F
:10F6E000012010BD21461846BDE81040BCE700BF10
:10F6F000E08E00202DE9F0414268C2F308030B447C
:10F70000B3F5007F82B004460D4657D390F91A3006
:10F71000591C0AD0304A03F5B17302EB0313FF21E1
:10F72000DA796FF30002DA71817694F91B305A1C92
:10F730000FD0294A03F5B17302EB0313FF20DA79E6
:10F74000C2F34501013921EAE17161F34602DA7140
:10F75000E0762378022B37D01F4A02F5C2531B688C
:10F76000B5EB432F4FEA432824DC41F64803676892
:10F77000D6583E407342AB421CDCAB19434511D313
:10F780002169207E01AAFFF797FF012812D167683F
:10F79000236963614744019B2361A5EB0801BF1BFB
:10F7A00067608D192046F8F717FE20B93D44656063
:10F7B000012000E0002002B0BDE8F0811544456062
:10F7C000012002B0BDE8F081616801202944616038
:10F7D00002B0BDE8F08100BFE08E002070B5154694
:10F7E00004460E46FFF786FF50B994F8280028B962
:10F7F000022384F82830C4E90B5670BD022070BD86
:10F800001DB12046A847012070BD012070BD00BF7A
:10F8100010B4D0E9011390F91A208B4238BF0B467F
:10F82000511C83600AD0144B02F5B17203EB021233
:10F83000FF21D3796FF30003D371817690F91B30E8
:10F840005A1C0FD00C4A03F5B17302EB0313FF24CB
:10F85000DA79C2F34501013921EAE17161F3460227
:10F86000DA71C4760022436A5DF8044B426142605B
:10F8700011460361B2E700BFE08E002038B5442294
:10F88000002111485DF037FD104B41F602011A7856
:10F890004FF6FF745C52022A41F2E87118BF03224E
:10F8A00003F5C05041F64C055A5441F60C0441F69C
:10F8B000010203215D5900F8181910211D519954B6
:10F8C000FFF7A6FF012038BDC8A60020E08E00206B
:10F8D0002DE9F041B1F904300F2B82B00C461646E9
:10F8E000054632D02846F8F79BFD95F91B80B8F104
:10F8F000FF3F074633D02D4B41F2186203EB08114E
:10F900008A58904211D1183303EB4823A188013162
:10F9100009B203EB4113A18028463360F8F780FD5C
:10F920002060012002B0BDE8F081FFF715FD2846F8
:10F93000F8F752FD28B100230120336002B0BDE882
:10F94000F081002002B0BDE8F0814FF40071FFF7B4
:10F95000D1FE0028F5D04FF6FF73A380C2E72846FA
:10F96000F8F73AFD0028E2D10FB9FFF7F5FC384669
:10F970000023112201A9FFF75FFD0128D7D1019BC8
:10F980000B4A9A1A48BF02F2FF12B2F5B05F4FEA73
:10F99000622106D24FFA81F885F81B80002BB5D181
:10F9A000C5E7FFF7D9FC019BF6E700BFE08E00201A
:10F9B000F88E002030B50446C06983B010B901202C
:10F9C00003B030BD0D460023032201A9FFF734FD2B
:10F9D0000128F5D1B4F92030002B03DAFFF7BCFC85
:10F9E0000220EDE7019A012D4FEA431102EB431388
:10F9F00003D0022D12D1E5255554A268DA61227890
:10FA0000032A04D100221A775A779A77DA77626A42
:10FA10005A83C2F30F429A8203B030BDE268DA61C2
:10FA2000EDE700BF10B50378023B012B0446037ECF
:10FA300002D913F0060F5AD198063AD494F91A3025
:10FA4000591C0AD02D4A03F5B17302EB0313FF21B1
:10FA5000DA796FF30002DA71A17694F91B305A1C3F
:10FA60000FD0264A03F5B17302EB0313FF20DA79B6
:10FA7000C2F34501013921EAE17161F34602DA710D
:10FA8000E076237E1B070BD51C4841F2C873C35C8C
:10FA9000072B01D0FFF760FC41F2C8730022C2546B
:10FAA000E26A0023237084F82830FAB1BDE81040E0
:10FAB000104700231249E0691A018A58904206D083
:10FAC00001330B2BBAD01A018A589042F8D10B4A55
:10FAD00003F5B17302EB0313DA79C2F3450101397F
:10FAE00021EAE17161F34602DA71A7E710BD012155
:10FAF000FFF760FF0128F9D1237E9DE7E08E00200B
:10FB0000F8A4002030B1027822B190F828201AB170
:10FB1000002070470120704710B5D0E90142A24291
:10FB2000C16238BF22460321826080F82810FFF7A7
:10FB300079FF012010BD00BF2DE9F04FDFF868917B
:10FB40008A4699F80010DAF800300229174683B087
:10FB5000834641F6300240F08B8059F80250DEB205
:10FB6000A6EB030805EB1325B8444FF480729044CC
:10FB7000BB4208F1FF38B8FBF2F875D2A84403295C
:10FB800006EB0704A4EB03040CBF80224FF4807241
:10FB9000944228BF1446A8EB050366B994422CBFD3
:10FBA0000A220B2201A92846FFF746FC012809D0AA
:10FBB00003B0BDE8F08F0B2201A92846FFF73CFCFB
:10FBC0000128F5D199F80020DAF80010022A01F195
:10FBD000010321D0A64210D2019906F18042013AD8
:10FBE000081F00EB840001EB820242F8043F8242CE
:10FBF00003F10103F9D1DAF80010A61B7318BBF169
:10FC0000010FCAF800301BD09F4205F101052BD926
:10FC100099F800100026B2E7A642EED2DDF804C043
:10FC200006F10042013AACF1020000EB44000CEB9B
:10FC3000420222F8023F904203F10103F9D1DCE7CE
:10FC4000BB42E1D199F80030022B21D004F180446D
:10FC5000019B013C4FF0FF3243F82420DAF80030DA
:10FC60009F4205F10105D3D8012003B0BDE8F08F14
:10FC700059F8022003F07F060329C3F3D415A6EB3D
:10FC800003081544B84414BF4FF4807280226EE715
:10FC900004F10044019B013C4FF6FF72584623F8E3
:10FCA000142003B0BDE8F08FE08E00202DE9F04174
:10FCB00090F838300446032B51D8DFE803F00232C5
:10FCC0003B462D4BC0681978E76A03F5C2520329F9
:10FCD00011680CBF80264FF4807601FB06F141F2DB
:10FCE000C47C00EB412041F2A87841F2AC7E53F88D
:10FCF0000C20E06053F80E0053F808502261A5EB89
:10FD00004125A0EB4121901943F8085043F80E100B
:10FD100043F80C00C4E90C205FBB6262012384F845
:10FD2000383016480021FFF745FE012811D1022383
:10FD300084F83830626B04F130010120FFF7FCFEDB
:10FD4000012806D1032384F8383000212046FFF72C
:10FD500031FE431EDBB2012B02D9BDE8F081022047
:10FD600094F82830062B04BF002384F82830BDE81F
:10FD7000F081921B2263D1E7E08E002080A6002054
:10FD80002DE9F04FDFF8248198F80060012887B052
:10FD90008CBF00230123032E02930C460B681546EB
:10FDA00039D0022E62D14FF480724FEA1329DFB2AC
:10FDB00001920138012823D8012203929D421AD9C9
:10FDC000384E06F1880A06F11C0B32681AB1DBF8CE
:10FDD000001099424ED0DAF800000023484409226E
:10FDE00005A9FFF729FB01281FD002280FD020B159
:10FDF00023689D42E9D82560032007B0BDE8F08F55
:10FE000087B1FFF7A9FA022007B0BDE8F08F022002
:10FE100007B0BDE8F08F80220192C3F3D41903F03C
:10FE20007F07C6E7019A0392C8E7DDE902C1059A98
:10FE3000DDF804E098F80030022B14D0032BE6D153
:10FE400052F8273023F07043B3FA83F35B0963451C
:10FE50000F44236823D00B4477452360EAD309F18C
:10FE600001090027C5E732F81730EDE74FF480723B
:10FE70000192D2E70C490968013A02EB412249029A
:10FE8000B2FBF1F203991344B3FBF1F201FB12321E
:10FE90000AB10B449B1A9D42236096D8ABE7AB4254
:10FEA000ABD3A8E788A6002020A70020E08E002082
:10FEB000F0B5104D2B7841F63002022B0BBF070A2C
:10FEC000C0F3D417C4B200F07F04A85883B00E4624
:10FED00000230322384401A9FFF7AEFA012807D115
:10FEE0002B78022B019B0CBF23F8146043F824608D
:10FEF00003B0F0BDE08E00202DE9F04390F83C30D7
:10FF0000002983B0044614BF02210021042B7BD8B2
:10FF1000DFE803F0030C3C476900FFF74BFD0128C5
:10FF200070D1626B002A75D184F83C00404EDFF836
:10FF30000881404D4FF6F7771DE01FFA80F9B9456B
:10FF400094BF4FF000094FF0010901A9B9F1000F6A
:10FF500046D1FFF789FB0128494650D1206BFFF7B6
:10FF6000A7FF01284BD1019B2A682363013B9342E1
:10FF700028BF13462B603378206B032BDDD140451F
:10FF800094BF4FF000094FF00109DEE7426B04F126
:10FF900030010020FFF7D0FD012833D1032384F87E
:10FFA0003C30234BE16A41F2C47003F5C2521D5844
:10FFB0001268195041F2A87741F2AC76D8596D1AFF
:10FFC000995902FB05F200EB422501EB422203F5B1
:10FFD000BD500021DD519A51FFF7ECFC012811D1F1
:10FFE000042384F83C3094F82830042B04BF002309
:10FFF00084F82830A36B8BB120469847012003B0CA
:020000040801F1
:10000000BDE8F0830228FAD194F82830042B09D0F7
:100010000220F4E7022384F83C30B8E7012003B063
:10002000BDE8F083002384F828300220E7E700BF12
:10003000E08E002024A70020F7FFFF0F38B590F8CE
:1000400034300446052B46D8DFE803F01F033F1089
:100050001963006B4FF0FF31FFF72AFF01283AD1F7
:10006000E06A002839D1032384F834300021204687
:10007000FFF7A0FC01282ED1042384F8343094F833
:100080002830082B2DD0012038BD41F63803224DF1
:10009000EA5800F1300102320120FFF771FE012819
:1000A00024D00238C0B2012815D8052384F8343092
:1000B00094F82830082B04BF002384F8283041F23C
:1000C000E5730122EA54022038BDC06A216BFFF7B4
:1000D000EFFE0128C7D0002038BD022384F8343059
:1000E000F4E7002384F82830012038BD05F5C2521A
:1000F000E3681168D4E90B2003EB412341F6440186
:100100006850C4E9033002B96062012384F83430D6
:10011000A0E7014DCCE700BFE08E00202DE9F04FB5
:10012000436883B0C3F308081646002A00F0E18054
:10013000714B05468946A3F1180B4FF0000AC8F52C
:10014000007495F91A70B44228BF3446791C2846C9
:100150002ED0F8F765F90BEB071341F218629B58A4
:10016000984205D0FFF7F8F8504603B0BDE8F08F8D
:10017000614B03EB47202246494640445DF05AF864
:10018000002221462846FFF729FBA2440028EBD095
:100190002B7E1B0706D5594B2A691B689A4201D34F
:1001A000FFF7DAF8361BA1444FF00008C7D1DBE7B0
:1001B000F8F712F9002849D12846F8F731F96968AB
:1001C000C1F308032BBB21F4FF7323F0010303F5F4
:1001D0000072AB689A422CBF062207222B7E03F0E6
:1001E0000C030C2B1CD0002301A9FFF725F90128D3
:1001F000BAD10198404BC31A48BF03F2FF13B3F5BD
:10020000B05F4FEA63224FD257B2AF760028B2D127
:10021000AAE72B7E03F00C030C2B4FF00702E2D170
:100220009BF800C0364BBCF1030F1B680CBF4FF0AE
:10023000800C4FF4807C03FB0CF34FEA432C0CF151
:10024000FF3C0CEA0101A3EB5123CDE72B7E1A07FB
:100250002ED59BF800102A4B95F828201B680329FF
:100260000CBF80214FF4807103FB01F3062A4FEA93
:1002700043233FF479AF23490868834230D891F88B
:100280003D30002B7FF470AF002A7FF46DAF6B69B7
:1002900085F83820062185F82810EB622846FFF7FC
:1002A00005FD012888D05FE7FFF756F80198ACE715
:1002B000154B1A78002A7FF457AF95F82820002AAA
:1002C0007FF452AF082185F8342085F82810D3F840
:1002D0005F206B692846C5E90B32FFF7AFFEE0E708
:1002E00041F2E573012250460BF8032003B0BDE84C
:1002F000F08F924638E700BFF88E0020A4A60020B9
:1003000020A7002088A60020C5A600202DE9F043E4
:1003100090F8384083B00546032C00F2A180DFE856
:1003200004F0021A8B0BFFF789FE012811D0022876
:100330000BD1032385F838302B6C002085F828007A
:10034000002B00F0898098470224204603B0BDE8C6
:10035000F08385F838002B78022B79D0414A6F68FA
:1003600041F64803D3581F40C7F34F272846F8F7F4
:1003700057F8DFF8F48006463F1A0AE0D8F8003054
:100380005A1E91454AD2FFF7B5F908B9FEF7E4FFC6
:100390000136022201A900233046FFF74DF8BC19AF
:1003A00001281FFA84F94FF400724FF0000104464F
:1003B000CBD101985CF09FFFEB694FF400712846A8
:1003C000002BDBD06B68002BD8D1019B4FF0203283
:1003D0004FF02E0C1A605A6083F800C0C3F8072053
:1003E0004FF0100E6C6A1A625A6283F820C083F8CC
:1003F00021C0C3F8272083F80BE0EA6B5C83C2F3CB
:100400000F4CC4F30F4483F82BE05A879C82A3F867
:1004100034C0D8F800305A1E9145B4D3C3EBC3534F
:10042000590201F500712846FFF764F908B9FEF793
:1004300093FF022385F838302B6C002285F82820A2
:1004400063B1284698470124204603B0BDE8F083F5
:100450006F68C7F34F2789E7022476E7012474E722
:10046000002472E7E08E002020A700202DE9F04F45
:1004700090F8303089B00446042B00F2A880DFE801
:1004800013F0A900B20005008A00E800C64D41F64D
:100490001003EB5C002B40F09A80C44F04F11C0960
:1004A000B84607F1380BBA4601AE324649464046D7
:1004B000FFF70EFA012840F03F810198002800F074
:1004C00021810378E52B01D0002BEED1B84A821AA6
:1004D00048BF02F2FF12B2F5B05F4FEA622380F02C
:1004E0006F811B01B34A13449A7B042A0CD041F25A
:1004F000C86104266A5801326A5041F2CC615A60E0
:100500009E736B5801336B5041F60202AB565E1C72
:1005100009D003F5B17305EB0313FF26D979AE5467
:100520006FF30001D97141F603016B565A1C0ED0CE
:1005300003F5B17305EB0313FF26DA796E54C2F3AA
:100540004501013921EAE17161F34602DA712022A5
:1005500000215CF0D0FE2346019A53F8311F586801
:100560005060116019899B7A93721181019B627EA0
:10057000DA7205A847F0F6FABDF81430002B40F007
:10058000578144F28172019903200A82CB810A8348
:10059000CB8284F83000237E980600F1D08020467C
:1005A000FFF736F92369002B00F0D580237E03F096
:1005B000F70213F00403227640F0DB80122A00F0E9
:1005C000E180002384F828302046E36A984709B088
:1005D000BDE8F08F7548FFF71BF94FF6FF72012356
:1005E000228484F83030714F04F11C0501AE04F10F
:1005F0003109324629463846FFF76AF901282FD0DB
:100600000228E4D1684D41F60202AB56591C09D0CC
:1006100003F5B17305EB0313FF20D979A8546FF3E9
:100620000001D97141F603016B565F1C0ED003F532
:10063000B17305EB0313FF20DA796854C2F3450167
:10064000013921EAE17161F34602DA71042384F889
:1006500030300020E36A2070984709B0BDE8F08F81
:10066000DDF804800B2249464046B8F1000F00F047
:10067000AD8098F80030002B00F0A8805CF067FE99
:100680000028B6D1B8F81410B8F81A304A4A43EA2C
:10069000014312686362D8F81C30A3605202B3FBB6
:1006A000F2F102FB113109B113445B1AE36098F8CF
:1006B0000B303D4D637641F60202AB565E1C09D00D
:1006C00003F5B17305EB0313FF20D979A8546FF339
:1006D0000001D97141F603016B56581C0ED003F589
:1006E000B17305EB0313FF20DA796854C2F34501B7
:1006F000013921EAE17161F34602DA71032384F8DA
:10070000303048E73B782D49022B4FF00902504624
:100710009CD00B78002B99D1C1E905330A708BF876
:1007200000304A6B0B7351F8143CC1E90132FFF7FA
:10073000EDFD01283FF4B9AE022887D047E7E06914
:100740000023112205A9FEF777FE01283FF427AF09
:1007500009B0BDE8F08F237E19077FF532AF124A4A
:1007600041F2C873D15C00297FF431AF0721D15425
:1007700027E70023E26AA16884F828302046FFF7C3
:100780002DF824E7626AE06AA0630421C4E9023319
:10079000C4E90B2284F83C30636384F82810636258
:1007A0002046FFF735F812E7E08E0020C8A60020AB
:1007B000F88E0020F8A4002020A70020F0A600203A
:1007C000FEF7CAFD01986FF00F038BE6294D41F645
:1007D0000202AB56591C09D003F5B17305EB0313A4
:1007E000FF20D979A8546FF30001D97141F60301B4
:1007F0006B565A1C0ED003F5B17305EB0313FF20A3
:10080000DA796854C2F34501013921EAE17161F3F3
:100810004602DA71237EDF067FF518AF1648FEF731
:10082000F7FF4FF6FF720223228484F830302EE661
:10083000124B05A9B3F95C2D02A847F0E7F99DF822
:100840000C309DF80D609DF80A509DF80B20BDF806
:1008500008109DF80E00DB0243EA461342EA4512F7
:10086000A1F2BC7143EA500342EA41229BB292B228
:1008700089E600BFE08E0020C8A60020A84E002018
:100880002DE9F04390F82830013B83B00446082B53
:1008900041D8DFE803F048054D525865406A4300EF
:1008A000384B4668056B41F6480103F5C2525F5864
:1008B00013683740EA19B2EB432F4FEA432816D2A8
:1008C00058E02169207EFEF7F7FE012823D1256B31
:1008D000666823696361A5EB08053D444644F61B41
:1008E000019B6660A84525634F46236142D8204698
:1008F000F7F772FD01AA81460028E2D06668A36876
:10090000E26A9E4238BF1E460023A66084F8283063
:100910000AB12046904703B0BDE8F083FFF7F6FC2C
:1009200003B0BDE8F083FFF7A1FD03B0BDE8F0839D
:10093000FFF778F803B0BDE8F0830021FFF7DCFA99
:1009400003B0BDE8F0830121FFF7D6FA0128E2D118
:100950000023216C84F828302046FFF7D3F8DAE72B
:10096000FFF7A4F903B0BDE8F083FFF767FB03B01E
:10097000BDE8F0832046F7F72FFD0028BFD12E44B5
:100980006660BCE7E08E002010B5114C94F8A63EDE
:1009900023B9104B4FF480225A6110BD0E4A1368E0
:1009A00023F00603136058F09BF994F8A63E002B41
:1009B000EFD0D4F8AC3E9B68DB07EAD5D4F8A82F7B
:1009C000136823F0030161F307031360E1E700BF3D
:1009D000B03D0020003C014010ED00E02DE9F04763
:1009E00004460D469046002144221E46089F5CF0B6
:1009F00082FC01234FF6FF722676628384F828304A
:100A00002B782E2B4CD02E4604F1310A307804F18D
:100A1000390968B12E280BD043F0B4FBC0B20AF8F4
:100A2000010BCA4506F1010607D030780028F1D144
:100A300020200AF8010BCA45F7D130782E2808BFCC
:100A4000707804F1380908BF013604F13B0A58B147
:100A500043F098FBC0B209F8010FD14506F1010639
:100A600007D030780028F3D1202009F8010FD145B4
:100A7000F7D118F0100F14BF0323012384F8198055
:100A80002370E7622B782E2B26D16B7823BB0323B0
:100A9000204684F83030FFF7E9FC2046BDE8F087B7
:100AA0006B78002BAFD1114B41F2F47241F60C0080
:100AB00041F2F0719A5818585958E26041F6010213
:100AC0006062A1609A5C627641F2E8729B5C23707E
:100AD000E7622B782E2BD8D00023204684F83030C4
:100AE000FFF7C4FC2046BDE8F08700BFE08E002081
:100AF00008B50121032003F077FB72B64BF086FEA8
:100B00002DE9F04FCE4CDFF844938DB000270090D4
:100B1000A4F2074504F6611A54F80B0C002800F003
:100B2000FE8039F0FBFC0646002800F0D381D9F89E
:100B3000003944F8073CE0260023A4F10B0B04F82D
:100B4000033C7E4354F80B0C39F0E8FC002800F01D
:100B5000E68054F80B0C39F0D9FC14F8023C5A1E0C
:100B600080460B2A0DD8DFE812F01F003A0046003D
:100B7000530083009B00E30016013501400173011F
:100B80008A0124280CD0009A3AB995F86E2C82423A
:100B900040F07B81012204F8032C0D2BD2D186E09A
:100BA000012304F8023CCDE700234D28C4F8C530EA
:100BB00084F8CD3084F8CE3004D0582808D004F81A
:100BC000023CBFE7022204F8022C84F8C430B9E7E3
:100BD000032304F8023C022384F8C430B2E7042360
:100BE0003C2804F8023C0BD0B8F13E0F0CD0002397
:100BF00004F8023CA6E70A233C2804F8023CF3D19F
:100C0000002304F8013C9DE7012304F8013C99E727
:100C1000D4F8C500AB190344421CC4F8C52083F8BE
:100C2000078494F8CD00022A88EA000184F8CD10E8
:100C300088D12378C02BDAD86278FF2A08D1052B17
:100C4000D5D9012384F8C430072304F8023C79E79E
:100C5000A4F8C12000229342C4F8C93014BF052370
:100C6000062384F8C320C4F8C52004F8023C69E7D1
:100C7000D4F8C500AB190344421CC4F8C52083F85E
:100C8000078494F8CD00D4F8C93088EA00019A426C
:100C900084F8CD107FF456AF062304F8023C51E7E8
:100CA00094F8CD308342A2D10D2304F8023C14F80D
:100CB00001CCBCF1000F40F0EE80624B08940FCBEA
:100CC00004AE86E80F00D4F8C930D4F8D100ADF8EE
:100CD0002CC023440993B4F8C130ADF8283094F8FF
:100CE000C3308DF82A3001238DF82E30324603AB05
:100CF00008A9CDF80CC032F07FFC48B1049B0593E5
:100D000094F8C420504B04933146584630F08AF989
:100D1000039E002304F8023C002E40F0D3800137EC
:100D2000032F04F1E0047FF4F7AE0DB0BDE8F08FBF
:100D3000D4F8C500AA190244431CC4F8C53082F88F
:100D4000078494F8CD2094F8CE00019388EA02023B
:100D5000414684F8CD2047F0EFF9019B84F8CE009E
:100D6000072B7FF4EFAEB4F80530C02B3FF63FAF52
:100D7000B4F80320A4F8C120A27884F8C32000228C
:100D80009342C4F8C93014BF08230923C4F8C5200E
:100D900004F8023CD6E6014694F8CE0047F0CCF9C0
:100DA00094F8CD3084F8CE0088EA0303D4F8C50067
:100DB00084F8CD30AB190344421CC4F8C52083F835
:100DC0000784D4F8C9309A427FF4BCAE092304F8F2
:100DD000023CB7E694F8CD30434084F8CD3094F827
:100DE000CE3083427FF403AF56E7D4F8C500AA198A
:100DF0000244431CC4F8C53082F8078494F8CE003E
:100E00000193414647F098F9019B84F8CE00052BE9
:100E10007FF498AEB4F80120B4F80330A4F8C120F0
:100E2000227884F8C32000229342C4F8C93014BF4A
:100E30000B230C23C4F8C52004F8023C82E600BF53
:100E4000AF520020ECD70608A0570120C01B00209D
:100E5000014694F8CE0047F06FF984F8CE00D4F83C
:100E6000C500AB190344421CC4F8C52083F80784AD
:100E7000D4F8C9309A427FF465AE0C239FE694F80B
:100E8000CE3083427FF4B3AE0EE7232804BF0222A4
:100E900004F8032C81E6BCF1010F4FF0000602D0EC
:100EA00004F8026C3BE7D4F8C93008942344099352
:100EB00008A8B4F8C130CDE90A66ADF828302FF0A3
:100EC00009F8EDE754F80B0C30F0EAFA54F80B0C83
:100ED000B04724E714F8033C002B3FF420AFD9F8C7
:100EE000002954F8071C521A632A7FF618AF012B09
:100EF00030D0022B7FF413AF54F80B3CC5F8603DA3
:100F0000C5F8643DC5F86C3D4023012285F8703D6D
:100F100095F8B73685F85E2D0F4AC5F8682D003B69
:100F20000E4A85F8710D18BF01230D4882F8AC3BBD
:100F3000C5F8E4AAC5F8B4AD3FF042FC4FF4005048
:100F400032F010FA07483FF031FC85F8B86D85F8AB
:100F5000B96DE4E6FFF7CCFD856B040814000010C2
:100F6000378707086D870708034B93F8240000387C
:100F700018BF0120704700BF201C0020202301481B
:100F80000B80704754040020642301480B80704795
:100F900074040020432301480B807047D8040020CC
:100FA00010B5074CD4F8C800FF2807D0054951F800
:100FB000042BF7F749F9FF23C4F8C830002010BD0F
:100FC0005404002038A70020EAE700BF08B5D0F895
:100FD000E4355B6A9847002008BD00BF08B5D0F82B
:100FE000E4351B6A9847002008BD00BFD0F8E435FF
:100FF00010B504461B689847D4F8E8359B689847B5
:10100000002010BD08B5D0F8E435DB6903B198477E
:10101000002008BD08B5042290F81211D0F8E83578
:1010200080F8131180F81221DB689847002008BD72
:1010300010B5D0F8E83504461B699847032384F8B7
:101040001231002010BD00BF0B0630B41CD401EBE0
:10105000810200EBC202002300EB810582F87413C9
:1010600082F8753301241A4604FA01F16D6D61F3BB
:101070001F4201696FF3CF332B60CB6923EA020370
:10108000002030BCCB61704701F07F0101EB81048F
:1010900000EBC404012200EB8105002384F81C113D
:1010A00084F81D2102FA01F11A46AD6961F30F02BD
:1010B000DFE700BF10B581210446FFF7C5FF2046DA
:1010C0000121FFF7C1FF024B0020187010BD00BFC7
:1010D000E45B002010B581210446FFF7B5FF2046F0
:1010E0000121FFF7B1FF82212046FFF7ADFFF7F79F
:1010F000F1F8002010BD00BF38B50D46044683212D
:10110000FFF7A2FF29462046FFF7E4FF002038BD85
:10111000F0B416460A063AD401EB810500EBC5058A
:101120002824002204FB0104022B85F87413C5F85F
:101130007C6385F8773385F8752304F55D7448D0B2
:10114000154600EB8107012202FA01F17F6D61F380
:101150001F45D7F800C01CF4004F11D1E488204986
:1011600046F0805242F4004242EA834204F00F0407
:101170001C4B42EA845211400CEA030319433960C4
:101180000269D3692B430020F0BCD361704701F0A2
:101190007F0101EB810500EBC5052824012204FB3A
:1011A0000104022B85F81C11C5F8246185F81F3154
:1011B000A5F8221185F81D2104F58E740CD00025A8
:1011C00000EB8107012202FA01F1BF6961F30F050B
:1011D000BFE722711546B4E700252571F0E700BF8F
:1011E000FF87CC13007833EC002310B51946044672
:1011F0004022FFF78DFF8021204600234022FFF789
:1012000087FFD4F8E835A078012284F812215B68C2
:101210009847002010BD00BF70B44B78012B26D03A
:101220000B784A6900EB83035C6D25682369D2B1B2
:101230008A684A6102F07F0223F4002323F07F03CF
:1012400042F4002213432361C378012B04BF0B69CE
:101250006361C5F3076363F07B0363F31F65256078
:10126000002070BC70478A6802F07F02E4E7826960
:101270004C691568136944B38E68B4428CBF06F09C
:101280007F0404F07F0423F4002323F07F0344F45D
:10129000002443EA040388BF4E611361C378012B25
:1012A0001DD0C5F3076464F07B0464F31F6515600B
:1012B000002BD5D14B69002BD2D002690878516B35
:1012C000012383400B435363CAE723F4002323F035
:1012D0007F0343F400231361C378012BE1D10B7822
:1012E0000C6900EB8300C5F30763816963F07B033E
:1012F00063F31F654C610020156070BC704700BF30
:101300002DE9F0434B78012B30D00B784C6900EB82
:1013100083035E6D356837691CB38B681C44013CE0
:10132000B4FBF3F4C4F3090203FB02F3C3F31203A7
:101330004B61144643EAC44363F31C073761C37827
:10134000012B04BF0B697361CB78012B44D0C5F32B
:10135000076363F07B0363F31F6535600020BDE81E
:10136000F0838A680124C2F31203E3E791F8008056
:101370004E6900EB880EDEF818C0DCF80050DCF88F
:10138000107076B3D1F80890384A06EB0904013C96
:10139000B4FBF9F402EAC444C6F312022243CC7847
:1013A00007F060473A43012C174649D0CCF810208B
:1013B000C278012A55D00269516B03FA08F30B4336
:1013C0005363C5F3076363F07B0363F31F65CCF8D6
:1013D00000500020BDE8F0834B7973B345F0005511
:1013E000B5E707F0604747F40027CC78CCF81070D9
:1013F000C378012B2FD0012CE3D102699268D2056A
:1014000054BF45F0005545F08055C5F3076262F0C2
:101410007B0262F31F65CCF80050002B9ED1B0B266
:1014200003308010DEF8D04098D0CA6852F8041B10
:10143000216001339842F9D190E745F0805586E765
:1014400064F35E77CCF81070C378012BD5D10A69AC
:10145000CCF81420D1E70A69CCF81420012CB0D1C3
:10146000CBE70B69CCF81430ABE700BF0000F81FE6
:101470000E4BDA68D20310D4DA68D1060FD4DA68DA
:10148000D20510D4DA6812F0E00F0AD1DB6813F04D
:10149000020F14BF08200920704701207047062062
:1014A0007047072070470220704700BF003C024091
:1014B00000207047002070477047704730B1044BE0
:1014C00093F90C000028D4BF00200120704700BF12
:1014D00038A7002008B5FFF7F1FF50B1054A537B4C
:1014E000927B5B0003F00203002A18BF43F0010364
:1014F0000B6008BD38A7002008B5FFF7DFFF10B16B
:10150000014B1B690B8008BD38A7002070B5FFF7A1
:10151000D5FF78B1084A958A65B196690023B34230
:101520001C4607DA02EB44040133A48BAC42DBB265
:10153000F5D30B7070BD00BF38A7002008B5FFF7CA
:10154000BDFF10B100230B70137008BD042070475D
:1015500028B1034B93F9CC00003818BF0120704725
:101560005404002008B5FFF7F3FF50B1054B93F981
:10157000CC20012AC3BF93F8CF30C3F340030B60E4
:10158000002008BD5404002008B5FFF7E1FF18B1A2
:10159000024B93F8CE300B7008BD00BF54040020FE
:1015A00070B5FFF7D5FF38B10E4C94F8CF30DB079C
:1015B00003D500230B70137070BD0B4D94F9CD3023
:1015C00095F82C6093FBF6F301330B7094F9CD4042
:1015D00095F82C1094FBF1F301FB134301331370C6
:1015E000EAE700BF5404002038A70020032070471A
:1015F00070B50A4A92F8303006255E1CB6FBF5F449
:1016000005FB146492F83150AC4205D002EBC303E1
:10161000C3E90D0182F8304070BD00BF38A700203B
:10162000002230B504461046914200DC30BDA35C78
:101630000825584010F0800F4FEA400318BF83F090
:10164000D503013DD8B2F5D10132EDE710B5D9B1DE
:101650000E4B586E814217DCB2B1DB6A9A4213DC42
:101660000B4C013A013903FB012184F8DA1004F133
:10167000D6000521FFF7D4FF062184F8DB0004F132
:10168000D600BDE81040B3E710BD00BF38A700206A
:1016900054040020024B93F868300B60012070471F
:1016A00038A70020024BB3F86A300B800120704746
:1016B00038A70020024B93F86C300B700120704764
:1016C00038A7002000230B700120137070470038EA
:1016D00018BF012070470120704770470023038026
:1016E00083708380C3800372704700BF074A084934
:1016F00092F86D3009780133DBB2994282F86D308F
:1017000004BF002382F86D30704700BF38A7002067
:10171000C40B0010F8B5774C236F83B1764B1B6870
:1017200093F82E305BB1754B94F87420A3FB001333
:10173000012A4FEA93132FD0022A08D002B1F8BD34
:101740006F4B9842FBD9012384F87430F8BDA26F27
:1017500064329A423CD894F86D3004EB031393F84A
:10176000EC24FF2A06D067490132012083F8EC24DB
:1017700081F8DC00FFF7BAFF634B1B780122092BCD
:1017800084F87420DBD1B4F86E35604A01339BB223
:10179000A4F86E355380F8BD94F86D105A48A367CD
:1017A0008C2303FB0143007883F88E20002384F808
:1017B0008A3004F180050A2202230928E56784F8AB
:1017C0008B2084F87430BAD1504B01311980F8BDA8
:1017D00094F88A2094F88B309A42B0D104F17F00BB
:1017E00004F18805002310F8012F082153405A0006
:1017F00013F0800F08BF5B0082F0070214BFD3B262
:10180000DBB20139F3D18542EDD194F889209A42B7
:1018100039D194F86D6094F8875094F88830B4F812
:101820008300B4F8852094F881C004EB061743EADE
:10183000052394F8825087F8EC1440BA52BA81B26A
:1018400092B245EA0C202F4DC7F8F0141BB294F960
:101850008010C7F8F424032E4FF00102A7F8EE041D
:10186000A7F8F83487F8ED1485F8DC2008D8264A64
:1018700012780C2A29D00D2A02D1244B23F81610F5
:10188000FFF734FF5FE794F86D3004EB031393F830
:10189000EC24FF2A06D01B490132012083F8EC24F6
:1018A00081F8DC00FFF722FF174B1B780122092B80
:1018B00084F874207FF443AFB4F86C35134A0133D5
:1018C0009BB2A4F86C359380F8BD1149114A897E0A
:1018D0000E4803EB830303EB830349089B0093FB50
:1018E000F1F382FB0312DB17C3EBA20320F81630DF
:1018F000C6E700BF38A700205C090010D34D621076
:101900003F4B4C0054040020992800209C280020C4
:1019100034310020676666660A4B93F88A1093F8A4
:101920008B2091420DD010B493F88A20DC6F511CAB
:10193000D2B2C0B2C9B283F88A10A0545DF8044B89
:101940007047704738A70020FD2870B522D0F028D6
:1019500004D0EF2822D00224204670BD114D032070
:10196000052641282E444FF0000405F1010580F0C2
:1019700080030DD0042B0BD9FFF7E6FF2044B542BE
:10198000C4B2E9D015F8010B412880F08003F1D1F1
:101990000420F3E7044D0B200426E2E7034D0C205E
:1019A0000626DEE724DD060820DD06082CDD060815
:1019B0000E4B0F4AD3F87035B2F904005B0707D419
:1019C00000EB8000400080B200F5C87080B2704724
:1019D000084B094A9B6B323382FB0312D817C0EBCA
:1019E000A20080B200F5C87080B2704738A700200E
:1019F000C40B0010BC4B0020676666660C4AD2F828
:101A0000883530B41C68D2F880555D601981002596
:101A1000611C19609D812070D2F88835D2F880153C
:101A20001A685A604FF6F67230BC19609A81704796
:101A300038A70020114B30B4D3F82C27C3F8302737
:101A400003F28C5003F21C6103F20C6503F21C7468
:101A50000132C3F88455C3F88845C3F82C2730BC3D
:101A6000C3F87C05C3F80C06C3F81006C3F880154C
:101A7000C3F81C17C3F82017704700BF38A7002011
:101A800000B583B00268084B8188CDF8012032226E
:101A9000D3F83437ADF805108DF800206846984724
:101AA00003B05DF804FB00BF38A700205E2810B526
:101AB00011D05D2805D00D4BBDE81040D3F8383764
:101AC00018470A4CD4F838379847D4F838373D20AF
:101AD000BDE810401847054C5D20D4F838379847CA
:101AE000D4F838373E20BDE81040184738A700200A
:101AF00070B5094E0546D6F838375E200C46984733
:101B0000D6F8383728469847E0B2FFF7CFFFC4F33E
:101B10000720BDE87040C9E738A7002003682DE919
:101B2000F041002B3D4D3E4F3E4EB8BF5B42A5FB02
:101B30000321890D07FB0137C7EB0717BF0096F894
:101B4000423785FB0725FA170446C2EBA555002B43
:101B500057D101EB810101EB810105EB810109B254
:101B6000DFF8BC801320FFF7C3FF2F4908FB057582
:101B700081FB0531ED17C5EBA11109B21B20FFF761
:101B8000B7FF2368254D002BB4BF53214E212320DE
:101B9000FFF7AEFF636896F8422783EAE376A6EB89
:101BA000E376A5FB0631890D08FB0168C8EB081830
:101BB0004FEA880885FB08354FEAE873C3EBA55563
:101BC0002ABB01EB810101EB810105EB810109B227
:101BD0001220FFF78DFF124B134903FB058581FB94
:101BE0000531ED17C5EBA11109B21A20FFF780FFEF
:101BF0006368002BBDE8F041B4BF57214521222086
:101C000076E7C1EB011105EB810109B2A8E7C1EB51
:101C1000011105EB810109B2DAE700BF6BCA5F6B06
:101C2000806967FF38A70020D34D6210044BD3F8BA
:101C30005C3730EA030314BF01200020704700BF67
:101C400038A7002030B40023022515244FF4167164
:101C500040F2D93205808471018130BC42814380D9
:101C6000838083817047134B10B400220F2483F8C4
:101C70006217090A83F8610783F86317C3F86427BA
:101C8000C3F86827C3F86C2783F8604703F5EC6056
:101C9000012110F8014F013122440E29D2B2F8D1AE
:101CA00083F86E270449D3F870075DF8044B1022BF
:101CB00038F004BC38A7002098AE0020054B002166
:101CC00083F87417C3F87817D3F8703703B1CAE7ED
:101CD000704700BF38A7002013B50446FFF738FC53
:101CE00008B300230DF106022046ADF806300DF0D2
:101CF000A9FCC0B10D4C9DF8062094F9CC1084F8D5
:101D0000E120032908BF62F07F024FF00501084877
:101D100008BF84F8E120FFF783FC062184F8E20085
:101D20000348FFF765FC02B010BD00BF540400205B
:101D30003105002008B5044BD3F87C0738F0EEFBE2
:101D4000B0FA80F0400908BD38A700202DE9F84F0F
:101D50001B4C05461E2094F880A794F881B794F890
:101D60008267B4F88497B4F8868794F8887722F06D
:101D7000DDFB30B1B8F1000F03D0C14601264FF0B2
:101D8000000A94F88A37DA070AD494F88F273AB908
:101D9000012F12D0022F03D113F0020F08BF01262A
:101DA00085F800A085F801B0AE70A5F80490A5F8FC
:101DB00006802F722846BDE8F88F3E46F0E700BF48
:101DC00038A700202DE9F84F2DED028BFFF7C0FB5F
:101DD000002844D0264B93F9CC0001283FDD93F82E
:101DE000E340DFF894809FED238A0FF27C0BDBE960
:101DF00000AB15468E1E02EB44094D4504D1BDECE7
:101E0000028B2046BDE8F88F38F8027B26F8027F67
:101E100007EE907AF8EEE77A67EE887A17EE900A86
:101E200057F06AF952465B4657F0BEF941EC100B89
:101E30005AF092FF51EC100B57F0DEFC0E2F80B2DF
:101E40000AD919303223B0FBF3F080B200EB8000E6
:101E500000EB8000400080B225F8020BCDE70024A3
:101E6000CDE700BFAFF300801655B5BBB16B0240A4
:101E700054040020CDCCCC3DECAE002038B50D464E
:101E8000FFF766FB044638B10C4890F8CF30DB070B
:101E900004D5B0F8D0002880204638BD084A90F913
:101EA000CD3092F82C2093FBF2F102FB113201327B
:101EB0000131E4300DF0DAFBEDE700BF54040020FF
:101EC00038A7002038B5134C94F8313094F83020FE
:101ED0009A4219D004EBC3030F49D3E90D20002324
:101EE000984212DC93780D4AC4F8C4075B0813705B
:101EF000FCF706FB94F8313006210133B3FBF1F215
:101F000001FB123384F8313038BDD55C01F8015B38
:101F10000133E5E738A70020585B0020865B0020EE
:101F2000A1F5AF53B3F5AF7F70B541D8214BD3F8CE
:101F3000C807A3F86A10B0B94FF47A744C434FF451
:101F4000C8714BF0F9FF2823B4FBF3F303F03F0310
:101F50004FF420610120B4FBF1F1BDE8704043EA89
:101F6000C1114BF0E9BF144C4068A1FB044580212E
:101F700056F0AEF843F210204CF03EF80A2037F04D
:101F8000B7FC0E4A00232046294657F0A5FCC0F3B3
:101F90000510460129462046094A002357F09CFCBB
:101FA00046EA003040F01100BDE870404CF024B823
:101FB00070BD00BF38A700200084D71740420F0033
:101FC0000000093D13B500230DF106020C46ADF8E3
:101FD00006300DF037FB30B1044B9DF8060083F856
:101FE0006C404CF041F802B010BD00BF38A7002093
:101FF000194B37B593F8682004461D4651B13AB9DC
:10200000D3F8CC07012283F8682008B13BF0A4FA8A
:1020100003B030BD002AFBD0D3F8CC0783F868109A
:1020200008B13BF093FA4FF4AF7037F07FFD95F9AC
:102030006C1000230DF106022046ADF806300DF0BD
:1020400001FB9DF806004CF00FF8B5F86A10204629
:10205000FFF766FFDCE700BF38A700202DE9F04F4F
:10206000AB4B1B788BB08046002B40F0B980A94D5C
:10207000D5F8D067002E00F0B380A74AD2F8E84028
:1020800004F0F021B1F1E02F70D1C2F8E830D5F8BA
:10209000D42794426AD004930593ADF81830B5F86C
:1020A000843795F880E7ADF8143095F881C795F836
:1020B000883795F882B78DF818300DF1100A8DF831
:1020C00010E08DF811C08DF812B09AE8070007AB48
:1020D00003C3924F1A80C4F342533B44C4F30342F8
:1020E000997CC5F8D4478E4502F1010201D194458F
:1020F00008D030468DF81C108DF81D200DF0B6FA72
:10210000ADF8200030460DF067FD032804F0070904
:1021100037D0042838D001283AD14F44FB7D9B4565
:1021200001A9304618BF8DF81E300DF0E3FA48B112
:10213000019BC4F3001103F001038B4202D030462F
:102140000DF0E8FC0A2207A950465BF0ACF868B134
:102150009DF81E30BDF81C2085F88237BDF8203070
:10216000A5F88027A5F8843746F040F995F8D8A758
:1021700004AF95F8D837032B7CD8DFE803F00B3495
:1021800077A44F44FB7FCAE74F4497F82730C6E750
:102190000023C4E7394630460DF0B2FA044658B180
:1021A00007A8FFF7D3FD9DF81E109DF810308B4255
:1021B00060D030460DF0B1FC95F8D837013303F00C
:1021C000030385F8D8370CB99A45D2D195F88A37E8
:1021D000DB0700D524B1336841461B683046984779
:1021E0000BB0BDE8F08F01A8FFF7B0FD95F88A9716
:1021F0009DF8044009F00109ECB1B9F1000F39D1A3
:102200003A460DF1030130460DF0E4FA044688B376
:1022100007A8FFF79BFD9DF81C109DF803309DF863
:102220001D208B4203D19DF81030934222D03046BE
:102230000DF07EFCC0E7B9F1000FBDD13946304644
:102240000DF05BFA0446A8B107A8FFF77FFDBDF8C3
:102250002010BDF810308B420CD085F8D99785F846
:10226000DA97336830469B699847A5E795F88A372F
:10227000D80701D500249FE707A930460DF03AFAA8
:1022800004460028F6D01E2022F050F995F8DB37DE
:1022900083428146EED085F8DB0760B1B5F886371A
:1022A000002BE7D1079BD907E4D4012130460DF07C
:1022B00031FC4C4680E7079BDA07DBD50146304608
:1022C0000DF028FC78E73846FFF740FD97E8070057
:1022D00007AB03C31A809DF810309BB10DF11D02AE
:1022E00007A930460DF076FA0DF11E0130460DF0CB
:1022F00007FA0A2207A938465AF0D5FF041E18BF6C
:10230000012459E708A930460DF0F7F9ECE700BFC2
:10231000065C002038A700205404002020DD0608B9
:10232000024B0146D3F8DC0738F0FCB838A7002090
:102330002DE9F041FD2984B0044600F0DE80F0294B
:1023400000F0BD80EF2900F031814AB103468618C4
:1023500003AD002003F8010B9E4205F8010BF9D1F3
:102360009A4B0B2003F1090501E013F8010F81429C
:1023700000F0C880AB42F8D14B1E832B00F2938053
:10238000DFE813F03201390143014E01BE01840040
:10239000580163016F01910091007501750175018C
:1023A0008B018B018B016F019100910096019E01C1
:1023B0009100910091009100910091009100910095
:1023C0009100910091009100910091009100910085
:1023D0009100910091009100910091009100910075
:1023E0009100910091009100910091009100910065
:1023F0009100910091009100910091009100910055
:1024000091009100B4019100910091009100910020
:102410009100910091009100910091009100910034
:102420009100910091009100910091009100910024
:102430009100910091009100910091009100910014
:102440009100910091009100910091009100910004
:1024500091009100910091009100910091009100F4
:1024600091009100910091009100910091009100E4
:1024700091009100910091009100910091009100D4
:1024800091009100910091001F011F01504BB3F882
:102490000C18002900F0668101922EF09FFA019A33
:1024A00080B2ADF80C003AB1224403AB13F8011B23
:1024B00004F8011BA242F9D104B0BDE8F081454FF8
:1024C00003214FF00508B844002501370CE0FFF761
:1024D0003BFA064660193246FFF72AFF7019474556
:1024E000C5B2E9D017F8011B412981F080030846E5
:1024F00001D0042BEBD80426ECE7374F0B214FF02B
:102500000408E0E7324BD3F8700580060CD4002AAB
:10251000D2D0224403AB13F8011B04F8011B9442F0
:10252000F9D104B0BDE8F08193F8E007870742D500
:102530002A4D287D052834BF02260326142917D9E1
:102540007C39C8B20628E2D80629E0D801A050F8A4
:1025500021F000BF3D2701083D270108272701087A
:102560000F2501084D2701084727010853270108B7
:102570000929CCD90A390A29C9D801A757F821F065
:102580000D270108592701080F2501080F2501080B
:102590000F2501080F2501080F2501080F25010847
:1025A0000F2501081F2701083D2701080C4F0C21AA
:1025B0004FF0060887E7094B0B29187DA7D10126A4
:1025C000CBE0084B5B6B03936DE700BF50DD060863
:1025D00038A7002024DD060820DD0608905A0020D8
:1025E0002CDD0608BC4B00200192FFF7E1F9019AAF
:1025F000ADF80C0057E76C4BD3ED037AFDEEE77AAC
:1026000017EE903AADF80C304DE7684B93F847075A
:10261000B3F8E417002840F0AB80ADF80C1042E7A7
:102620006249B1F8E43791F8EC17B3FBF1F3ADF878
:102630000C3038E75D4D95F88A37DE0700F19D8054
:10264000B5F80C38ADF80C302DE7584B5849B3F9B4
:10265000303881FB0301DB17C3EBA103ADF80C306D
:1026600021E7524BB3F83238ADF80C301BE7514B31
:10267000DFED516AD3ED027A0C39C9B203EB810365
:1026800093ED167A67EEA67A67EE877AFDEEE77A23
:1026900017EE903AADF80C3005E7444B03EB4101DF
:1026A000B1F80E3803EB83035B00ADF80C30FAE6AB
:1026B0003E4B93F88A3703F00103ADF80C30F2E695
:1026C0003A4BB3F82818CD055ABFCB4303F00103AA
:1026D000032311F0440F18BF042311F0020F18BF99
:1026E000072311F4806F18BF0923ABE70192FFF7AE
:1026F0005FF9324B019ADB6B43EAC0400390D2E6AC
:102700002A4BD3F81C38ADF80C30CCE62B8A03EBFF
:10271000830303EB83039B00ADF80C30F7E6EB89F2
:10272000ADF80C30F3E6EB89254903EBC3039B00BE
:10273000A1FB03135B09ADF80C30E8E6B3F8E23710
:10274000ADF80C30E3E66B680393E0E62B68039387
:10275000DDE6AB680393DAE6F6B28DF80C608DF82F
:102760000D00D4E6D3F8240880F3100080B298E678
:1027700093F8EC37B1FBF3F14FE705F5FE650192F5
:1027800022F0E4F8D5ED037A019AFCEEE77A17EE31
:10279000903A9BB200287FF455AF0A49096811F0BE
:1027A000100F18BF00234DE728AF002038A70020E6
:1027B00067666666C40B001000007A44BC4B0020BC
:1027C0001F85EB515859002070B5214D95F83438CC
:1027D000EA181C4692F838288AB11E4E09225C1C61
:1027E000A6FB04135B0803EBC303E31AE918DCB28E
:1027F00091F8381809B1013AF1D185F834480268E6
:102800001549561C06600C2616700268561C066098
:10281000002616700268561C066003EB430603EBA5
:102820008603147019440D2240F050F995F83418BD
:10283000084B4A1CA3FB02035B08294403EBC303B8
:102840000120D31A81F8380885F8343870BD00BFEC
:1028500038A70020398EE3387CAF00202DE9F04105
:102860006A4ED6F8D07784B0044638460D460DF04F
:10287000B3F986F8B90857B10DF1090202A9384633
:102880000CF0A8FF002840F0838096F8B9080023D8
:10289000ADF808308DF80A301A46431EDBB200212D
:1028A000FF20FD2B8DF80C20ADF80E108DF80B00DD
:1028B00003D9002004B0BDE8F0819DF80830042B56
:1028C00000F09D80052B00F09D80032B00F09C8084
:1028D000022B00F09380012B08BF042100F08F80B1
:1028E0009DF809309DF80A10D6F8D007013B0DF18C
:1028F0000E028DF809300CF0A5FE96F8B938032BBE
:102900007AD0042B76D0012B64D0D6F8BC28029B59
:102910003F4F9A420DF108084FD023680D22591CF1
:1029200021601A7023680022591C21601A702368E4
:102930009DF80820591C21601A7023689DF8092011
:10294000591C21601A7023689DF80C20591C2160C5
:102950001A7023689DF80A20591C21601A70BDF86E
:102960000E10204640F0FAF823689DF80B20591C01
:10297000216020461A700721FAF78EFF98E80300BD
:1029800087E803000120C6F8C45804B0BDE8F08110
:1029900001A938460CF0AEFE00283FF476AF384669
:1029A0000DF10A010CF0ACFE00283FF46EAF019B64
:1029B00096F8B90803F001026FE77A68D8F8043096
:1029C0009A42AAD1D6F8C438124AEB1A93427FF63B
:1029D00070AFA2E7104A9DF80A000121002304E02D
:1029E0000133082B91D012F8011F8142F8D38DF8E2
:1029F0000A308AE7094AEEE7094AECE703218DF835
:102A000008106DE70121FAE70221F8E738A7002056
:102A1000F4AF002080841E0037DD060847DD06087D
:102A20003FDD06082DE9F0412A4C2B4AD4F81C382A
:102A3000B4F8C878B4F8246882FB0352DB17C3EB00
:102A4000A2031FFA83F8474582B00D4603D1B4F8BC
:102A5000CA38B34233D002680190511C342301605C
:102A6000137002680023511C01601370414640F04E
:102A700075F80198314640F071F8019847F6FF71FA
:102A800040F06CF8019847F6FF7140F067F8019844
:102A900047F6FF7140F062F8019847F6FF7140F089
:102AA0005DF801980221FAF7F7FE0120A4F8C88822
:102AB000A4F8CA68C4F8CC5802B0BDE8F081D4F8D4
:102AC000CC38064ACB1A9342C5D8002002B0BDE8E4
:102AD000F08100BF38A700206766666680841E000C
:102AE000026810B57F21541C046011700268002434
:102AF000511C01600E211470FAF7CEFE012010BDAA
:102B00002DE9F04FC24B1B68804613F0800083B064
:102B100000F07181BF4B93F8E00710F0020000F065
:102B20006A81DFF810B39BF81430052B40F26881FE
:102B3000DBF80030B84D0093002BB8BF5B42A5FB1B
:102B40000342B648B649920D00FB0233C3EB0313B0
:102B50009B0085FB034502EB8202DC1702EB82023D
:102B6000C4EBA55400FB043304EB8204A4B281FB44
:102B70000321DB17C3EBA111BCB10025A94F2E46E1
:102B8000A7FB0432D20802EB8203A4EB4303E8B2B2
:102B9000A4469BB280008340BCF1090F94B246EA80
:102BA000030605F10105EBD8340489B2B9B100255B
:102BB0009C4F2E46A7FB0132D20802EB8203A1EB09
:102BC0004303E8B28C469BB280008340BCF1090FFE
:102BD00091B246EA030605F10105EBD83443DBF870
:102BE00004E08D4D8D4E8E498EEAEE70A0EBEE70B6
:102BF000A5FB0032920D06FB0200C0EB0010830023
:102C000085FB035002EB8202DD1702EB8202C5EB6B
:102C1000A05506FB053305EB8205ADB281FB032110
:102C2000DB17C3EBA111C5B10020DFF8F8C10646E0
:102C3000ACFB0532D20802EB8203A5EB4303C7B21B
:102C4000A9469BB2BF00BB40B9F1090F95B246EA55
:102C5000030600F10100EBD8350489B2C1B10020B0
:102C6000DFF8C0C10646ACFB0132D20802EB82039A
:102C7000A1EB4303C7B289469BB2BF00BB40B9F189
:102C8000090F91B246EA030600F10100EBD8354383
:102C9000DBF80830634A0193002B1846B8BF58424E
:102CA000A2FB0030604E6149030AA6FB0363DB0907
:102CB00001FB03F1C1EBD00189B2B9B10026914605
:102CC0003746A9FB0132D20802EB8203A1EB430392
:102CD000F0B28C469BB280008340BCF1090F91B2E8
:102CE00047EA030706F10106EBD8B9B2BBF810704A
:102CF000DFB10026DFF82CA1B446AAFB0732D208C8
:102D000002EB8203A7EB43035FFA86F938469BB2D6
:102D10004FEA890903FA09F3092897B24CEA030C30
:102D200006F10106E9D81FFA8CF7BBF812303D4ACC
:102D3000A2FB0306F608632E28BF6326092B63D97E
:102D4000002093468146ABFB0632D20802EB820399
:102D5000A6EB43035FFA80FAB4469BB24FEA8A0AB5
:102D600003FA0AF3BCF1090F96B249EA030900F12C
:102D70000100E8D85FFA89F9009B019A002BCCBFCB
:102D8000392338231616BEF1000F26F07F0635DDF5
:102D9000274A3343964543F00206C8BF43F0060670
:102DA000D8F800301622581CC8F800001A70D8F85D
:102DB00000300022581CC8F800001A7040463FF04E
:102DC000CDFE214640463FF0B1FE294640463FF049
:102DD000ADFE404639463FF0C1FED8F800305A1CDF
:102DE000C8F8002083F80090D8F800305A1CC8F8C2
:102DF000002001201E7003B0BDE8F08F1E43CFE716
:102E0000002003B0BDE8F08F4FF00009B4E700BF29
:102E10005859002038A700206BCA5F6B806967FF94
:102E2000D34D6210CDCCCCCCC55A7C0AA086010013
:102E3000FFC99A3B905A00202DE9F047AB4B1B6825
:102E4000064613F0800084B000F09E80A84B93F8F3
:102E5000E00710F0020000F09780A64F397D0529A9
:102E600040F29780632900F292800024DFF898C234
:102E700089B22546ACFB0132D20802EB8203A1EBFA
:102E80004303E0B28E469BB280008340BEF1090F3F
:102E900091B245EA030504F10104EBD8EDB2BB6839
:102EA000954A82FB0312D917C1EB623189B200291E
:102EB00000F018814FF0000CDFF84CE26446AEFBE6
:102EC0000132D20802EB8203A1EB43035FFA8CF0DC
:102ED00088469BB280008340B8F1090F91B244EA62
:102EE00003040CF1010CEAD8E4B2FB8983494FF4E6
:102EF000F36707FB03F7A1FB0737C7F38F1742F20E
:102F00000F739F4249D8CFB10020DFF8FCE184461F
:102F1000AEFB0732D20802EB8203A7EB4303C1B238
:102F2000B8469BB289008B40B8F1090F97B24CEAC2
:102F3000030C00F10100EBD81FFA8CF7704BD3E9BA
:102F4000002313433ED14FF0FF3833681722591C3A
:102F500031601A7033680022581C306039461A708C
:102F600030463FF0FBFD414630463FF0DFFD336821
:102F70005A1C32601D7033685A1C326030461C7017
:102F80000621FAF789FC012004B0BDE8F0879925F5
:102F900085E7002004B0BDE8F0870021DFF868C1B4
:102FA0000F46ACFB0302D20802EB8200A3EB400306
:102FB0009BB28B400431102947EA030793B2F0D14A
:102FC000BFB2BBE701A844F0CDFD9DF80810002971
:102FD00000F08A804FF0000CDFF82CE1E046AEFBF9
:102FE0000132D20802EB8203A1EB43035FFA8CF0BB
:102FF00089469BB280008340B9F1090F91B248EA3B
:1030000003080CF1010CEAD84FEA08289DF80910D2
:10301000E1B10020DFF8F0E08446AEFB0132D208D7
:1030200002EB8203A1EB43035FFA80F98A469BB26D
:103030004FEA890903FA09F3BAF1090F91B24CEA90
:10304000030C00F10100E8D848EA0C089DF80A10CA
:103050004FEA0828E1B10020DFF8ACE08446AEFB7F
:103060000132D20802EB8203A1EB43035FFA80F93D
:103070008A469BB24FEA890903FA09F3BAF1090FAC
:1030800091B24CEA030C00F10100E8D848EA0C08C0
:10309000BDF80C301B49632BA1FB03214FEA081834
:1030A0004FEA51117FF651AF0020DFF85CE0844613
:1030B000AEFB0132D20802EB8203A1EB43035FFABD
:1030C00080F98A469BB24FEA890903FA09F3BAF1FB
:1030D000090F91B24CEA030C00F10100E8D848EA6C
:1030E0000C0832E70C4600E788468FE75859002065
:1030F00038A70020905A002089B5F814D34D6210EB
:1031000008B000201F85EB51CDCCCCCC08B5A0F188
:103110000103B3FA83F302284FEA531301D0184690
:1031200008BD0F2021F07AF930B9064B93F88A37A1
:1031300003F00103184608BDBDE808400F2021F048
:10314000F5B900BF38A7002010B5084CE26D13890F
:103150009907FCD513891B06F9D40A2036F0C8FB61
:10316000206EBDE810403AF0F7B900BF201C0020E7
:10317000014B1B681B6A184748520020024B186815
:1031800008B183691847704748520020024B1868FD
:1031900008B14369184770474852002010B5074CE2
:1031A000606D40B13BF050FA94F8513013B180F0AB
:1031B0000100C0B210BD012010BD00BF201C0020C6
:1031C00010B5FFF7EBFF0E4C48B194F82430032BF9
:1031D00010D8237E0133DBB2072B237603D90023DB
:1031E00084F8243010BD074A01231268626184F814
:1031F000243010BDE06D4FF4807154F069FFE8E7B2
:10320000201C0020C024002030B40A490A480A7853
:10321000531CDBB20525042B00EBC20400F832502E
:1032200008BF00234FF404520B7062604FF0FF3070
:1032300030BC7047B05B0020B45B0020037870B4F2
:10324000FBB10446C0F10106A31914F8015FDBB21B
:10325000002DF9D101335B00DCB2032513800C7023
:103260004D7004785CB1022300255A1CD2B2CC54B4
:103270008D5410F8014F0233DBB2002CF5D170BC35
:10328000704702242346E8E70B0617D401EB8103BD
:1032900000EBC30310B400EB81000124002283F88B
:1032A000764383F8741383F87523426D5DF8044BFD
:1032B000136843F4001300201360704701F07F018E
:1032C00001EB810300EBC303012200EB810083F8D3
:1032D0001C1183F81E2183F81D2182691368002BBD
:1032E00001DA43F0804343F4001313600020704779
:1032F00070B501F07F0505EB850400EBC4042821BF
:1033000001FB05010126C4F830310023C4E94A223B
:1033100084F81C5184F81D61C4F8343101F58E71B4
:103320001DB9FDF779FF002070BDFDF7E9FF002012
:1033300070BD00BF2249F8B5D1F8D8380F2B04D0A2
:103340005A1CC1F8D8280020F8BD1E4C257800234F
:10335000C1F8D838002DF6D11B4E1C4B3268B2F59F
:10336000006F17D01B689A4227D017D9C2F50063A7
:10337000402B15D9403B02F14005C1F8DC38012350
:103380002370356092B2402311490A448121FFF72E
:10339000AFFFD8E71B6835607BB12A469B1AE7E789
:1033A0004FF0000502EB0307C1F8DC580CBF022107
:1033B0000121376092B22170E6E700232370C2E753
:1033C00038A7002030290020982400209C240020C9
:1033D00034290020AEE700BFF8B51D4C2378012B3F
:1033E00003D0022B09D00020F8BD01461948D0F8BF
:1033F000DC3853B923700020F8BD00231A46812120
:10340000FFF776FF00232370F5E7402B11D9124C0C
:103410002268403B02F14005C0F8DC38256092B2DA
:1034200040230E4C084622448121FFF761FF002013
:10343000F8BD094D2A684FF0000603EB0207C0F8FB
:10344000DC6808BF02202F6092B208BF2070E8E756
:103450003029002038A7002098240020342900209B
:1034600038B5134602250A46C0E94E3380F811519B
:103470000021FFF73DFF002038BD00BF10B50C78DC
:1034800014F0600413D0202C0AD14B78023B092B96
:1034900018D8DFE803F01B21171717171717272E67
:1034A00022490122FFF7DCFF0024204610BD4B78A3
:1034B000062B24D00A2BF3D01D4B8A78C3F8E828BA
:1034C000204610BDFBF74EF80224EEE71949012211
:1034D000FFF7C6FF0024E8E717490122FFF7C0FF06
:1034E0000024E2E74B88124A1B0AC2F8E4380024A1
:1034F000DBE70F4B8A78C3F8E0280024D5E74B8838
:103500001B0A222B0CD0212B04D021462246FFF788
:10351000A7FFCAE7CA880949092A28BF0922F6E78E
:10352000CA880749362A28BF3622F0E720B0002093
:1035300038A700201CB0002018B000208A05002009
:103540004005002038B501EB810400EBC4040D46B2
:10355000002184F87453C4F88C1384F87513C4F8EC
:103560008833C4F88023C3782821012B01FB05018F
:1035700008BFEDB201F55D7108BFC4F884231DB921
:10358000FDF74AFE002038BDFDF7BAFE002038BD29
:10359000144B9A6870B5044662B1134A1B7B92F8CB
:1035A000EC582B4316D081212046FFF76DFE022DEB
:1035B00009D070BD0C4B93F8EC5881212046FFF7E1
:1035C00063FE022DF5D12046064ABDE870401F2358
:1035D0000121B7E70121FFF757FE20468121BDE811
:1035E000704051E6905B002038A7002070B5094A72
:1035F000094D1173094B13600021044629700D23F6
:103600008121FFF775FE2046054ABDE870401F2363
:10361000012197E7F05B0020E45B00205553425303
:10362000905B002010B5064B597B0446FAF7A8FFC3
:10363000002800DB10BD20460121BDE81040D5E781
:10364000905B00202DE9F041314D2C7834B1012CF4
:1036500001D1FFF7E7FF0020BDE8F0812D4FDFF833
:10366000D080B0F8B4337A68C8F804201F2BBA6849
:10367000C8F80820064606D1274B3A689A4202D17C
:10368000797B01291AD9254A25491378052401F89F
:10369000334001EBC3000133DBB2042B08BF00232E
:1036A0004FF4005113701F4B41600222304683F8E3
:1036B000EC28FFF76DFF0020BDE8F081BB7B013BEC
:1036C0000F2BE0D8FAF75CFF002819DB2B78013BC1
:1036D000022BC0D9144B1988B1B1BB68D8F80820A7
:1036E00088F80C408B4228BF0B46D11A0424C8F836
:1036F00008100E4A2C7030468121FFF7F9FDAAE729
:103700003046FFF745FFA6E73046FFF76FFFA2E719
:10371000E45B0020905B002055534243B05B0020E7
:10372000B45B002038A70020D85B0020E07E00209A
:10373000F05B002008B5084B1B78022B07D0033B39
:10374000012B02D80021FFF751FF002008BDFFF731
:1037500069FF002008BD00BFE45B002010B501EB4D
:103760008101084A00EBC1010446B1F88C131046F0
:10377000F4F740FD034A204640230121FFF7E2FE13
:10378000002010BD28B00020E8E700BF70B50A781F
:1037900012F060050C46064611D0202D16D1CD88BA
:1037A000D5B113062AD52A461F496078F4F74CFD97
:1037B000E2881D493046FFF753FE00250AE04B78AA
:1037C0000A2B16D00B2B0ED0062B03D13046FAF75E
:1037D000C9FE0225284670BD022260781144F4F724
:1037E00033FD284670BD8B78D3B9104BC3F83059E0
:1037F000F0E70F490122FFF733FEEBE70D4964784C
:103800000A4AC1F8C8400321C0E9E45542F8045B04
:103810002B4680F811110021FFF794FE0025D9E70F
:10382000FAF7A0FED6E700BF3CA7002038A700208B
:1038300068B00020540400200B7803F00303012B30
:1038400003D0022B04D0002070478B881BB915E6EB
:103850008B88832BFBD099E710B5022304464022C6
:103860008121FDF755FC2046022340220121FDF76E
:103870004FFC8221204603230822FDF749FC064B1A
:1038800002229A80F4F72EFD044A204640230121AB
:10389000FFF758FE002010BDA001002028B0002036
:1038A00038B509220D46044603238321FDF730FC79
:1038B00029462046FFF7D0FF002038BD82B0002304
:1038C000016801930B6901930E4B03E00A690192B1
:1038D000013B13D0019A002AF8DA019A094B42F011
:1038E00001020192019A0A610A69019203E00A69E0
:1038F0000192013B02D0019AD207F8D4002002B015
:10390000704700BF400D0300436D064A1A61C2783C
:10391000012A06D100F2CC5058614FF0802219687C
:103920001A6070471800086010B50023042204468E
:10393000194680F811211A46FFF7DAFC2046FFF7F6
:10394000E3FF002010BD00BF10B5044629B990F870
:103950001131032B0DD0002010BDD0F8E4359B6948
:10396000002BF8D090F81221032AF4D198470020B8
:1039700010BDD0F89013D0F87C33994214D9C07898
:10398000D4F880230128A1EB030104BFD218C4F8A6
:1039900080238B4228BF0B46C4F890139BB220466D
:1039A0000021FFF7CFFDD6E7D0F8E4351B691BB146
:1039B00090F81221032A03D02046FFF7B5FFCAE78B
:1039C0009847F9E7F0B5012190F8D17590F8D365E3
:1039D00090F8CFC590F8CE5590F8D03590F8D22514
:1039E00080F8111190F8CC1585B005EB0C2503EB90
:1039F000072302EB062201F01F06AFB292B290F845
:103A0000CD558DF808109BB2012E0446ADF80A7012
:103A1000ADF80C30ADF80E20C0F840218DF80950FB
:103A200017D0022E1FD036B101F08001FFF72CFC19
:103A3000002005B0F0BD092D0FD8DFE815F0BF005C
:103A4000AC000E00D5000E00EA0085000E007700E5
:103A5000540090F81221032A2FD02046FAF782FD55
:103A6000002005B0F0BD01F060012029DAB234D0A9
:103A7000012D00F02081032D00F00681002DD7D10B
:103A800090F81211022900F0DF800329E5D11B060E
:103A900000F14B8102EB820200EBC20393F8763314
:103AA000002B00F04D81BF4B0122C3F84429BE49D1
:103AB00020460222FFF7D4FCBAE7DAB2012ACCD8BA
:103AC000D0F8E43502A99B689847BDF80E30002B6A
:103AD000AED12046FFF728FFAAE7D0F8E43502A9C7
:103AE0009B689847A4E7F9B2AE4D012985F83419CF
:103AF000B3D890F81231022B00F02781032BACD100
:103B0000002900F0868190F810110129E1D0D0F849
:103B1000E4355B68984795F8341984F8101120460D
:103B2000FDF764FA2046FFF7FFFE81E7012A94D1F2
:103B300090F81231022B00F01781032B8DD100F584
:103B40008871FFF78DFC73E73D0A022DADF8062062
:103B500000F05081032D00F00B81012D7FF47DAF2B
:103B6000D0F8EC3580781B680DF106019847BDF858
:103B70000620002A3FF45CAFBDF80E30002B3FF466
:103B800057AF9A4228BF1A4601462046ADF8062094
:103B9000FFF766FC4CE790F81231023B012B3FF631
:103BA0005CAF012F7FF444AFD0F8E43500229B686E
:103BB000C0F8182102A9204698478AE790F81231E8
:103BC000023B012B3FF649AF764BD0F8182100217C
:103BD000C3F83C1912B10222C3F83C2973492046AC
:103BE0000222FFF73DFC23E7012F00F09880022F0F
:103BF0007FF41EAF13F0FF0F7FF41AAF02691B0AA8
:103C0000023B5268032B00F21D81DFE803F03935D7
:103C100031241A437FF421AF90F81231032B3FF483
:103C20001CAF036907F07F0580F81451196867F32A
:103C30000A120A431A60FFF777FE002D00F0E580B4
:103C4000022384F81231F3E651063FF4F1AE114637
:103C5000FFF71AFBECE6052363F30612514B012133
:103C600084F816112046C3F84029FFF75DFEDFE611
:103C7000042363F30612F1E7032363F30612EDE76F
:103C8000022363F30612E9E790F81231022BDBD02E
:103C9000032B7FF4E2AE27B9550602D01146FFF799
:103CA000F3FAD4F8E43502A99B68204698472046E9
:103CB000FFF73AFEBCE690F812110229C4D003299E
:103CC0007FF4CBAE002F7FF4B3AE12F07F013FF450
:103CD00000AF180600F1A78002EB820304EBC303D8
:103CE00004EB810083F8767383F8741383F875739B
:103CF000282303FB0243416D03F55D73DA780B68FB
:103D0000023A6FF35553012AD4F8E42598BF43F0E3
:103D100080530B602046936802A99847D9E6D0F8F3
:103D2000E435C0F818719B6844E702F07F0202EBAB
:103D3000820200EBC20393F81E31002B7FF4B3AE76
:103D4000184B0022C3F84429B1E600293FF4C1AE64
:103D50000121032380F8101180F81231FDF746F994
:103D60002046FFF7E1FD63E61149FFF779FB5FE6C7
:103D7000FDB2052D3FF671AEDFE805F0342C241CB2
:103D80000B03D0F8EC3580789B690DF1060198475C
:103D9000EDE6D0F8EC3580785B690DF106019847C7
:103DA000E5E600BF38A700207CB0002074B00020FA
:103DB00070B00020D0F8EC3580781B690DF1060159
:103DC0009847D4E6D0F8EC358078DB680DF1060131
:103DD0009847CCE6D0F8EC3580789B680DF1060169
:103DE0009847C4E6D0F8EC3580785B680DF10601A1
:103DF0009847BCE6D0F8E43580789B6A0DF106015F
:103E000098474570C4F8F005B1E6012384F81231F3
:103E10000EE60222D0F8E43580F8101180F8122165
:103E20005B68984755E6282202FB014304EB8100BA
:103E300083F81E7183F81C1183F81D51816903F505
:103E40008E735BE7012363F3061207E770B5044640
:103E500049B990F81131022B1BD094F81631012B7F
:103E60000DD0002070BDD0F8E4355B69002BF8D090
:103E700090F81221032AF4D19847002070BD2A4AF5
:103E80002369D2F840295A60002384F816310020B3
:103E900070BDD0F83831D0F82451AB4217D9C27870
:103EA000012AD0F82821A3EB050308BF5219C0F856
:103EB000383108BFC0F828219BB20021FFF718FA5B
:103EC00000231A4619462046FFF73CFBC5E7D0F809
:103ED0003C31B3FBF5F605FB163666B99D420AD8B0
:103EE000D0F84021934206D233463246FFF700FA1B
:103EF000C4F84061E4E7D4F8E435DB681BB194F81A
:103F00001221032A0CD00023052284F8112119461E
:103F10001A462046FFF716FB2046FFF7F5FC9CE704
:103F200020469847EFE700BF38A7002082B0002363
:103F30000193019A094B42F010020192C168019A63
:103F40000A610A69019203E00A690192013B02D009
:103F5000019AD206F8D4002002B07047400D030049
:103F600082B000230193019A0B4B42F02002019290
:103F7000019A61F38A120192C168019A0A610A6981
:103F8000019203E00A690192013B02D0019A920674
:103F9000F8D4002002B07047400D0300F8B50B784C
:103FA00013F060050C4606461CD0202D17D14A7828
:103FB000FE2A44D0FF2A3DD14A88002A56D1CD8816
:103FC000002D53D11B0651D43749384B0D700121B8
:103FD00083F8EC18364A1F23FFF7B4FA00E00025F7
:103FE0002846F8BD4B780A2B4BD00B2B44D0012B25
:103FF000F6D191F904308988002B47DBFFF796FF53
:1040000021792A4F3046FDF71FF8022321794022FB
:104010003046FDF77DF897F8EC38022B3BD094F949
:104020000420002ADCDA012BDAD030460121FFF728
:10403000DDFAD5E70225FAF795FA2846F8BD4D884E
:10404000A5B9CC88012C11D11A060FD5194B1B68C4
:104050009B6998471549C0B281F8480930B122469A
:1040600001F648113046FFF7FBF9B9E73046022563
:10407000FAF778FA2846F8BD0C4B4A8883F84929A4
:10408000AEE70D490122FFF7EBF9A9E701F07F0147
:10409000FFF766FFB4E730468121FFF7F5F800230C
:1040A00087F8EC389CE700BFE45B002038A70020CD
:1040B000905B0020D45B002081B0002038B504461E
:1040C000FCF7F8FF2046022340228121FDF720F86B
:1040D0002046022340220121FDF71AF80C4B0D491E
:1040E0001B680D4A00250D701B6882F8EC582846A5
:1040F00098472046FFF71AFF20460121FFF730FFBF
:10410000064A20461F230121FFF71CFA284638BD26
:10411000D45B0020E45B002038A70020905B0020E7
:10412000012905D008B50321FFF71AFF002008BDBB
:10413000FFF752B9104B70B4DA684378017886788B
:104140000E4CD243C2F30222C2F10405E8B283400E
:104150000F2040FA02F23240DBB2134360181B0119
:1041600001F01F0501224909DBB2AA4080F80033A3
:1041700044F8212070BC704700ED00E000E100E051
:10418000C27802B1D6E7037805485A09203203F015
:104190001F03012101FA03F340F82230704700BFEA
:1041A00000E100E000B583B009238DF80730FDF78A
:1041B0005FF98DF807009DF80730012BF7D09DF8C7
:1041C000070003B05DF804FB82B0064B00220192A9
:1041D0000193019B03EB80000190019B186802B0E2
:1041E000704700BF5028004082B0064B0022019269
:1041F0000193019B03EB80000190019B196002B0C9
:10420000704700BF502800400023C0E90033C0E9D8
:104210000233C0E90433C0E90633C0E90833C0E91A
:104220000A33C0E90C338363704700BF0B6870B476
:10423000D1E90524CD682B431343D1E90725234356
:104240001343D1E909422B43D1E90D6523431343BD
:1042500004680B4A334322402B4313430360D1E9E4
:104260000B3442690D6922F0070223431343D1E95D
:10427000014243614560846070BCC260704700BF0A
:104280003F801CF002683649002310B422F001027E
:10429000212488420260036043608360C36003613D
:1042A000446138D02F4B98422ED02F4B98423CD0AF
:1042B0002E4B984240D02E4B984232D02D4B9842F4
:1042C00041D02D4B984246D02C4B984217D02C4BC6
:1042D00098423CD02B4B984216D02B4B984224D07E
:1042E0002A4B984228D02A4B98421AD0294B984200
:1042F00029D0294B98422ED0284B984208D14FF014
:104300003D5243F8AC2C03E04FF4746243F8202C88
:104310005DF8044B7047224B5DF8044B3D229A60D8
:104320007047204A43F8642CF2E74FF474125DF8AA
:10433000044B43F8382C70474FF074625DF8044B1F
:1043400043F8502C7047184A43F87C2CE0E73D2294
:1043500043F8082CDCE7154A43F8942CD8E700BF53
:1043600010600240286002404060024058600240F5
:104370007060024088600240A0600240B860024065
:1043800010640240286402404064024058640240C5
:104390007064024088640240A0640240B864024035
:1043A000006002403D000020400F002000003D2042
:1043B0000B88F0B433BB028C4C880E898B88C9887B
:1043C00022F001021204120C0284058B028CADB2A1
:1043D00025F0F30592B22B4322F00A0243EA0613BA
:1043E00022439BB242F0010203830284038B23F039
:1043F0000C031B041B0C0383038B9BB21943F0BCFF
:1044000001837047042B048C2CD0082B4E888A889B
:104410000D89C98851D024F480542404240C0484C8
:10442000838B078C2C0344EA022440F6FF421A4097
:1044300045F6FF733B4043EA063322439BB292B2F8
:1044400043F4805382830384828B22F440621204FB
:10445000120C8283838B9BB243EA01239BB2F0BC94
:104460008383704724F010042404240C4D880F89A2
:104470008A88C9880484068B038C12029BB242EAA4
:10448000073423F0A00340F6FF42324043EA05130D
:1044900022439BB292B243F0100302830384028B47
:1044A00022F440621204120C0283038B9BB243EA93
:1044B00001239BB2F0BC0383704724F4807424046E
:1044C000240C0484848B038CA4B29BB224F0F304E8
:1044D00023F42063224343EA062342EA05129BB2F7
:1044E00043F4807392B282830384838B23F00C03A2
:1044F0001B041B0C8383838B9BB21943F0BC818309
:10450000704700BF214A038890429BB212D002F547
:10451000806290420ED0B0F1804F0BD0A2F5803275
:10452000904207D002F58062904203D002F580628B
:10453000904203D14A8823F070031343144A9042F7
:1045400018D002F58062904214D030B423F4407346
:104550000C894D6802F56C429BB2234390420C8853
:104560000380C56204850DD18B7A0386012330BC9C
:104570008382704703800B884A68C26203850123E7
:1045800083827047034B9842EED0EFE70000014072
:104590000010004000040140024A536A23EA000070
:1045A0005062704700380240024A136A23EA000052
:1045B0001062704700380240484B98422ED0B0F14C
:1045C000804F32D0464B984236D0464B98421ED050
:1045D000454B984237D0454B98423BD0444B98428C
:1045E0003FD0444B98424BD0434B984240D0434B32
:1045F00098424CD0424B984251D0424B984256D0B0
:10460000414B98425AD0414B98425ED07047404A45
:10461000136A43F0040313620420C5E73C4A536A5B
:1046200043F0010353620120B6E7394A136A43F0AD
:10463000010313620120B7E7354A136A43F002030E
:1046400013620220B0E7324A136A43F00803136290
:104650000820A9E72E4A136A43F0100313621020C2
:10466000A2E72B4A136A43F02003136220209BE742
:10467000274A536A43F4803353624FF480308BE708
:10468000234A536A43F002035362022084E7204A1C
:10469000536A43F4003353624FF400307CE71C4A02
:1046A000536A43F4802353624FF4802074E7184A1E
:1046B000136A43F040031362402075E7144A136AFB
:1046C00043F08003136280206EE7114A136A43F4BB
:1046D000807313624FF4807066E700BF00000140F2
:1046E0000004004000080040000C004000100040A2
:1046F000001400400004014000400140004401401B
:104700000048014000180040001C0040002000400C
:1047100000380240224A936803F00C03042B10B4C3
:1047200021D0082B22D01F4B03601D4C1E4AA168CC
:10473000C1F30311114491F84811CB404360A168C3
:10474000C1F38221114491F8481123FA01F18160EB
:10475000A1685DF8044BC1F342310A4492F8482144
:10476000D340C3607047114B0360DEE75468516863
:1047700052686302C2F388124CBF0C4B094B01F024
:104780003F01B3FBF1F303FB02F3054A5268C2F3A6
:10479000014201325200B3FBF2F30360C5E700BFF0
:1047A000003802400024F4005404002000127A0073
:1047B0002DE9F04700230F6801264FF0030C02E0BB
:1047C0000133102B41D006FA03F232EA0704F7D185
:1047D000D0F800E05C000CFA04F52EEA050EC0F8F3
:1047E00000E091F80490D0F800A009FA04FE09F165
:1047F000FF394EEA0A0EB9F1010FA846C0F800E0F1
:104800006FEA050515D8D0F808E005EA0E058560C1
:104810004D79D0F808E0A54045EA0E058560456869
:1048200025EA020242608A7945689A4092B22A4398
:104830004260C26822EA0802C260CA79C568A24022
:1048400001332A43102BC260BDD1BDE8F0870D4B68
:1048500093F88A27D20703D5012283F84A297047A3
:1048600093F84A2962B9D3F8D0274AB193F8802740
:10487000104493F8812783F88007114483F8811747
:10488000704700BF38A70020044B93F90C000128A3
:1048900006BF02221A730020704700BF38A700200D
:1048A000114AD2F84C09A0B1D2F850398BB18842E4
:1048B0000DD88B4234BF002301239BB11369C2F88A
:1048C000541999421CBF142382F85839DCE700239D
:1048D000F3E7A1F59C53083BB3F57A7F2CBF002387
:1048E0000123EAE7704700BF38A7002007B500237F
:1048F0000DF10602ADF806300AF0A4FE60B1084BD7
:10490000BDF80620998AA3F85A2991421CBF1422A7
:1049100083F85C29FFF7B8FF03B05DF804FB00BF24
:1049200038A7002013B50446262001911FF0FEFD94
:10493000019948B9054BD3F870372BB1204602B026
:10494000BDE81040FDF78FB902B010BD38A70020B8
:10495000B1FA81F149094920E4E72DE9F341BE4C60
:1049600094F90C3001330D4600F06681D4F87037AD
:10497000002B00F0B380022700264FF00108D4F886
:10498000700735F0CBFD002800F0A880D4F8700740
:1049900035F0BCFDD4F878375A1C2344C4F8782786
:1049A00083F85D0994F87437012B09D0022B15D0D8
:1049B00063B90F280CBF84F87487C4F87837DEE732
:1049C000A0F17203012B06D9762804D084F874670D
:1049D000C4F87867D3E784F87477D0E7102ACED18B
:1049E0009E490023012211F8010F013203440E2ACF
:1049F000DBB2F8D194F86B2984F874679A42C4F852
:104A00007867BCD194F86C39002BB8D194F85E3932
:104A1000732B59D0762B1BD0722B5FD194F8602961
:104A200094F85F3994F90C1053EA022356D0C4F875
:104A30004C390029B4F86139C4F850394EDC94F887
:104A40007A2901232373002A48D184F87A3945E072
:104A500094F8602994F85F3953EA02233ED0D4F8E1
:104A6000702994F8621994F86609236193421CBF77
:104A7000142284F8582994F86129C4F8703942EA5C
:104A80000122B4F87419A28291421CBF142184F847
:104A90005C1994F86319617394F86419A17394F81C
:104AA0006519A4F8742941EA0021A4F87619D4F80C
:104AB000541909B9C4F85439B4F85A390BB9A4F8DF
:104AC0005A290223237309E094F8642994F863397E
:104AD00043EA02231AB20BB1A4F8782994F90C30F6
:104AE000022B35D00FDCDAB2012A15D9636E13B16F
:104AF000A369002B6CD15A495A481F2202B0BDE865
:104B0000F04158F036BC032BF0D1D4F87C39564A2A
:104B1000EB1A9342EADD13E0D4F87C295349AA1A30
:104B20008A42E3DD2BB97220FDF7C8F8C4F87C593E
:104B3000DCE7D4F880395A1CD907C4F8802903D49B
:104B40007620FDF7BBF8F1E77320FDF7B7F8EDE746
:104B5000D4F85419D1B194F85839BBB123699942AA
:104B600014D0637BDA0703D489B24620FFF7DAFE5C
:104B700094F85839013B84F8583905F592250323F8
:104B800005F578752373C4F87C59AFE7B4F85A1962
:104B9000A38A81B194F85C296AB18B420BD0637B04
:104BA000DB0702D45020FFF7BDFE94F85C39013BCF
:104BB00084F85C39E1E701222273A4F85A392269AA
:104BC000C4F85429002384F85C3984F858398DE7F7
:104BD000274DD4F8D0772A2385F858310DF10702F4
:104BE00020230DF10601384685F859310AF0F2FD0F
:104BF00030B19DF806109DF8076051EA06031ED1FA
:104C0000552385F85A31462385F85B3122691948C6
:104C1000202385F85C31002A34D0174947F0D8FBAF
:104C2000B4F8763915488BB3A28A15499A420CBF5D
:104C300020222A2247F0CCFB02B0BDE8F0813846A2
:104C40000AF046FD314685F85A0138460AF02CFD37
:104C5000037885F85B31D9E738A7002095B00020AC
:104C600072870708AC050020400D030040420F008A
:104C700054040020B1050020EBC00708B505002052
:104C80008C870708034947F0A3FBC9E7024947F0AF
:104C90009FFBD1E7948707089387070810B50E4C50
:104CA00040F0080284F87B2194F9CC20022A06DD2A
:104CB000420704D583071CBF012384F8D4300521A3
:104CC0000648FCF7ADFC062184F87C01BDE81040E5
:104CD0000248FCF78DBC00BF54040020CB05002027
:104CE00010B5FCF735FCA8B31B4C94F9CC30012B64
:104CF00030DD59B3022B2DD094F8D4309BB971B16B
:104D000080230521154884F88131FCF789FC0621B0
:104D100084F88201BDE810401048FCF769BCBDE88A
:104D200010400420BAE7002914BF0020042094F8A2
:104D3000CF301A0748BF40F002005B0701D411B121
:104D400008B940F00100BDE81040A7E7022BD3D11D
:104D50000420ECE710BD00BF54040020D105002062
:104D6000F8B5224C04F28317030A84F8880105463B
:104D70000621384684F88731FCF752FC94F8CF308E
:104D800084F88901DB072AD4B4F8D020AA4226D1BE
:104D9000174DD4F88331C5F88439C3B285F88A3900
:104DA00041F26F714FF6FF738A4218BF012313441B
:104DB00005F68416C3F307220621304685F88829B4
:104DC00085F88939FCF72CFC072185F88A093046DB
:104DD000FCF70EFC052104F5C570FCF709FCBDE8E5
:104DE000F84004480721FCF703BC00BF540400202E
:104DF00038A70020D705002008B5FCF7A9FB48B16B
:104E0000A1F59C53083BB3F57A7F03D2BDE8084077
:104E10000846A5E708BD2DE9F0476B4E3368002B27
:104E20003AD06A4D6A4C05F1CC07306835F076FB14
:104E3000002833D1674B198809291D4609D95F8895
:104E400064227A43B2FBF1F2452A40F3A481188030
:104E5000588094F8C539012B00F0C881022B00F06E
:104E6000E38133B95C480521FCF7C2FB012384F8D8
:104E7000C5395A4B1D685A4B1B78002B00F0DE8158
:104E8000584B1B68EB1A782B40F2D881D4F8C40732
:104E9000F9F736FBC4F8C859BDE8F087306835F03B
:104EA00035FB94F88B398046052BBED8DFE803F03C
:104EB0000309171D3745AA28B7D1012384F88B3978
:104EC000B3E7552803D1022384F88B39ADE7414A73
:104ED000938801339380002384F88B39A5E703235B
:104EE00084F88C0984F88B399FE7132884F88D099E
:104EF000C4F8A80907DD374AD3880133D3800023DB
:104F000084F88B3991E718B9052384F88B398CE73D
:104F10000023C4F8AC39042384F88B3985E7D4F82E
:104F2000AC39E218013382F88E09D4F8A829C4F804
:104F3000AC3993427FF479AFE6E7D4F8A8392A4830
:104F400003F1020A4FFA8AF1FCF76AFB804594F8F4
:104F50008C9940F0178126201FF0E8FA204B48B1C9
:104F600000221A701B4A538801335380002384F8AF
:104F70008B395AE71A784A4519D100221A7009F17B
:104F8000FF33102B00F2F980DFE813F030008E00C1
:104F90008E00E1008E00F700F700F7003000F70008
:104FA000F700F700F700F700F700F7003000B9F15D
:104FB000090F02D0B9F1110F01D1012ADDD0054A44
:104FC000538901335381DAE7545B002054040020F5
:104FD00038A70020785B0020DE050020C0240020D8
:104FE000865B0020885B0020C4B00020BAF1060F69
:104FF0005ADDB9F1010F06D0B9F1090F0CBF4FF01E
:1050000002094FF0030994F8910994F8921994F861
:10501000902994F98EE994F990C994F88F3985F81C
:10502000CC9041EA002109B2900785F8CDE085F8DF
:10503000CFC0A5F8D01006D512F00C0F14BF012276
:10504000002285F8D420B9F1030F13D1BAF1090F6A
:105050002ADD94F99429082AA8BF082222EAE272DC
:1050600085F8E320002043B29A4200F101005CDCA5
:1050700094F89339D4F818A0002002469BB2524508
:1050800090465ADB7D4B85F8CE001B78232B0BD145
:1050900009EB89037A4A03EB83030CEB8303138048
:1050A000A2F802E09180D080764977480A2258F031
:1050B000FAF810B1002384F8BA39724B3A681A60D2
:1050C0007A685A603A891A8194F8BA3943BB95F8DC
:1050D000D43094F8802784F8BC29002B14BF022315
:1050E000012384F8BA3995F8CF3094F8820784F810
:1050F000C00913F001031CBFB2FA82F35B0994F8F4
:10510000812784F8BD29D9B2B4F8842784F8BB1963
:10511000A4F8BE2913B10AB1A4F8C22984F8C419AD
:105120000EF084FE0EF082FE1CE704EB43082344DD
:1051300093F89639A8F8B43795E704EB480801329C
:10514000B8F81C8052B2984508BF104697E7BAF1EC
:10515000040FA9DD94F88E2994F88F3943EA0223CD
:1051600059041AB204D5C3F30D03A5F8D2309BE756
:10517000002AF8DBA5F8D03096E7444A938901333A
:105180009381EFE619F0010F7FF4F0AE3F4A1389E7
:1051900001331381EAE63E4BD3F89021B3F8941122
:1051A000012A1AD141F25632914203D14FF0FF3217
:1051B000C3F89021D3F89021306802EB820202EB11
:1051C000820201EB420189B2A3F8941103681B69C2
:1051D000984700232B806B803BE60132EAD1B1F582
:1051E000965F04BF0122C3F89021E3E7284D95F9AB
:1051F000CC60002E3FF43DAE022E11D14FF4804022
:10520000FFF7AEFD84F8C56995F9CC30012B7FF727
:1052100030AE95F8CF30C3F3400385F8D43028E69C
:10522000032384F8C539EFE7194BB3F8D230002BCC
:105230003FF41FAE032384F8C5391AE694F83020F2
:1052400094F831309A4204D0FCF73CFEC4F8C859B7
:1052500022E6D4F8C839EB1AB3F57A7FBFF41CAE56
:105260000C4B1B68ED1A952D7FF616AE0A480521EA
:10527000FCF7BEF9BDE8F047FCF724BE99280020F2
:105280009C280020E8B0002020050020785B00204A
:1052900054040020885B0020DE05002010B5134C6C
:1052A000D4F8D00700B394F8801759B194F8812747
:1052B0000AF0DCF9B4F8843783421ABFA4F88407F3
:1052C00001210021B4F8862762B141F2883393426C
:1052D000B8BF13469A4205D0A4F88637BDE81040FF
:1052E00043F084B80029F9D110BD00BF38A70020D1
:1052F00010B401440446002014F8013B0822584031
:10530000430010F0800F08BF400083F0070314BF74
:10531000D8B2C0B2013AF3D18C42EDD15DF8044B62
:10532000704700BF30B54FF4806085B02DF0F4FCBD
:1053300040B3154C90F9040094F8CC39134A002B73
:1053400018BF08234FF4E1310125CDE90153009145
:1053500000234FF480612DF040FDFF2320670038CB
:1053600018BF012084F8EC3484F8FC3484F80C3540
:1053700084F81C3584F82C3584F83C3584F84C3599
:1053800084F85C3505B030BD38A700201919010834
:10539000374B1B6813F000635CD02DE9F04F354BA1
:1053A0001F78B84251D3FF2856D1334B93F8DC30E5
:1053B000002B47D0DFF8D4A00022CAF8D029CAF8C1
:1053C000D429CAF8D829AAF8DC29002F4CD00AF22F
:1053D000EC431046144611461546164603EB071BD0
:1053E000B946B3F802C09F8993F8008093F901E0B1
:1053F00061443A444645D3E901C738BF46461033B5
:105400007545B8BF75469B4509B212B2644438442D
:10541000E7D191FBF9F192FBF9F28AF8D0698AF8A9
:10542000D159CAF8D449CAF8D809144BAAF8D219E4
:105430001B781149AAF8DC29092B4FF0000281F8EA
:10544000DC200CD00E48BDE8F08F0E4A02EB0010B5
:10545000BDE8F08F184670470020BDE8F08F0A4B7A
:105460009AF8D029DA80EDE73A463946DDE700BF01
:1054700058590020C40B0010540400209928002023
:1054800008B1002024AC00209C28002038A7002070
:105490000268F8B53A4E3B4CB6F9E039511C016050
:1054A0007E2111700168054603EBC30384FB0302F0
:1054B000481CDC17002328600B70FF20C4EB62043B
:1054C000FFF766FF2034304BA4B200284DD01B7884
:1054D000B0F90C102BBB2D4BA1F57A729A4246D82D
:1054E0002B48B0FBF1F189B228463DF011FB96F84C
:1054F0004737B6F8E41783B196F8EC37B1FBF3F110
:1055000028463DF005FB214628463DF001FB284694
:105510000821F8F7C1F90120F8BD28463DF0F8FA56
:10552000F1E71C4B1F78002FD5D01B48002300EB60
:10553000830201339289BB421144F8DB174B9FED84
:10554000186A9B7E07EE103A07EE901AB8EEC77AFB
:10555000F8EE676AC6EE077A67EEA67AFCEEE77A9F
:1055600017EE901AB1FBF7F1B5E71B7813B94EF6B9
:105570009C21B9E7074B1F78002FF8D00146D4E7EC
:1055800038A70020676666666009001017839303DA
:1055900000879303C40B00102C0C00103431002042
:1055A000000048432DE9F8434A4C427894F8E23928
:1055B00002F00F05C3B9EDB92B46002184F8E419B8
:1055C000EB1AD9B20E290BD8234493F8481739B1F6
:1055D00002F0F002802A4AD0902A5FD0A02A0DD093
:1055E00000273846BDE8F8830021AB4284F8E4196F
:1055F000F6D8E5E784F8E2592B46DEE7412966D084
:1056000081F08003042B62D90846FCF79DF9031D45
:105610000246DBB2304884F8E43965F05F0584F86F
:10562000E559FCF785FE94F8E479002FD8D0BE1E2A
:1056300016F0FF0024D1FF25A946022756B1DFF856
:105640009C80464418F8011BD4F8080A34F06AFF1D
:105650004645F7D1D4F8080A494634F063FFD4F838
:10566000080A294634F05EFF3846BDE8F88365F045
:105670007F050427022684F8E55984F8E47930464A
:10568000164A4FF6FF71104412F8015B491B904215
:1056900089B2F9D15FFA81F90D0ACFE7412914D017
:1056A00081F08003042B10D90846FCF74DF965F012
:1056B0006F050627042684F8E70984F8E55984F87D
:1056C000E61984F8E4793046DAE70420EFE70823A6
:1056D00004229FE738A700201EB100201CB1002043
:1056E0002DE9F047C31DDFF8348182B003F4FC7369
:1056F00000AFD8F88865ADEB030DC7F800D032686D
:10570000D8F8803568449A420C4698F80C3A78608C
:105710006D4658D0591C0DF1010203F00F0388F8B3
:105720000C1A8DF800303A60A0EB0209D6E900129D
:105730005FFA89F9521A09F107035FFA82FA03F452
:10574000FC73CA45ADEB030D55D25246684657F07F
:1057500071FD3368534433605246694638463DF024
:10576000B5F9D8F88825D8F880353068117A706096
:10577000C21A4A40D2B28342336088F80D2A09D057
:105780000133336013F8011C984282EA0102F7D119
:1057900088F80D2A3B68591C39601A70D7E9003225
:1057A000D21A012A08DD00215A1C3A601970D7E983
:1057B0000032D21A012AF7DC2846A0470020083719
:1057C000BD46BDE8F087B6F90C20591C03F00F0365
:1057D00043F01003002A2A46B8BF43F0200302F822
:1057E000023B88F80C1A691C3960D6E900135B1A71
:1057F0003A606B7098E74A46684657F01BFD33687D
:105800004B4433604A46694638463DF05FF92846C6
:10581000A04701200837BD46BDE8F08738A7002023
:105820002DE9F04F7C4C83B0D4F88855D5E900536E
:105830005B1B002B00AF83460D4616462ADD002376
:1058400084F80E3AFCF7F6F800200BEB05030BF199
:10585000010AC4F87835C4F874A59BF80050D4F850
:1058600084856909012940F09F8005F00F0915F032
:10587000100514D150B194F8102A013202F00F0231
:105880004A4500F09A8084F80E5A28460C37BD46E7
:10589000BDE8F08F94F80E0A0028D6D1D2E70BF1BC
:1058A0000203C4F874350BF103029BF80130D4F8FD
:1058B0007C05C4F874259BF80250C8F80000C21893
:1058C000C8F804206B404FF0000C84F80F3AD4F86D
:1058D00074A5D4F8783584F80E1AA8F80850A8F8FA
:1058E0000CC0A3EB0A03DDB2121AEB1D5FFA82FBB8
:1058F00003F4FC73AB45ADEB030D6BD25A46514636
:10590000684657F097FC0AEB0B035A464046694637
:10591000C4F874353DF0DAF8D4F87C35D8F80000D6
:1059200094F80F2A8342C8E900300AD00133C8F83E
:10593000003013F8011C984282EA0102F6D184F883
:105940000F2AD4F874351B78934239D1B8F908304E
:10595000FA2B54D0D8F80020D4F87C35D4F884152C
:10596000D4F83007C8E90032D4F88825D4F8803557
:1059700053600025158195813B1D84F80E5A7D608A
:105980002DF03AFE01303FD07B680BB100209847E4
:10599000D4F88835D4F88025196801200C37C3E97C
:1059A0000021BD46BDE8F08F00210846FCF726F82F
:1059B00001200C37BD46BDE8F08FD8E9000290E722
:1059C00000230120B8F9081084F80E3AFCF716F805
:1059D00001205BE72A465146684657F02BFC0AEB4C
:1059E000050340462A466946C4F874353DF06EF812
:1059F00000200C3784F8109ABD46BDE8F08F002EC9
:105A0000A8D005233370A5E7D4F8882513680221B0
:105A1000581C10601970B7E738A700200B4B93F89B
:105A20000A2812B1B3F858274AB9B3F93038084AEE
:105A3000D81782FB0323C0EBA30000B27047D3F852
:105A4000240890FBF2F000B2704700BF38A7002096
:105A500067666666F8B5184CC6B205463146D4F896
:105A6000140A34F05FFD94F8181AD4F8140AC5F338
:105A700007274E40394684F8186A34F053FD94F8ED
:105A8000181AD4F8140AC5F307464F40314684F873
:105A9000187A34F047FD94F8181AD4F8140A2D0E29
:105AA0004E40294684F8186A34F03CFD94F8181AE0
:105AB0004D4084F8185AF8BD38A7002070B50C4D39
:105AC000C6B231460446D5F8140A34F02BFD95F8D9
:105AD000181AD5F8140A240A4E40214685F8186A87
:105AE00034F020FD95F8181A4C4085F8184A70BD1E
:105AF00038A7002038B50B4C002305462421D4F8E4
:105B0000140A84F8183A34F00DFDD4F8140A54211C
:105B100034F008FDD4F8140A2946BDE8384034F0C2
:105B200001BD00BF38A700202DE9F047DFF858A3DA
:105B30002DED028B9AF8194A82B00F461646002CBA
:105B400000F0E781013C8AF8194ADFF840839FEDB5
:105B5000C88ADFF83C933B78002B00F090809AF8DD
:105B6000194A002C40F08B8036B133F061FF336866
:105B7000C01A002880F2DB839AF81A1A002940F034
:105B80007A839AF81B5A062D40F28481B94B93F818
:105B90009D0193F89C21824200F0AB81D3F89821BB
:105BA0009AF81C1A32F810400C440135013003F504
:105BB000CC73A4B2EDB2C0B2B4F5C06F8AF81B5A70
:105BC000587100F07E817CD8B4F5806F00F0298296
:105BD00024D8B4F5067F4FD8B4F5007F54D3A4F58C
:105BE0000073182B48D8DFE813F0E701DE01DE016F
:105BF000DE01DE01DE01DE01DE01DE0147004700DD
:105C000047004700470047004700C601AB01AB0112
:105C1000AB01AB01AB01AB01AB01AB01B4F5846FE0
:105C200000F0E68140F2E280B4F5A06F00F06482FB
:105C30006FF4A06C04EB0C03072B1DD8601EC0B2E0
:105C4000FFF7A6FBC0B1B0F90C308B4AADF80140AC
:105C5000917EDAF8342703EB830303EB83034908CF
:105C60009B0093FBF1F31021CDF803308DF8001069
:105C70006846904700233B70002E7FF46CAF02B063
:105C8000BDEC028BBDE8F087B4F5807F00F0FD81AC
:105C9000B4F5887FF0D1BAF93238CDF8033001225B
:105CA00010238DF800308DF801308DF80220DAF8DD
:105CB00034376846002498473C70002E7FF44BAF81
:105CC000DDE7B4F5046F00F0A48265D8B4F5006F89
:105CD00000F082821AD9B4F5026F00F0F181B4F5B8
:105CE000036FC9D19AF8E0379D07C5D5634BDAF841
:105CF0003427D9894FF4F36303FB01F3A8FB0313A3
:105D00005B091020CDF8033030218DE2B4F5E26F4D
:105D100000F03782B4F5E46F1FD1594B93ED180AA8
:105D2000D3ED027A20EE270A002420EE080A54F070
:105D30007DFF102320228DF800300723CDF80300CB
:105D40008DF802308DF80120DAF83437684698472C
:105D50003C70002E7FF4FFAE91E7B4F5E06F8BD17D
:105D6000474B93ED160AD3ED027A20EE270A002462
:105D700020EE080A54F05AFF10220723CDF8030042
:105D80008DF802308DF80020DAF834378DF80140B4
:105D9000684698473C70DCE740F678339C4248D828
:105DA000B4F5376F00F2E281B4F5116F00F0808135
:105DB000B4F5376F7FF460AFFF20FFF7E9FA0028F2
:105DC0003FF45AAF90F90130CDF803301021702222
:105DD0000B238DF802308DF80010DAF834378DF887
:105DE00001206846002498473C7066E740F2014372
:105DF0009C4200F02882B4F5826F7FF43DAFDAF860
:105E00007035980600F146821E4B1B681B0640F158
:105E100094820024102304228DF800308DF8013084
:105E20008DF803408DF804408DF805408DF806404C
:105E3000BBE145F230239C4200F0848145F24023CF
:105E40009C427FF419AFBAF92C38CDF803301021F9
:105E5000402252238DF802308DF80010DAF83437E2
:105E60008DF801206846002498473C7025E700BF64
:105E70000000C8425404002034310020905A002011
:105E8000C40B00105859002038A700201F85EB5183
:105E9000C5B3A2910135CA4BEDB293F8A52193F891
:105EA000A411914220D0501CC0B25200D3F8A011CE
:105EB000C44B8C5A8AF81B5AB4F5C06F58717FF4E2
:105EC00082AEDAF82438CDF80330102200240623FD
:105ED0008DF802308DF80020DAF834378DF8014063
:105EE000684698473C7034E7002283F8A5210120DA
:105EF000DCE7B5489AF81C2A007883F89D11013236
:105F0000D2B2013082428AF81C2A00F0B081012509
:105F1000C3E700283FF419AE0378303B012B3FF66E
:105F200014AE01300AF619220621FFF779FC9AF81F
:105F3000193A8AF81A0A002B3FF407AE3C7004E6BF
:105F4000A4F11100C0B2FFF723FA00283FF494AE89
:105F5000B0F90230CDF8033010238DF80030ADF8E1
:105F60000140DAF834376846984700233B70002E2A
:105F70007FF4F1AD83E69AF84727BAF8E437002AB0
:105F800040F0CF8110220221CDF803308DF800209F
:105F9000DAF834378DF801208DF8021068460024B5
:105FA00098473C7089E6601EC0B2FFF7F1F90028FF
:105FB0003FF462AE4368CDE7DAF81C388349DAF87B
:105FC000342781FB0301DB17C3EBA103002410215D
:105FD000CDF8033002238DF800108DF801408DF8C4
:105FE0000230684690473C70002E7FF4B4AD46E620
:105FF0009AF8E0379A077FF53FAEBAF8E237CDF866
:1060000003301021202204238DF802308DF8001077
:10601000DAF834378DF801206846002498473C7040
:106020004BE69AF8243A0133DAB2042A00F06E8182
:1060300042F210738AF8242A03FB02F3DAF8282AC2
:10604000002A00F0258102339AF88A27D507BAF88A
:10605000282848BF0433D40748BF0A33900748BFF5
:106060001433D10548BF2833550748BF643354065D
:1060700048BF03F57A63102100240422CDF80330D1
:106080008DF800108DF801408FE0DAF8203ACDF855
:1060900003301022002401238DF802308DF80020F7
:1060A000DAF834378DF80140684698473C7050E67E
:1060B0009AF8EC37002B40F02F811022092163E77A
:1060C0009AF8E0379B077FF5D7AD414ADAF83437C5
:1060D0009268CDF80320102220218DF8002008229C
:1060E0008DF801108DF802206846002498473C7016
:1060F000002E7FF430ADC2E5FF20FFF749F90028FC
:106100003FF4BAADB0F90C303249DAF83427897E61
:1061100003EB830303EB83031020490800249B0057
:1061200093FBF1F305218DF80000CDF803308DF8D5
:1061300001408DF80210684690473C70002E7FF4B5
:106140000AAD9CE5BAF92E38CDF803301021302283
:1061500052238DF802308DF80010DAF834378DF8BC
:1061600001206846002498473C70A6E5A4F1710020
:10617000C0B2FFF70DF900283FF47EAD90F9013071
:10618000E8E6114B93ED170AD3ED027A20EE270AC9
:10619000002420EE080A54F049FD1023CDF8030036
:1061A00007228DF800308DF80130DAF834378DF899
:1061B0000220684698473C70002E7FF4CCAC5EE528
:1061C00054040020F4050020C40B001067666666C6
:1061D000905A0020343100209AF8E0379C077FF570
:1061E0004BADC107814B40F1B5805A6882EAE2733A
:1061F000A3EBE27303EB5303A8FB0313DB08002AB2
:10620000ACBF43F0004343F0404310210024082278
:1062100034E7BAF93038DAF8342703EB83035B004C
:106220001020CDF80330402108238DF800008DF8B0
:1062300001108DF802306846002490473C70002E13
:106240007FF489AC1BE5BAF9E039CDF803301021B1
:10625000012204238DF802308DF80010DAF834376B
:106260008DF801206846002498473C7025E58AF89F
:106270001C1A012511E65E490620FFF731FA0023BA
:106280008AF81A0A3B7002B0BDEC028BBDE8F087B9
:106290000133D9E6554A9AF8E017538A643BC3EBB9
:1062A0004370C3EBC00389FB03401844DB17C3EB07
:1062B00020230933092BA8BF092323EAE37303EB47
:1062C000830311F0020F03EB830314BF4FF47A70C2
:1062D00000209B00C90748BF00F5FA60117DDAF87D
:1062E00034279BB203440B44042010218DF8020094
:1062F000CDF803308DF800108DF8011068460024A9
:1063000090473C70002E7FF426ACB8E401238AF855
:10631000243A42F2107391E6BAF8E427B2FBF3F3A1
:10632000CBE69AF8EC27002A57D113462AE63C70B0
:1063300002B0BDEC028BBDE8F0879AF84637002B1F
:106340003FF49AAC9AF82C3A032B49D8DFE803F0D3
:106350003B3122111A6882EAE273A3EBE27303EB8A
:106360005303A8FB0313DB08002AB8BF43F08043A4
:106370004BE7DAF8302A537A907AD17A03F14073F6
:1063800003EB0023002203EB01438AF82C2A10229E
:106390000421F9E5174A11688A7D087C897A12047C
:1063A00002EB00220A44591C8AF82C1A02EB036300
:1063B000EDE7104A11684A7DC87B497A120402EB66
:1063C00000220A44EFE70B4A11680A7D887B097AAC
:1063D000120402EB00220A44E5E7B3FBF2F3D1E535
:1063E0005A1C8AF82C2A1B06D1E700BF905A0020BD
:1063F000811A0108185B0020CA4A38B5082000231A
:1064000082F8A531FBF712FC002800F08C80D2F84E
:10641000A0314FF4806102204FF48264198082F829
:10642000A50101465C804FF40020FBF7FFFB50B153
:106430004B1CD2F8A001DBB240F2014482F8A53136
:1064400020F811401946B84C94F80938002B6CD14B
:1064500094F80A38002B40F088804FF40070FBF766
:10646000E5FB50B14B1CD2F8A001DBB24FF4046540
:1064700082F8A53120F811501946D4F87045A507C7
:1064800000F10181600700F1DB80A84B1B681B064F
:1064900000F1938000234FF4803082F8A41182F839
:1064A000A53182F89D31FBF7C1FBD0B3D2F898310A
:1064B00001214FF4047082F89D1118804FF40040C0
:1064C000FBF7B4FB50B14B1CD2F89801DBB24FF490
:1064D000007482F89D3120F8114019464FF40030C5
:1064E000FBF7A4FB50B14B1CD2F89801DBB24FF480
:1064F000A06482F89D3120F8114019464FF48020A5
:10650000FBF794FB38B1D2F898014FF437644B1C79
:1065100020F81140D9B2002382F89C1182F89D31F5
:1065200038BD0146CAE701467DE70120FBF77EFB47
:1065300000288DD04FF48030FBF778FBD2F8A051C3
:1065400028B94FF4047325F811300131C9B20BB2E8
:10655000481CC1B24FF4116082F8A51125F8130050
:1065600094F80A38002B3FF478AF0220FBF75EFB6B
:1065700000283FF472AF4FF40040FBF757FB50B9CF
:106580004B1CD2F8A001DBB24FF4007582F8A531A4
:1065900020F8115019460420FBF748FB00283FF46F
:1065A0005CAF4B1CD2F8A001DBB24FF4C06582F89F
:1065B000A53120F8115019464FE74FF40050FBF772
:1065C00035FB50B14B1CD2F8A001DBB24FF4036491
:1065D00082F8A53120F8114019464FF48050FBF79E
:1065E00025FB68B1D2F8A0014B1C4FF40064DBB26C
:1065F0008D1C20F81140E9B282F8A51120F8134053
:106600004FF48040FBF712FB50B14B1CD2F8A001B5
:10661000DBB24FF4846482F8A53120F811401946AA
:106620004FF48060FBF702FB00283FF433AFD2F851
:10663000A0014FF402644B1C20F81140D9B229E7A5
:106640004FF48060FBF7F2FA50B14B1CD2F8A00176
:10665000DBB24FF4807482F8A53120F8114019465E
:106660004FF40060FBF7E2FA00283FF40EAF4B1C3A
:10667000D2F8A001DBB24FF4887482F8A53120F87B
:106680001140194601E78020FBF7D0FA50B14B1CAE
:10669000D2F8A001DBB245F2302582F8A53120F80E
:1066A000115019464FF48070FBF7C0FA50B14B1CE3
:1066B000D2F8A001DBB245F2402582F8A53120F8DE
:1066C000115019461020FBF7B1FA50B14B1CD2F80B
:1066D000A001DBB24FF4E06582F8A53120F811503B
:1066E00019462020FBF7A2FA50B14B1CD2F8A001AA
:1066F000DBB24FF4E26582F8A53120F8115019465B
:106700004020FBF793FA00283FF4BCAE4B1CD2F8B4
:10671000A001DBB24FF4E46582F8A53120F81150F6
:106720001946AFE65404002038A70020585900202D
:1067300030B5A0F17D03012B044683B00D46104611
:1067400008D9214633F0EEFE15B1288804442C8088
:1067500003B030BD7D21019233F0E4FE019884F056
:10676000200133F0DFFEEFE730B50F4B85B0D3F8F3
:106770007C2700230446C51DADF80E3014F8010B2C
:1067800001920DF10E01FFF7D3FFA542019AF5D159
:106790000DF10E0014F040FF019A9DF80E0000214B
:1067A000FFF7C6FF05B030BD38A700207E28F8B53A
:1067B0000F4652D0324E96F8A84164B9314D95F843
:1067C0003C1A51B11B2885F83C4A3DD00D2837D0E2
:1067D000012386F8A8310020F8BD7D284AD095F81D
:1067E000402A1AB180F0200085F8401A95F83B2A1B
:1067F000062A14D8B5F83E4A511C2A440444C9B2AA
:10680000A5F83E4A85F83B1A82F8340A002BE2D1FB
:106810000729E0D101231C4886F8A831F8BDB5F856
:106820003E3A1844C0F3072353FA80F0FF284FF094
:106830000103A5F83E0A86F8A831CCD11248F8BD6C
:10684000A5F83E4A2046F8BD90470028C0D0012355
:1068500020463B7086F8A831F8BD0A4B084A002450
:10686000012183F83B4A83F83C1A3C7082F8A84126
:106870002046F8BD0123084685F8403AF8BD00BF20
:106880005404002038A700206CB10020044AD2F83C
:10689000443A43F4DF2343F48063C2F8443A704738
:1068A00038A70020013070B5094EC4B203E045F0AE
:1068B000C5FD013448B9E5B2152D21463046F6D95B
:1068C000162D04BF034B93F8485A284670BD00BFED
:1068D0007CB1002038A7002000B1D7E7044AD2F8E5
:1068E000443A23F4DF2323F48063C2F8443A704728
:1068F00038A7002070B5114C84B00546D4F84C0A76
:106900000E462CF0C5F994F8402794F84137003A28
:1069100018BF01220BB142F00802CDE90162002349
:106920004FF4964195F9000000911A4608212CF089
:1069300054FAC4F84C0A04B070BD00BF38A7002058
:1069400010B5064C03E0D4F84C0A33F0DFFDD4F860
:106950004C0A33F0E3FD0028F5D110BD38A7002024
:1069600010B50D4CD4F8503A1B791E3B012B0DD9B4
:10697000D4F84C0A01213830FFF7BCFF0023C4F8DB
:10698000543A84F8583ABDE81040D9E7D4F84C0A94
:10699000012133F0B3FDF1E738A70020F0B5C64C74
:1069A00094F8603AD4F87015C4F85C0A013388078B
:1069B00085B084F8603A12D411F0340F34D109074D
:1069C00094F8602A41D412F007055AD0282A00F022
:1069D000BA80D4F838375E20984705B0F0BD7020F3
:1069E000FBF724F90028E7D0B44E2425A6F1580778
:1069F000F6EC017A97ED027A67EE877A2846FDEE8B
:106A0000E77A013517EE901AC1EB411301EB8301D0
:106A1000C90009B2EDB2FBF76BF8272DE8D1D4F825
:106A2000701511F0340FCAD04FF40060FBF7FEF878
:106A3000002840F0058194F8602A12F0030100F06C
:106A4000DB80D4F870150907BDD54FF40070FBF753
:106A5000EDF80028B7D012F00305B4D1984AB4F984
:106A60003038D91782FB0323C1EBA30109B21420EC
:106A7000FBF73EF829461C20FBF73AF894F8602A09
:106A8000A1E7FF20FEF784FC002800F0DF800378F8
:106A9000FF2B7AD090F901100220FBF729F8FF2094
:106AA000FEF776FC002872D00378FF2B6FD0B0F988
:106AB0000C20844B8248997E02EB820202EB820218
:106AC0009300490893FBF1F3D91780FB0320C1EB36
:106AD000A00001B20320FBF70BF894F80938002B53
:106AE0005DD1D4F870359A067AD54FF40050FBF793
:106AF0009DF8002840F0C980734D4FF48060FBF78B
:106B000095F8002840F04C816B8A94F8602A297D22
:106B1000B3F5967F02D9100740F1118194F84337FD
:106B2000002B40F0958009B20520FAF7E1FF4FF401
:106B30008050FBF77BF8002840F0D88094F8602A5A
:106B4000282A7FF446AF614A614B15686149A3FB6F
:106B50000535AD09A1FB05367609A1FB06314909CA
:106B6000C1EB0111A6EB81010902C6EB0616002359
:106B700009B21720A5EB860684F8603AFAF7B8FF49
:106B800031B21820FAF7B4FF23E7294684E7002141
:106B90000320FAF7ADFF94F80938002BA1D00120AB
:106BA000FBF744F8002840F00D8194F80A38002BD8
:106BB00097D00220FBF73AF8002840F05C810420CF
:106BC000FBF734F800288CD0B4F80C38002B00F018
:106BD0005F8129F003FF01B20420FAF789FF80E703
:106BE0001B07ABD53C4B93E8030002AB83E80300E3
:106BF0001846FAF793FFA1E74FF48060FBF716F809
:106C000000283FF41EAF354BD4F85C2AD4F8205A44
:106C10009A4240F20D81324BE91783FB0523C1EB09
:106C20006313642101FB13510DB219B21020FAF75E
:106C30005FFF29462120FAF75BFF94F8602A00E7FE
:106C4000B4F932183020FAF753FFF4E6014623E78F
:106C5000A1F1200307EE903A9FED227AF8EEE77A51
:106C6000F6EE006A67EE877ABEEE007AF5EEC07A3D
:106C7000F1EE10FA58BFB0EE667A77EE877AFDEE45
:106C8000E77A17EE903A19B24EE794F8E0379F078B
:106C90005BD44FF48060FAF7C9FF0B4D00283FF436
:106CA00033AF002631460120FAF722FF3146092092
:106CB000FAF71EFF28E700BF38A700201C0C0010C1
:106CC0006766666634310020905A0020C024002098
:106CD000D34D6210898888885CDD06083F4B4C00E4
:106CE0001F85EB51E4380E3F0050C34794F8E0276E
:106CF00000239207CDE9003347D494F8643A012B7E
:106D000043D0B4F93C375FED086A07EE103AB4F9A6
:106D10003E3707EE903AB8EEC77AF8EEE77A27EEFC
:106D2000267A67EEA67ABDEEC77AFDEEE77A02A86C
:106D30008DED027ACDED037AFAF7F0FEFEE642F22F
:106D40000F719942A8BF1946E8E6544D544BE989A2
:106D50004FF4F36606FB01F14909A3FB0131C909B0
:106D60001120FAF7C5FEE9894E4B06FB01F1A3FBA2
:106D700001214909A3FB01235B09642202FB1311D2
:106D800009B21920FAF7B4FEB7E6D5E900230121CC
:106D90006846CDE9002384F8641AFAF7BFFECDE611
:106DA00094F8E0379E077FF57CAFAB683D4AD91772
:106DB00082FB0302C1EB6211642606FB113636B278
:106DC00009B270E794F8EC1700293DD10B46062074
:106DD000A4F8623AFAF78CFEB4F8623A0133A4F8E8
:106DE000623A29F0EFFD94F8443794F8EC27012B30
:106DF00094F847371ED000EB800086B213B10AB179
:106E0000B6FBF2F6274BA3FB062343F34F113A20C0
:106E10005D09FAF76DFE642101FB1561224B89B211
:106E20000531A3FB0131C9083B20FAF761FEBCE63E
:106E30000D46FBE61BB112B1B0FBF2F080B201B21D
:106E40003920FAF755FEB0E6B4F8620AB4F8E42740
:106E5000B0FBF1F301FB1303642000FB02129BB2B1
:106E60004900B2FBF1F2110241EA0311C2F303221D
:106E7000114309B2ABE7D4F81C380C49DA1781FB8F
:106E80000313C2EBA30319B22820FAF731FE96E6EA
:106E9000D4F8243883F3100319B29DE6905A0020E9
:106EA000C55A7C0A1F85EB51CDCCCCCC6766666693
:106EB0000B2814D810B401EB4103094C01EB8303F8
:106EC0002344184490F84438934205D021440023C9
:106ED00080F8442881F838385DF8044B70477047D3
:106EE00038A70020F0B5454C94F8653A012B83B0E3
:106EF00005464FD994F8660A4149424E94F8677A9C
:106F0000421CA1FB02C1184406EB800001F4FE768E
:106F100006EB9101521A466C84F8662A2FB1D4F818
:106F2000681A04F66C2291420DD06EB9364A0133CC
:106F3000A2FB031222F0010101EB52029B1A84F81A
:106F4000653A03B0F0BD314E94F8803A93B9304BB6
:106F5000019348F2A501123B15226F46A4F8841A4A
:106F6000009384F8862A29463846B04758B994F8E1
:106F7000653ADBE76F46384611F07CFB2946384618
:106F8000B0470028F3D094F8801A51B1384611F078
:106F9000EBFAECE71B4A02EB8302566C002EC5D0DD
:106FA000D2E7009E1B4A964214D9013A013E41F2B3
:106FB000210512F8013F81EA0321082311F4004F53
:106FC00085EA41000ABF490081B289B2013BF5D18F
:106FD0009642EED138463BF0C1FD0F49009D6D1A37
:106FE000152DA8BF15252A4601F1180056F022F9E3
:106FF00094F8653A84F8B15A98E700BF38A70020A2
:10700000CDCCCCCC20DD0608ABAAAAAAC9270108A2
:10701000D1B10020BFB10020BCB1002070B50B4E33
:10702000054606F6B62141F047F82C686C6006F676
:10703000B421641A402CA8BF40242960224606F6D9
:10704000F42056F0F7F886F8344B70BD38A70020CE
:1070500030B50C4B0C4AC3F8B42A83B0C8220146A1
:1070600003F6F42503F6B92483F8B82A68463A22D1
:10707000CDE900453BF02AFD6846FFF7CFFF03B09E
:1070800030BD00BF38A70020C83E7BEA03685A061F
:1070900007D513F4057F04D007298CBF00200120F9
:1070A000704703F48253B3F5825F03BFC81FB0FA81
:1070B00080F040090020704770B5BC4C94F8353B17
:1070C000012B84B000F04C8194F8410BFCF71EF8C2
:1070D00094F8423B834205461FD0002800F0D5803B
:1070E000D4F8503ACBB194F8412793F90400002A20
:1070F00018BF08224FF4964100230325CDE9015221
:1071000000911A4608212BF068FEC4F84C0A20B101
:10711000FFF726FC012384F8423B94F8433B012B04
:1071200000F0C080D4F84C6B3EB1A14B304659788A
:10713000FFF7ACFF002840F0F18094F8510BFBF70B
:10714000E5FF94F8503B8342054621D0002800F02B
:10715000F580EEB1337A002B00F01781954A02EBEF
:1071600083031B6E94F8402796F904000093003ABD
:1071700018BF012202210023CDE901121A46102175
:107180002BF02BFEC4F8140A10B1012384F8503BF5
:10719000D4F8546B3EB1864B30465978FFF776FFF2
:1071A000002840F0AB8094F8600BFBF7AFFF94F839
:1071B000583B8342054622D0002800F0C880F6B133
:1071C000337A002B00F0E4807A4A02EB83031B6ED3
:1071D00094F8402796F904000093003A18BF012262
:1071E00002210023CDE901121A464FF400712BF061
:1071F000F4FDC4F85C0B10B1012384F8583B94F8FB
:10720000610BFBF783FF94F8623B8342054630D065
:1072100088B3694BD4F8646B4FF47A72C3F8BC2618
:107220003EB34FF48052402130462BF061FD0546BD
:10723000F8B994F8403796F90400002B14BF0921DF
:10724000082103224FF4E133CDE9012100932A46BE
:107250002B464FF480512BF0C0FDC4F8680B40B1B1
:107260000123C4F8080A84F8E25984F86C5B84F8B6
:10727000623B04B070BDD4F8680B2BF009FDC4F874
:10728000685B84F8625B04B070BDD4F84C0A2BF0E4
:10729000FFFC94F8433BC4F84C5A012B84F8425B42
:1072A0007FF440AF94F8440BFBF730FF054600280D
:1072B00071D0D4F87C37002B7FF434AFD4F8482B4E
:1072C000002A3FF42FAF94F8415794F8401792F9F1
:1072D0000400002D14BF08220022002908BF42F03C
:1072E000010203254FF46141CDE9015200911A4694
:1072F00020212BF072FDC4F87C0713E794F8583B6B
:10730000002B7FF47CAFD4F83C3B002B3FF477AFED
:107310000122C4F85C3B84F8582B70E794F8503B8A
:10732000002B7FF435AFD4F83C3B002B3FF430AF5B
:107330000122C4F8143A84F8502B29E7D4F8140A2F
:107340002BF0A6FCC4F8145A84F8505B20E7D4F85C
:107350005C0B2BF09DFCC4F85C5B84F8585B4EE73B
:10736000D4F8385B124B28465978FFF78FFE28B3C4
:10737000D4F8DC37002B7FF4A7AED4F83C3B002BCD
:107380003FF4A2AEC4F8DC379EE64FF49643E9E63C
:107390004FF461431CE7D4F87C0700283FF4C2AEE9
:1073A0002BF076FCC4F87C57BCE600BF38A7002061
:1073B0001C56002020DD06085404002094F8400BE1
:1073C000FBF7A4FE0646D8B1D4F8DC37002B7FF4D7
:1073D0007BAE002D3FF478AE94F8402795F9040079
:1073E000B2FA82F252094FF416510225CDE9015248
:1073F00000911A4604212BF0F0FCC4F8DC0763E688
:10740000D4F8DC0700283FF45FAE2BF041FCC4F851
:10741000DC6759E670B5B14C94F8353B002B00F0B1
:10742000218108202BF078FCC4F8500A00283BD0BA
:1074300008212BF067FC00260346A949A94884F8D7
:10744000413BC4F8746B37F01DFB41F20853012235
:10745000A448A4F8783B84F87C2B0DF065FC3146F9
:107460002B22A14855F047FF48F67C607D25E0239C
:1074700031462B22A4F8840B9C4884F8873B84F87F
:10748000AF5B55F038FF48F67C21A0224EF27B031B
:1074900084F8DB5B84F8DE6B84F8875CA4F8B01BAF
:1074A00084F8B32BA4F8DC3B94F8433B002B00F0AA
:1074B000C38010202BF030FC1021C4F84C0B2BF0B3
:1074C00021FC8B4B84F8510B3A2140F23B1094F88D
:1074D000092818809F254AF21E40197100219D71CC
:1074E00098601973002A40F08E8094F80A38002BB7
:1074F00048D1D4F8703558077ED4990773D41A0749
:107500006AD47C4D2868C0F3C010FFF7E5F900206D
:10751000FFF7C8F903464FF4007084F8483A2BF09F
:10752000FBFB4FF40071C4F8540B2BF0EBFBD4F8C9
:10753000883C84F8600B002B14BF0123002384F8DF
:107540008C3C26D1D4F8FC2C0023C4F8F83C002A4B
:1075500069D0012284F8803A84F8002D4FF48050DD
:107560002BF0DAFB4FF48051C4F8640B2BF0CAFB0C
:10757000002384F8610B84F8623BFAF75BFABDE8FC
:10758000704099E5D4F8443A43F00403C4F8443A0F
:10759000AFE7D4F87025002312F0020284F88D3C86
:1075A00084F88E3C40F0828094F8093823B10120A1
:1075B000FAF73CFB002873D194F80A38002B6AD103
